:020000040800F2
:1000000000A0002051BE0008A1BE0008A1BE00084B
:10001000A1BE0008A1BE0008A1BE000800000000AB
:10002000000000000000000000000000A1BE000869
:10003000A1BE000800000000A1BE000867A30008E0
:10004000A1BE0008A1BE0008A1BE0008A1BE000814
:10005000A1BE0008A1BE000825A500082BA5000828
:1000600031A5000837A500083DA50008A1BE00087D
:10007000A1BE0008A1BE0008A1BE0008A1BE0008E4
:10008000A1BE0008A1BE0008A1BE0008000000003B
:1000900000000000000000000000000043A5000870
:1000A000759D0008159D0008A1BE0008399D000837
:1000B0004D9D00080000000000000000A1BE0008E7
:1000C000A1BE0008A1BE0008A1BE0008A1BE000894
:1000D000A1BE0008C1AF0008D9AF0008F5AF000805
:1000E00059A50008A1BE00080000000000000000A3
:1000F0000000000000000000000000000000000000
:1001000000000000000000000000000000000000EF
:100110000000000000000000619D000800000000D9
:10012000A1BE0008A1BE0008A1BE0008A1BE000833
:10013000A1BE000800000000000000000000000058
:10014000A1BE0008A1BE0008A1BE0008A1BE000813
:10015000A1BE0008A1BE000811B00008A1BE0008A1
:10016000A1BE0008A1BE00080000000000000000C1
:1001700000000000A1BE0008000000000000000018
:0C018000A1BE0008A1BE0008A1BE00083E
:1001900010F8012B11F8013B012A28BF9A42F7D031
:1001A000D01A7047034613F8012B002AFBD1181A06
:1001B000013870470000000000000000000000004F
:1001C00001F0FF01102A2BDB10F0070F08D010F808
:1001D000013B013A8B422DD010F0070F42B3F6D10C
:1001E000F0B441EA012141EA014122F007047FF025
:1001F00000070023F0E80256083C85EA010586EA7C
:10020000010685FA47F5A3FA87F586FA47F6A5FAB7
:1002100087F68EB9EED1F0BC01F0FF0102F00702C3
:1002200032B110F8013B013A83EA010313B1F8D16E
:100230000020704701387047002D06BF354603384F
:10024000073815F0010F07D1013015F4807F02BF88
:10025000013015F4C03F0130F0BC0138704700BFD9
:1002600081F0004102E000BF83F0004330B54FEA67
:1002700041044FEA430594EA050F08BF90EA020FD4
:100280001FBF54EA000C55EA020C7FEA645C7FEA67
:10029000655C00F0E2804FEA5454D4EB5555B8BF8A
:1002A0006D420CDD2C4480EA020281EA030382EAFB
:1002B000000083EA010180EA020281EA0303362D8D
:1002C00088BF30BD11F0004F4FEA01314FF4801C60
:1002D0004CEA113102D0404261EB410113F0004F72
:1002E0004FEA03334CEA133302D0524263EB430329
:1002F00094EA050F00F0A780A4F10104D5F1200EC7
:100300000DDB02FA0EFC22FA05F2801841F1000121
:1003100003FA0EF2801843FA05F359410EE0A5F1F5
:1003200020050EF1200E012A03FA0EFC28BF4CF026
:10033000020C43FA05F3C01851EBE37101F00045DC
:1003400007D54FF0000EDCF1000C7EEB00006EEBE9
:100350000101B1F5801F1BD3B1F5001F0CD3490873
:100360005FEA30004FEA3C0C04F101044FEA4452CA
:1003700012F5800F80F09A80BCF1004F08BF5FEA51
:10038000500C50F1000041EB045141EA050130BD31
:100390005FEA4C0C404141EB0101013C28BFB1F543
:1003A000801FE9D291F0000F04BF01460020B1FA8E
:1003B00081F308BF2033A3F10B03B3F120020CDA61
:1003C0000C3208DD02F1140CC2F10C0201FA0CF03F
:1003D00021FA02F10CE002F11402D8BFC2F1200CA4
:1003E00001FA02F120FA0CFCDCBF41EA0C0190405A
:1003F000E41AA2BF01EB0451294330BD6FEA0404A3
:100400001F3C1CDA0C340EDC04F11404C4F120028D
:1004100020FA04F001FA02F340EA030021FA04F39F
:1004200045EA030130BDC4F10C04C4F1200220FAF6
:1004300002F001FA04F340EA0300294630BD21FA34
:1004400004F0294630BD94F0000F83F4801306BFFA
:1004500081F480110134013D4EE77FEA645C18BFEE
:100460007FEA655C29D094EA050F08BF90EA020F85
:1004700005D054EA000C04BF1946104630BD91EA7D
:10048000030F1EBF0021002030BD5FEA545C05D180
:100490004000494128BF41F0004130BD14F58004BF
:1004A0003CBF01F5801130BD01F0004545F0FE4133
:1004B00041F470014FF0000030BD7FEA645C1ABF68
:1004C000194610467FEA655C1CBF0B46024650EA9F
:1004D000013406BF52EA033591EA030F41F40021CB
:1004E00030BD00BF90F0000F04BF0021704730B551
:1004F0004FF4806404F132044FF000054FF0000126
:1005000050E700BF90F0000F04BF0021704730B5E6
:100510004FF4806404F1320410F0004548BF4042BB
:100520004FF000013EE700BF42004FEAE2014FEA10
:1005300031014FEA02701FBF12F07F4393F07F4FEB
:1005400081F06051704732F07F4208BF704793F0EE
:100550007F4F04BF41F40021704730B54FF4607401
:1005600001F0004521F000411CE700BF50EA010204
:1005700008BF704730B54FF000050AE050EA0102AD
:1005800008BF704730B511F0004502D5404261EB1D
:1005900041014FF4806404F132045FEA915C3FF45E
:1005A000D8AE4FF003025FEADC0C18BF03325FEAFB
:1005B000DC0C18BF033202EBDC02C2F1200300FAAC
:1005C00003FC20FA02F001FA03FE40EA0E0021FAD1
:1005D00002F11444BDE600BF70B54FF0FF0C4CF4BF
:1005E000E06C1CEA11541DBF1CEA135594EA0C0F71
:1005F00095EA0C0F00F0DEF82C4481EA030621EAAC
:100600004C5123EA4C5350EA013518BF52EA0335E6
:1006100041F4801143F4801338D0A0FB02CE4FF098
:100620000005E1FB02E506F00042E0FB03E54FF0C8
:100630000006E1FB03569CF0000F18BF4EF0010EC0
:10064000A4F1FF04B6F5007F64F5407404D25FEABC
:100650004E0E6D4146EB060642EAC62141EA55516F
:100660004FEAC52040EA5E504FEACE2EB4F1FD0CB1
:1006700088BFBCF5E06F1ED8BEF1004F08BF5FEA2F
:10068000500E50F1000041EB045170BD06F00046E1
:1006900046EA010140EA020081EA0301B4EB5C048E
:1006A000C2BFD4EB0C0541EA045170BD41F4801186
:1006B0004FF0000E013C00F3AB8014F1360FDEBFAB
:1006C000002001F0004170BDC4F10004203C35DA87
:1006D0000C341BDC04F11404C4F1200500FA05F30A
:1006E00020FA04F001FA05F240EA020001F00042AB
:1006F00021F0004110EBD37021FA04F642EB060121
:100700005EEA430E08BF20EAD37070BDC4F10C044A
:10071000C4F1200500FA04F320FA05F001FA04F20E
:1007200040EA020001F0004110EBD37041F10001FA
:100730005EEA430E08BF20EAD37070BDC4F1200505
:1007400000FA05F24EEA020E20FA04F301FA05F26D
:1007500043EA020321FA04F001F0004121FA04F215
:1007600020EA020000EBD3705EEA430E08BF20EAE5
:10077000D37070BD94F0000F0FD101F0004640001F
:1007800041EB010111F4801F08BF013CF7D041EAA1
:10079000060195F0000F18BF704703F000465200A5
:1007A00043EB030313F4801F08BF013DF7D043EA76
:1007B0000603704794EA0C0F0CEA135518BF95EA2C
:1007C0000C0F0CD050EA410618BF52EA4306D1D1B3
:1007D00081EA030101F000414FF0000070BD50EAD2
:1007E000410606BF1046194652EA430619D094EA5C
:1007F0000C0F02D150EA013613D195EA0C0F05D146
:1008000052EA03361CBF104619460AD181EA030199
:1008100001F0004141F0FE4141F470014FF0000051
:1008200070BD41F0FE4141F4780170BD70B54FF0EC
:10083000FF0C4CF4E06C1CEA11541DBF1CEA13556C
:1008400094EA0C0F95EA0C0F00F0A7F8A4EB05044E
:1008500081EA030E52EA03354FEA013100F0888045
:100860004FEA03334FF0805545EA131343EA12630E
:100870004FEA022245EA111545EA10654FEA0026C3
:100880000EF000419D4208BF964244F1FD0404F57C
:10089000407402D25B084FEA3202B61A65EB0305D8
:1008A0005B084FEA32024FF480104FF4002CB6EB95
:1008B000020E75EB030E22BFB61A754640EA0C0015
:1008C0005B084FEA3202B6EB020E75EB030E22BF55
:1008D000B61A754640EA5C005B084FEA3202B6EB96
:1008E000020E75EB030E22BFB61A754640EA9C0055
:1008F0005B084FEA3202B6EB020E75EB030E22BF25
:10090000B61A754640EADC0055EA060E18D04FEAE2
:10091000051545EA16754FEA06164FEAC30343EA82
:1009200052734FEAC2025FEA1C1CC0D111F4801F4F
:100930000BD141EA00014FF000004FF0004CB6E748
:1009400011F4801F04BF01430020B4F1FD0C88BFE7
:10095000BCF5E06F3FF6AFAEB5EB030C04BFB6EBF2
:10096000020C5FEA500C50F1000041EB045170BDE5
:100970000EF0004E4EEA113114EB5C04C2BFD4EB12
:100980000C0541EA045170BD41F480114FF0000E96
:10099000013C90E645EA060E8DE60CEA135594EA12
:1009A0000C0F08BF95EA0C0F3FF43BAF94EA0C0F15
:1009B0000AD150EA01347FF434AF95EA0C0F7FF48A
:1009C00025AF104619462CE795EA0C0F06D152EADE
:1009D00003353FF4FDAE1046194622E750EA4106C2
:1009E00018BF52EA43067FF4C5AE50EA41047FF4D3
:1009F0000DAF52EA43057FF4EBAE12E74FF0FF3C38
:100A000006E000BF4FF0010C02E000BF4FF0010C08
:100A10004DF804CD4FEA410C7FEA6C5C4FEA430C81
:100A200018BF7FEA6C5C1BD001B050EA410C0CBFD0
:100A300052EA430C91EA030F02BF90EA020F002032
:100A4000704710F1000F91EA030F58BF994208BF99
:100A500090422CBFD8176FEAE37040F00100704756
:100A60004FEA410C7FEA6C5C02D150EA013C07D1AD
:100A70004FEA430C7FEA6C5CD6D152EA033CD3D0F8
:100A80005DF8040B704700BF8446104662468C46F2
:100A90001946634600E000BF01B5FFF7B7FF002825
:100AA00048BF10F1000F01BD4DF808EDFFF7F4FF4E
:100AB0000CBF012000205DF808FB00BF4DF808EDD9
:100AC000FFF7EAFF34BF012000205DF808FB00BFFC
:100AD0004DF808EDFFF7E0FF94BF012000205DF81E
:100AE00008FB00BF4DF808EDFFF7CEFF94BF0120D3
:100AF00000205DF808FB00BF4DF808EDFFF7C4FFCC
:100B000034BF012000205DF808FB00BF4FEA410C14
:100B10007FEA6C5C02D150EA013C0AD14FEA430CF7
:100B20007FEA6C5C02D152EA033C02D14FF0000034
:100B300070474FF0010070474FEA410212F5001272
:100B400015D211D56FF47873B3EB625212D94FEA14
:100B5000C12343F0004343EA505311F0004F23FAFE
:100B600002F018BF404270474FF00000704750EA53
:100B7000013005D111F0004008BF6FF00040704710
:100B80004FF00000704700BF4A0011D212F500126A
:100B900011D20DD56FF47873B3EB62520ED44FEAD5
:100BA000C12343F0004343EA505323FA02F0704755
:100BB0004FF00000704750EA013002D14FF0FF3093
:100BC00070474FF0000070474FEA4102B2F1E04336
:100BD00024BFB3F5001CDCF1FE5C0DD901F0004C24
:100BE0004FEAC0024CEA5070B2F1004F40EB830074
:100BF00008BF20F00100704711F0804F21D113F1A0
:100C00003872BCBF01F00040704741F480114FEAD8
:100C10005252C2F11802C2F1200C10FA0CF320FA61
:100C200002F018BF40F001004FEAC1234FEAD3237E
:100C300003FA0CFC40EA0C0023FA02F34FEA4303E8
:100C4000CCE77FEA625307D150EA01331EBF4FF071
:100C5000FE4040F44000704701F0004040F0FE408C
:100C600040F40000704700BF53B94AB9002908BFDB
:100C700000281CBF4FF0FF314FF0FF3000F00CB8E0
:100C8000ADF1080C6DE904CE0CF0F6FBDDF804E0E4
:100C9000DDE9022304B07047704700BF10B5054C72
:100CA000237833B9044B13B10448AFF30080012318
:100CB000237010BD40030020000000003CD7000856
:100CC00008B5034B1BB103490348AFF3008008BDCF
:100CD00000000000440300203CD70008C0000C22A4
:100CE00090FBF2F302FB130202B1013310300B222E
:100CF00002FB0303002B1846B8BFD81DC0105B07CA
:100D000018BF0130704700002DE9F047CB1D23F0DC
:100D1000070300AFADEB030DCD0006460C46914630
:100D200068460A4600210BF093FC1E4AADB2E84625
:100D30000123114632F8020FA8420ED3013B31F8CD
:100D400013C000210A46954209D822464146304642
:100D50000BF016FDBD46BDE8F0870133EAE7B1FBB5
:100D6000F5FA05FB1A1AB9F1000F19D1D6469246C9
:100D70004FEADA030AF0070AF35C4FEADE0043FAAF
:100D80000AF30EF0070E03F0010303FA0EF318F84E
:100D900000E043EA0E0308F8003001326144D2E774
:100DA0009646E5E700000020F0B5C9004FF49546EF
:100DB000002501278D4200DBF0BD4FEAE50C05F070
:100DC000070410F80CE086EA56024EFA04F302F02B
:100DD000010203F001035340A34007FA04F42EEA92
:100DE000040E43EA0E03920300F80C3042EA560662
:100DF0000135DFE7B0F5006F0FDA70475B10034293
:100E0000FCD0002B1A46B8BF03F2FF72D2124A433D
:100E10005040B0F5006FF2D270474FF4800340F6B7
:100E20007541ECE72DE9F74F064610469246FFF76D
:100E300055FF42F2244326F8023B002452468046E6
:100E400030468B4606EB0A070BF09AFCA1464FEAA8
:100E5000CA02254623460C21934239DB394BBAF1AD
:100E6000000FB8BF00225A43374BB3EBB20F14D276
:100E70004FEA69000003FFF7BDFF0B350A2240FA75
:100E800002F303F001032343AC1A14F007040CBF70
:100E900007F8013B5C00013AF1D215F0070308D0D6
:100EA0006D4205F0070558BF6B42C3F107039C4034
:100EB0003C70A8F10204002221463046FFF724FFCF
:100EC00030462146FFF770FF404603B0BDE8F08F83
:100ED000D8106FEA030C1BF800000CF0070C40FA66
:100EE0000CF0013300F0010049EA0000B3FBF1F916
:100EF00001FB1939B9F1000F02D04FEA4009ABE705
:100F0000C002CDE90032FFF775FFDDE900324FF096
:100F1000010E0C21CEF10B0C40FA0CFC0CF0010C74
:100F20004CEA040C05EB0E0414F007040EF1010E5C
:100F30000CBF07F801CB4FEA4C04BEF10C0FE9D10E
:100F40000B3589E7ABAAAAAA5555551538B54B1EDE
:100F50005C420D465C41072864D8DFE800F00426B7
:100F600036393C3F4D5B214613200BF0C3F8214638
:100F7000C3200BF0BFF821462D200BF0BBF8214613
:100F80002E200BF0B7F8214629200BF0B3F82146AC
:100F90002A200BF0AFF821462B200BF0ABF82146AE
:100FA0001C200BF0A7F821460AE0214613200BF085
:100FB000A1F821461C200BF09DF8691E18BF0121E5
:100FC000BDE83840C2200BF095B82146C320EEE7BB
:100FD00021462D20EBE721462E20E8E72146292057
:100FE0000BF088F8691E18BF01211C200BF082F855
:100FF0002146C2200BF07EF821462A200BF07AF819
:10100000691E18BF01211C200BF074F82146C22074
:101010000BF070F821462B200BF06CF8691E18BFFE
:101020000121BDE738BD006804F074BF04F02EBF95
:101030002DE9F043A1B0E9460546884600244F4615
:1010400008EB0406B6B23046FFF7F0FF68B904F1CA
:1010500080030DEB0304394604F8800C28460AF09F
:10106000D1FC284621B0BDE8F0833046FFF7DEFF13
:10107000013409F8010BE3E7F7B507460E460024F3
:10108000214630460AF0A4FD01783D19ADB229B9D8
:1010900001A80195FFF7C7FF03B0F0BD2146304618
:1010A0000AF096FD0178019501A8FFF7BCFF013415
:1010B000E6E738B50546FFF7B9FF0446681CFFF7B9
:1010C000B5FF04EB0024A81CFFF7B0FF04EB0044BD
:1010D000E81CFFF7ABFF04EB006038BD37B50D46E9
:1010E00004460190C9B201A8FFF79DFF631CC5F338
:1010F000072101A80193FFF796FFA31CC5F3074141
:1011000001A801930334FFF78EFF290E01A8019473
:10111000FFF789FF03B030BD38B50546FFF786FFFE
:101120000446681CFFF782FF44EA002038BD70B512
:10113000CEB204460D46FFF779FF864203D0314612
:10114000204604F0E7FE01342046FFF76FFFC5F3A9
:101150000725854205D029462046BDE8704004F0A9
:10116000D9BE70BDF8B52DED048BDFED2A8A04469B
:101170000026B2EE048A314620460AF029FD0378A3
:101180002E2B354606F1010615D0294620460AF0D9
:101190001FFD03787BB1294620460AF019FD03782C
:1011A00003F00F0307EE903AF8EEE77AE8EE887A5C
:1011B000F0EE678ADFE79FED178A0025B2EE049A0A
:1011C0007719394620460AF003FD03786BB9F2EE31
:1011D000047ADDB978EE887A17EE900AFFF7A4F961
:1011E000BDEC048B41EC100BF8BD394620460AF0EB
:1011F000EFFC037803F00F0307EE903AF8EEE77A7E
:101200000135E8EE097AB0EE678AD9E788EE278AD9
:10121000013DDEE70000000070B50C4E05460C46AF
:101220002C2000210AF066FF45F0800100223046A4
:1012300004F09EFC21463046002204F099FCBDE8F3
:10124000704001212C200AF055BF00BF880B002000
:1012500008B500210620FFF7DFFF01210720FFF777
:10126000DBFF7F210920FFF7D7FF05210A20FFF7C9
:10127000D3FFF4210B20FFF7CFFFEF210C20FFF766
:10128000CBFF00210D20FFF7C7FF00210E20FFF745
:10129000C3FF80210F20FFF7BFFF00211020FFF7C1
:1012A000BBFF20211220FFF7B7FF00211320FFF71B
:1012B000B3FF20217020FFF7AFFF1D211C20FFF797
:1012C000ABFF40211D20FFF7A7FFA1212020FFF742
:1012D000A3FF20212120FFF79FFF4E212220FFF7AF
:1012E0009BFFA5212320FFF797FF00212420FFF774
:1012F00093FF0A212520FFF78FFF00212C20FFF705
:101300008BFF00212D20FFF787FF00212E20FFF704
:1013100083FF27216E20FFF77FFF52216F20FFF709
:101320007BFF8C213020FFF777FFFF213220FFF772
:1013300073FF42213320FFF76FFF40213420FFF776
:101340006BFF20213520FFF767FF2D213620FFF7A7
:1013500063FFD4213720FFF75FFF73213A20FFF7A7
:101360005BFF6F213B20FFF757FF6E213C20FFF70B
:1013700053FF67213D20FFF74FFF334B3E20197885
:10138000FFF74AFF73213F20FFF746FF6F21402000
:10139000FFF742FF6E214120FFF73EFF6721422009
:1013A000FFF73AFFFF214320FFF736FFFF214420DC
:1013B000FFF732FFFF214520FFF72EFFFF214620D8
:1013C000FFF72AFF01215620FFF726FF07216D2096
:1013D000FFF722FF00217920FFF71EFF00217A206E
:1013E000FFF71AFF08217220FFF716FF0021732074
:1013F000FFF712FF00217420FFF70EFF2121752057
:10140000FFF70AFF18217620FFF706FF0A21772051
:10141000FFF702FF7F215A20FFF7FEFE40215920EF
:10142000FFF7FAFE80215820FFF7F6FE0B216A2015
:10143000FFF7F2FE04216820FFF7EEFEBDE808404A
:1014400003211F20FFF7E8BEA00100204B21072049
:10145000FFF7E2BE43210720FFF7DEBE4021072051
:10146000FFF7DABE00217120FFF7D6BE38B50C4D6C
:10147000044600212C200AF03DFE04F07F010022EA
:10148000284604F075FB00221146284604F070FB44
:10149000012104462C200AF02DFE204638BD00BF55
:1014A000880B0020000000002DE9F04710EE100A24
:1014B000FFF73AF838A3D3E9002306460F46FFF7B3
:1014C0008BF8314B002204460D46FFF70BFB2F4BE8
:1014D000B0F1000A4FF000022046294618BF4FF035
:1014E000010AFFF7A3F9FFF74FFB5FFA8AF84FFAFB
:1014F0008AFABAF1000F08F10109C4B214BF6FF003
:10150000170300234846183C1C44FEF7FBFF94FBDE
:10151000F9F41BA3D3E90023FFF75EF802460B465C
:1015200030463946FFF782F90646E0B20F46FEF72D
:10153000E9FF02460B4630463946FEF795FE144B4E
:101540000022FEF791FE134B0022FFF745F8FFF74C
:101550001BFB04F01F0141EA481185B241F0400134
:101560007520FFF759FE290A7620FFF755FEE9B2EC
:101570007720BDE8F047FFF74FBE00BFAFF3008014
:10158000555555555555214000007E4000002440DA
:10159000000038400040EF40622776622776F23F35
:1015A00000F007016D20FFF737BE01467320FFF7FB
:1015B00033BE03280DD8DFE800F00204080AFFF765
:1015C00051BF11217120FFF727BE1221FAE7222116
:1015D000F8E70021F6E7000008B5A0B10B4B18684A
:1015E0000130C0B2FFF7E1FF094B0A4A1B68B3FBA9
:1015F000F2F3094A09491268486853434A68121AC3
:101600009342FBDC08BD0120ECE700BF1002002084
:10161000D402002040420F001C020020001000E015
:10162000104B1868013010B5C0B2FFF7BEFF0E4B6B
:101630000E49D3ED007A0E4B0E4A93ED007A4868BE
:1016400012680D4CB2FBF4F2F8EEE77A67EE877A97
:10165000FDEEE77A17EE903A53434A68121A934226
:10166000FBDC10BD100200201C020020001000E076
:1016700014020020D402002040420F0070B505463D
:101680000020FFF7A9FF084E00243368A34203DCC3
:10169000BDE87040FFF7C4BF45FA04F000F0010058
:1016A000FFF79AFF0134F0E71802002010B5044656
:1016B0000120FFF791FF64200AF05AFD013C14F865
:1016C000010F00B910BDFFF7D9FFF8E7022808B5F0
:1016D00016D0032816D0012814BF01200220FFF7DE
:1016E00064FF094B094A1B68B3FBF2F3084A094936
:1016F0001268486853434A68121A9342FBDC08BDDB
:101700000320ECE70420EAE7D402002040420F0067
:1017100068030020001000E00020FFF7D7BF38B5B5
:1017200004460425A009FFF7D1FFA400013DE4B25F
:10173000F8D1012038BD38B505460024A54200DCAB
:1017400038BD1B20FFF7EBFF0134F7E770B5044607
:1017500046180025B44201D1284670BD14F8010B8B
:10176000FFF7DDFF0544F5E780EA0120082341F299
:10177000210200F40041400001B15040013BF8D18A
:10178000704738B5044645184FF6FF70AC4200D19B
:1017900038BD14F8011BFFF7E7FFF7E730B5024645
:1017A000014441F221054FF6FF708A4200D130BD5D
:1017B00012F8013B082480EA032003B2002BB4BFD7
:1017C00085EA4303430098B2631E13F0FF04F4D18B
:1017D000EBE7000010B5124B124C1B782DED028B7D
:1017E000C520B0EE088AA3B10AF0A2FB07EE900A6A
:1017F0009FED0D7AF8EE677A87EE870A20EE080AE9
:10180000BDEC028B30EE000AD4ED007A20EE270A00
:1018100010BD0AF08DFB00EE100ABBEECB0AEDE71F
:10182000710200209C01002000F07F4500000000B4
:1018300008B5C9200AF07CFB334B1B78002B45D040
:10184000FEF760FE24A3D3E90023FEF7C5FEFFF7F1
:10185000BBF9FEF769FE02460B4600202B49FEF756
:10186000E5FF2B4B0022FEF7FFFC1DA3D3E900236D
:10187000FEF7B2FEFFF7A8F99FED260A07EE900AE1
:1018800080EE270A0BF048FB10EE100AFEF74CFE24
:1018900015A3D3E90023FEF79FFE15A3D3E9002388
:1018A000FEF7E4FC02460B4600201949FEF7BEFF96
:1018B000FFF78AF9FEF738FE0FA3D3E90023FEF7FE
:1018C000D3FCFFF781F900EE100A08BDFEF71AFEFF
:1018D0000BA3D3E90023B8E7188001188001483F23
:1018E000000000000050C4407DB968C570842E3FE0
:1018F00083DBB5DCE1796B3F666666666612714034
:10190000061860800106683F710200200000084050
:101910000000F03F0080224610B51120FFF7A6FD21
:10192000802104460F20FFF777FC60104038C0B2DA
:1019300010BD002119200AF0DDBB012119200AF099
:10194000D9BB000008B51E4B1860032837D8DFE864
:1019500000F0021C2E3401211C200AF0CBFB0121D7
:10196000C2200AF0C7FB174B1B782BB10021BDE842
:10197000084025200AF0BEBB134B1B78FBB10121A8
:10198000BDE808400C20FFF747BC01211C200AF0ED
:10199000B1FB0021C2200AF0ADFB0A4B1B780BB152
:1019A0000121E4E7084B1B784BB10021E8E7002157
:1019B0001C200AF09FFB0121ECE70021E6E708BDAF
:1019C000D407002071020020080C00200000000055
:1019D0002DE9F84F01210646FFF7B8FAFA200AF080
:1019E000C7FB0AF0C3FBDFF8E08004464FF09045E8
:1019F00000272B699A0713D4DFF8CC804FF090476B
:101A00003D6915F002051CD00AF0B0FBDFF8B8A064
:101A1000054647F230574FF090494FF0000823E059
:101A20000AF0A4FB001B63EB0303804577EB030381
:101A3000DFD200213046FFF789FABFEE000ABDE889
:101A4000F88F0AF093FB001B63EB0303804575EBF3
:101A50000303D5D2EDE70AF089FB001B63EB030318
:101A6000824578EB0303E4D3D9F810309B07F2D416
:101A70004FF0904BDBF8103013F0020817D0013F05
:101A8000CBD10AF073FB394604463046FFF75EFAC5
:101A9000601B61EB0101FEF769FD0CA3D3E9002394
:101AA000FEF7C4FEFFF790F800EE100AC7E70AF051
:101AB0005DFB054A001B63EB0303824278EB0303E3
:101AC000D8D2B6E7AFF3008080841E00000000008B
:101AD000004CDD4008B5FFF77BFFB5EEC00AF1EE24
:101AE00010FAC8BF9FED047AF0EE407ACCBF87EEC3
:101AF000270A9FED020A08BD002474490000000077
:101B000070B50120FFF7E6FF0021084610EE104AED
:101B1000FFF71CFA0220FFF7DDFF0021084610EE58
:101B2000106AFFF713FA2046FEF7FEFC0D4B002269
:101B3000FEF752FD044630460D46FEF7F5FC0A4B13
:101B40000022FEF749FD02460B4620462946FEF7D5
:101B50008DFB064B0022FEF73FFDFFF735F800EE48
:101B6000100A70BD0070874000908F400000E03F79
:101B70002DE9F843844B1B782DED028B002B00F0F0
:101B8000FE800020FFF7DEFEFFF7BAFF7F4C804F9C
:101B900084ED000A0420FFF79DFF7E4BB5EEC00ADE
:101BA000F1EE10FA83ED000A6DD801233B7000219D
:101BB0000846FFF7CBF90320FFF78CFF764B774EF3
:101BC000774D83ED000AB5EEC00AF1EE10FA74D835
:101BD0000123337000210846FFF7B8F90520FFF70D
:101BE00079FF704B95ED008A83ED000A6E4BD3EDC3
:101BF000007A6E4B93ED007A37EEC00A77EEC77A23
:101C0000C0EE277A17EE900AFEF78EFC684B002292
:101C1000FEF7E2FCFEF790FFFEF774FC044618EEB8
:101C2000100A0D46FEF780FC624B0022FEF7FEFD17
:101C300002460B4600200021FEF716FB02460B462B
:101C400020462946FEF712FBFEF776FFFBEE047AEC
:101C5000B4EEE78AF1EE10FA574D044646D42C60F4
:101C60002B68692B40F3828065232B603B7803B996
:101C70003378524ABDEC028B002113700846BDE850
:101C8000F843FFF763B994ED007ADFED4D6AC7EED4
:101C9000007A00233B704B4B9FED4B7AC3ED007AEB
:101CA00077EEC77A494B87EEA67AD3ED007A484B98
:101CB00077EE277AC3ED007A79E794ED007ADFEDCD
:101CC000406AC7EE007A00233370424B9FED3E7AA4
:101CD000C3ED007A77EEC77A3F4B87EEA67AD3ED55
:101CE000007A77EE277AC5ED007A73E777EEC87A47
:101CF00017EE900AFEF718FC384B0022FEF796FD0F
:101D0000374B0022FEF7B2FA804620468946FEF79E
:101D1000F9FB02460B4640464946FEF75DFCFEF7DE
:101D20000BFFDFED307AB4EEE78AF1EE10FA0446ED
:101D300095D577EEC87A17EE900AFEF7F5FB2A4B99
:101D40000022FEF773FD264B0022FEF78FFA804635
:101D500020468946FEF7D6FB02460B4640464946DA
:101D6000FEF73AFCFEF7E8FE286079E7642B01DD18
:101D700064237AE7002BBFF679AF002375E7BDEC4B
:101D8000028BBDE8F88300BFDC010020E0070020E3
:101D9000DF0700200C08002000080020DE070020DC
:101DA000F8070020F4070020F0070020EC070020CF
:101DB0000000594000001A40E8070020DD0700201D
:101DC000666676400808002000007A44D8010020AA
:101DD00004080020FC070020D40100200080664099
:101DE0000000F03F000020C200806B4070B5134E31
:101DF000134D144C0AF0B8F93368C01AFEF772FBA1
:101E0000114B0022FEF712FDFEF7DEFE07EE900AF0
:101E1000F5EEC07AF1EE10FA0ADDD4ED006A95ED28
:101E2000007A0A4B37EE667AC7EE276AC3ED006A7E
:101E30000AF09AF92B683060236070BD940100208D
:101E40005C0800203408002000408F40300800204B
:101E500038B5214D214C0A217320FFF7DDF9204AC6
:101E600023686968B3FBF2F3CE2253436A68521ABF
:101E70009342FBDC00217320FFF7CEF9184A696812
:101E80002368154DB3FBF2F3CE2253436A68521A0E
:101E90009342FBDC0A217320FFF7BEF9104A696800
:101EA00023680D4DB3FBF2F3CE2253436A68521AF6
:101EB0009342FBDC00217320FFF7AEF9084A236848
:101EC0006968B3FBF2F30448CE2253434268521AC6
:101ED0009342FBDC38BD00BF001000E0D4020020BC
:101EE00040420F0038B5124C124D0A217320FFF703
:101EF00093F9114A2B686168B3FBF2F34FF4C8728F
:101F000053436268521A9342FBDC00217320FFF7AF
:101F100083F9094A2B686168B3FBF2F304484FF474
:101F2000C87253434268521A9342FBDC38BD00BF6B
:101F3000001000E0D402002040420F0008B1FFF77B
:101F4000D1BFFFF785BF0000064B1A88504040F311
:101F5000000020F4F74020F0770080EA520018805B
:101F6000704700BF8C0100202DE9F843174D184E33
:101F700004468846082704F001094846FFF7E4FFB5
:101F80002878B9F1000F18D0FFF7D8FF3378013364
:101F9000DBB23370B8F1000F09D0052B07D12878D8
:101FA00080F001002870FFF7C9FF00233370013F64
:101FB0004FEA5404DFD1BDE8F88380F001002870B7
:101FC000FFF7BCFF86F80090F1E700BFD3070020C1
:101FD00010060020074B10B51C88E0430121C0B259
:101FE000FFF7C2FF6FEA14200121BDE81040C0B224
:101FF000FFF7BABF8C01002070B53C483B4EFEF79E
:10200000D1F800250446AC4243DC062C09D0C4F1CB
:1020100006040025012140200135FFF7A5FFA54258
:10202000F8D1334E01216020FFF79EFF347A00255E
:10203000AC4238DC052C4BD92E4B2F4E1878303063
:102040004000012100F0FE00FFF78EFF2A48FEF756
:10205000A9F800250446AC423EDCC4F10604002584
:10206000012140200135FFF77FFFAC42F8D1234B1F
:102070001878400061300121C0B2FFF775FF0121DF
:102080000320FFF771FFBDE870400121F020FFF74A
:102090006BBF16F8010B4000012100F0FE00FFF7B6
:1020A00063FF0135AFE72946304609F091FD00781E
:1020B0004000012100F0FE00FFF756FF0135B7E7B1
:1020C00001214020FFF750FF0135AC42F8DCB3E7B7
:1020D0000025C4F10604F8E716F8010B40000121C1
:1020E00000F0FE00FFF740FF0135B4E735020020A5
:1020F000C40800203C0200202F0200202E020020F5
:1021000070B506460D460024AC4200DB70BD305D64
:102110000121FFF729FF0134F6E7000010B514494B
:10212000044614480AF024FB012C0CD11248FEF797
:1021300039F801461048FFF7E3FF1048FEF732F880
:1021400001460E4806E0022C08D10D48FEF72AF899
:1021500001460B48BDE81040FFF7D2BF032C05D164
:102160000848FEF71FF801460648E4E710BD00BF27
:10217000A8D7000835020020A1070020D9060020BA
:1021800011060020BA07002038B505460024A542F4
:1021900000DC38BD00217E20FFF7E6FE0134F6E7C3
:1021A00038B5002104467220FFF736F80B4B0025A6
:1021B00064201D70FFF7E8FF094B4FF6FF721A808D
:1021C000084B1D70FFF718FF2046FFF7A7FFFFF72A
:1021D00001FFBDE838400320FFF7D6BFD30700203A
:1021E0008C01002010060020F0B50028124F134C7F
:1021F000D8BF4042B0FBF4F60E8007FB06004FF05C
:102200003C0606FB00F090FBF4F4E4B2147004EB1F
:102210008402C4EBC204D8BF002542F21072C8BFCA
:10222000012590FBF2F000EB8400187015B90B88C3
:102230005B420B80F0BD00BFC0BDF0FF40420F000D
:102240002DE9F04FDFED767A764E20EE277A8BB0CF
:10225000BDEEC77A0DF1220308AA09A9824617EE3E
:10226000100AFFF7C1FF60EEA77A0DF12303FDEE20
:10227000E77A0DF1210217EE900A0DF12601FFF722
:10228000B3FFD6ED007ABDF924309DF822509DF8B9
:1022900021809DF82390F2EE046A87EEA67A002B47
:1022A000B8BF5B424FF00A0E9BB2B3FBFEF10EFBD0
:1022B0001133CAB29DF82010B1FBFEF000F13004DA
:1022C000E4B20EFB10110694FDEEE77ABCEEC77A7D
:1022D000B5FBFEF40EFB1455E0B2BDF926408DEDC2
:1022E000077A17EE906A9DF81C7096FBFEFB002C97
:1022F000B8BF64420EFB1B66142FE4B206EB8606E1
:10230000B5EEC00AC9B28CBF1C376C37DBB2F1EE38
:1023100010FAEDB24FEA4606A4F10A0ED4BF3031EE
:10232000503105F1300C203650325033BEF1590F88
:102330005FFA8CFCFFB2F6B2D2B2DBB2C9B262D99C
:10234000F5EEC00A5030F1EE10FAC0B263DC503541
:10235000632C5FFA85FC52D96D2C94BF0834483C3D
:10236000314DD5ED007A0191FDEEE77A06990091A5
:1023700017EE905A05F51C55B8F1090F42F2590EA7
:10238000CDE9020C29492A4805F1100598BF08F14A
:102390005808B5FBFEFB88BF08F11C080EFB1B5557
:1023A0000AF01CF9234B24491B780593234B1B7817
:1023B00004931C239944CDE90263E4B25FFA89F3E4
:1023C0005FFA88F8009322464346019750460AF088
:1023D00005F95B21B5FBF1F201FB125521352132E4
:1023E0000BF12103EDB2D2B2009215490195DBB297
:1023F000524650460AF0F2F80BB0BDE8F08F092CB7
:102400000BD91C34ACE7F5EEC00A3030F1EE10FA0F
:10241000C0B2F6DC9BE7632C9ED87634A0E700BF01
:1024200000247449580800205C080020B4D7000834
:10243000350200202C020020AFD700082D0200201A
:10244000C1D7000830B52DED048BDFED308A9FED4C
:10245000309A60EE287A8BB0FDEEE77A0DF1090331
:10246000044602AA17EE900A03A9FFF7BDFEB4EED8
:10247000C90ABDF90C202749F1EE10FAACBF4E2372
:102480005323002AB8BF524201939DF809300093AC
:10249000B0EE608A9DF8083092B204A80AF09EF867
:1024A00068EE288A0DF10B03FDEEE87A0DF10A02C1
:1024B00017EE900A0DF10E01FFF796FEBDF90E2002
:1024C0001549B4EEC98AF1EE10FAACBF4523572383
:1024D000002AB8BF524207AD01939DF80B3000931C
:1024E00092B29DF80A3028460AF078F80B4B0C4956
:1024F0001B78CDE900530B4B04AA1B7820460AF049
:102500006DF80BB0BDEC048B30BD00BF00247449E6
:1025100000000000CBD70008DBD700082D02002008
:10252000EBD700082C02002008B50021272009F075
:10253000E1FDBDE808400121262009F0DBBD08B51A
:10254000FFF7F2FFFEF78AFF40F6B83009F010FE01
:10255000BDE808400121092009F0CCBD08B5FFF70E
:1025600039F9194BD3ED007AB4EEE70AF1EE10FA1F
:1025700008D5F5EE407AF1EE10FA03D0FEF76EFFC3
:10258000FFF7DDFF114B1B685A1C1BD007EE903A7A
:102590000F4B104A93ED007A1068F8EEE77AF4EEEC
:1025A000C77AF1EE10FA08D5431C0BD00A4B18601D
:1025B000BDE80840C0B2FEF7F3BF013002D0074BC0
:1025C0001868F3E708BD00BF9C080020FC0100204C
:1025D0005C0800206002002038080020640200200F
:1025E00008B50121272009F085FDBDE8084000213C
:1025F000262009F07FBD08B50021272009F07AFDCB
:10260000BDE808400021262009F074BD08B501216D
:10261000272009F06FFDBDE808400121262009F0C0
:1026200069BD00002DE9F047DFF880814C4F4D4D2A
:102630004D4E4E4CDFF878A100234FF0010988F889
:1026400000303B702B70337023708AF80090FFF7D6
:10265000C1F8474BD3ED007AF4EEC07AF1EE10FAF0
:102660002DDD88F80090434B1A68434B1B689A4253
:1026700003DA424B1B686BBB2B70414B414A197804
:10268000414B1878414B38B339B301211170002107
:10269000197098F8001009B912782AB3012322782A
:1026A000337000238AF8003062BBC82338490B60BE
:1026B000384B1B7873BBBDE8F047FFF7A7BF364B1D
:1026C000D3ED007AF4EEC07AF1EE10FAC8BF87F8C5
:1026D0000090C8E70123CFE721B100211970012143
:1026E0001170D6E71970FBE73A7832B92A7822B927
:1026F0001B7813B9294B1B783BB1012323700023AE
:102700008AF8003000226423D0E7012223708AF87F
:102710000020CBE7224B2349D3ED007A224BF8EE81
:10272000E77A93ED007AF4EEC77AF1EE10FA54BF2F
:10273000012300230B7083B133781BB1BDE8F04750
:10274000FFF7F2BE23781BB1BDE8F047FFF753BF98
:102750001AB1BDE8F047FFF743BFBDE8F08700BFFF
:1027600043080020420800204608002045080020B9
:10277000A008002050080020F8010020E4010020FB
:10278000DE07002040080020DF070020410800206D
:102790004808002004020020A4080020DC070020D4
:1027A00000020020880800205C0800204408002067
:1027B0009801002010B50424FFF71DFF7D2009F0CB
:1027C000D7FCFFF723FF7D2009F0D2FC013CF3D1B9
:1027D000FFF7AAFE2146192009F08CFC40F6B8301C
:1027E00009F0C6FC0121192009F084FCFFF7F8FE6E
:1027F000322009F0BDFCFFF709FF322009F0B8FCD8
:10280000FFF7F9FE024A13680133136010BD00BFE1
:102810001408002008B50B4B1B788BB109F0A4FC01
:10282000094B98420CD9BFF34F8F0849084BCA682F
:1028300002F4E0621343CB60BFF34F8F00BFFDE7AC
:1028400008BD00BFA8010020FF07194800ED00E007
:102850000400FA0510B5FFF75FF80446FEF7E8FF3D
:10286000FDEEC07A782C17EE900A0ADC80EAE0735D
:10287000A3EBE073782BDDBF241804EBD474601055
:10288000204610BDF0B52DED028BA9B08849044655
:1028900007A809F0B7F88649204609F0B3F8854A39
:1028A000834913680AA80133136009F0ABF8824B1F
:1028B000824A1B680093824B12681B68814903A8F7
:1028C00009F08CFE03AD06460027B742C0F2DA805D
:1028D0007D4B052193ED000A0DA809F019F97B4BFA
:1028E000052193ED000A10A809F012F9784B1B7826
:1028F00023B9784B1B78002B40F0CB80FFF7AAFF61
:102900000246754905A809F069FE6949064613A8FB
:1029100009F078F805AD0027B742C0F2C2806F4BCE
:102920006F4993ED008A16A809F0ABF816A919A80B
:1029300009F0A7F86B4919A809F036F95D4B0A228E
:10294000196805461CA809F0D1F81CA9284609F009
:102950001FF9644909F028F90AA909F019F9614930
:1029600009F022F90DA909F013F95E4909F01CF9E3
:1029700010A909F00DF95B4909F016F9BCEEC88AF7
:102980000A2218EE101A05461FA809F09DF81FA983
:10299000284609F0FDF8534909F006F9524B0A227E
:1029A0001968054622A809F08FF822A9284609F0DF
:1029B000EFF84C4909F0F8F80546FEF70BFF022145
:1029C00025A809F0A5F825A9284609F0E1F8454908
:1029D00009F0EAF813A909F0DBF8014607A809F0A5
:1029E00041F825A808F0CCFF22A808F0C9FF1FA8CD
:1029F00008F0C6FF1CA808F0C3FF19A808F0C0FF24
:102A000016A808F0BDFF09990798FEF7C7FE374AD8
:102A1000034605211FA809F0ADFD354922A808F09D
:102A2000F1FF07A922A809F0B3F8324909F0BCF870
:102A30001FA9054625A808F0E5FF25A9284609F0A5
:102A4000A7F82D4909F0B0F80146204609F00AF828
:102A500025A808F095FF22A808F092FF13A808F017
:102A60008FFF10A808F08CFF0DA808F089FF0AA8B6
:102A700008F086FF07A808F083FF204629B0BDECC8
:102A8000028BF0BD15F8011B0AA809F074F8013794
:102A90001BE71A4BD3ED007AFDEEE77A17EE902A8A
:102AA0002FE715F8011B13A809F065F8013733E784
:102AB000E0E00008180800206008002068080020F6
:102AC00064080020F5D7000898080020940800202A
:102AD00041080020DC01002004D800085C08002028
:102AE000AC08002007D800085008002009D80008CA
:102AF0000ED8000813D80008DFE000080408002002
:102B00001FB5144B1B781BB3134B1B7803B3134C2B
:102B100001A8FFF7B7FE01A9204608F0BCFF01A8F5
:102B200008F02EFF2468FEF79DFC0D4B93ED000A84
:102B3000FEF7BAFC09F018FB0A4B1860FEF786FC9A
:102B40002046FEF7B3FD04B0BDE81040FEF786BC9A
:102B500004B010BD240200205D0200207C0800208B
:102B6000200200202808002030B5494A2DED028BB4
:102B700013689FED488A8BB001331360ADF80A30BB
:102B8000454B464A1B688DF80C30454B12681B6854
:102B90008DF80D30434BADF808201B688DF80E30D2
:102BA000414B1B68CDF80F30404B1B68CDF81330FC
:102BB0003F4BD3ED007AFCEEE77A044617EE903AED
:102BC000ADF817303B4BD3ED007AFCEEE77A0AAD57
:102BD00017EE903A8DF81930FEF7FCFD20EE080A4A
:102BE000FF23FDEEC07A009300234FF4FA721946DA
:102BF00017EE900A08F0BAFE2F4B8DF81C001B68E8
:102C00008DF81A30FFF726FE2C4B8DF81B00D3ED04
:102C1000007A67EE887AB2EE047AFDEEE77A1E213A
:102C200017EE903AADF81D30254BD3ED007A67EEE4
:102C3000877A02A8FDEEE77A17EE903AADF81F30DA
:102C4000204B1B688DF821301F4BD3ED007A67EEC7
:102C5000877AFCEEE77A17EE903AADF822301B4BFC
:102C60001B68ADF82430FEF78CFD02AAADF82600F3
:102C70002346144603CCAC4218605960224603F147
:102C80000803F6D120200BB0BDEC028B30BD00BF95
:102C90003C0800200000C842680800204C020020C8
:102CA0006408002060080020980800209408002094
:102CB0005C08002054080020500800203008002044
:102CC00004080020E8070020E4070020480800204E
:102CD0001F4B1B7810B59BB31E4B1B7883B31E484C
:102CE000FFF742FF1C4902461C48FEF79BF80446CA
:102CF000FEF7B8FB1A4B1868FDF716FC12A3D3E9D0
:102D00000023FDF7B3FAFDF75FFF00EE100AFEF7B0
:102D1000CBFB09F029FA134B1860FEF797FBFEF77F
:102D2000FBFC40F2EE2009F023FA0820FEF703FD39
:102D300021460A48FEF70AFDBDE81040FEF78EBBAB
:102D400010BD00BFAFF300802D431CEBE2364A3FBD
:102D5000540200205D020020EC0300206C030020E0
:102D6000500200202808002070B52DED028B2A4B60
:102D700086B0D3ED008A0546FEF72CFD274B1B7865
:102D8000B0EE408A13B9264B1B7863BBFFF762FD98
:102D90000446244B1E68244B1B7863B318EE900A3C
:102DA000FDF7C2FB1AA3D3E90023FDF715FCFDF7DD
:102DB000C3FEDFED1E7A1E4A049628EE278A02948F
:102DC000BDEEC88A03468DED038A12680192194A46
:102DD00012680092C821184A284609F0CBFB06B0B9
:102DE000BDEC028B70BD154BD3ED007AFDEEE77A9A
:102DF00017EE904ACDE7FDEEE87A114A009617EEFD
:102E0000903AC821284609F0B5FBE8E7AFF3008007
:102E1000E544BB0A293F0A405C0800204108002025
:102E2000DC010020B8080020D008002000007A440F
:102E3000500800200C06002015D8000804080020C7
:102E400034D800082DE9F0472DED028BDFED4F8AD5
:102E5000DFF864A160EE287A94B0FDEEE77A0DF118
:102E600031030CAA0DA9064617EE900AFFF7BCF92C
:102E7000B5EEC00AF1EE10FAACBF4E235323019316
:102E80009DF83130BDF9342041490093B0EE608A9D
:102E90009DF830300EA809F0A1FB68EE288A0DF1EC
:102EA0003303FDEEE87A0DF1320217EE900A0DF1D0
:102EB0003601FFF799F9B5EEC08AF1EE10FAACBF12
:102EC0004523572301930DF144089DF83330BDF994
:102ED00036203049009340469DF8323009F07EFBA1
:102EE0002D4B93ED008A18EE100AFDF71DFB2B4BBE
:102EF0000022FDF771FB2A4B0022FDF797FC294BBE
:102F00000022FDF7B3F9FDF717FEDAF80040632C55
:102F1000074638DC002C08BF0124234BD3ED007A90
:102F2000B2EE047A67EE877AFDEEE77A17EE905AF2
:102F3000FFF790FCDAF800A08146FEF74BFCDFEDCE
:102F40001B7A1B4B1B4A1B680B9320EE270ABDEE16
:102F5000C88ABDEEC00A0023CDE90233CDE9008363
:102F6000CDE9089ACDE905458DED0A0A8DED078A70
:102F700004970EABC821304609F0FCFA14B0BDEC42
:102F8000028BBDE8F0870024C7E700BF0024744926
:102F9000CBD70008DBD7000804080020000022403F
:102FA0000000144000004040E407002000007A4484
:102FB000B808002040D80008E80700200000000002
:102FC00038B5334B1B78002B5CD0324B1B78002B71
:102FD00058D00220FEF7EDFA2F4B304D1868FDF760
:102FE000A3FA29A3D3E90023FDF73EF9FDF7ECFD91
:102FF00000EE100AFEF758FA09F0B6F8284B294AF5
:1030000018602B682849032B2BD12848D2ED000AE1
:1030100091ED000AFFF714F9254A13680133136094
:10302000FEF714FA8024FEF75DFF013CFBD12878FF
:10303000FFF7B6F8FEF712FA1E4B1B7813B3FEF734
:1030400005FA41F28834FEF703FF013CFBD141F25F
:103050008834FEF747FF013CFBD1BDE83840FEF75E
:10306000FDB9022B91ED000AD2ED000A03D11248FE
:10307000FFF7E8FED0E71148FFF7E4F91048FFF743
:1030800073FEC9E738BD00BFFA7E6ABC7493583F2F
:10309000450200205D02002040020020280200209E
:1030A000280800209408002098080020BA07002073
:1030B0000C0600209008002011060020A107002027
:1030C000D90600202DE9F04F564CDFF864A12DED14
:1030D000088B884605460FCC97B00DF1080CACE87C
:1030E0000F000FCCACE80F0094E8030008348CE824
:1030F00003000FCC0DF1300CACE80F000FCCACE8A6
:103100000F0094E80300484B8CE80300002251ECC8
:10311000110B57EC106BFDF7A9F8444B41EC190B60
:10312000002230463946FDF7A1F808F1FF330A2B9B
:1031300028BF4FF006084FEA680341EC180B0193D3
:103140000DF1080B0024019B9C420CD1384900234F
:10315000284601F8143008F055FC284617B0BDEC9D
:10316000088BBDE8F08FBBEC02BB51EC190B53ECA4
:103170001B2BFDF75BFB0CAB03EBC40393ED00AB28
:10318000804653EC1A2B894651EC180BFDF74EFB89
:10319000E30706460F4636D5264B002240464946F1
:1031A000FDF764F8FDF7F0FC224B5FFA80F800228F
:1031B00030463946FDF75AF8FDF7E6FCB0EE4B1AFB
:1031C000F0EE6B1AB0EE490AF0EE690AC0B28AF866
:1031D00001008AF8008009F069FEB0EE4A1AF0EEAC
:1031E0006A1AB0EE409AF0EE609AB0EE480AF0EE3D
:1031F000680A09F05BFE01340AF1020AB0EE408A67
:10320000F0EE608A9FE740464946FDF795FC394657
:1032100000F141083046FDF78FFC5FFA88F8413035
:10322000CCE700BF58D700080080664000805640B9
:103230005C0300200000484070B52DED048B2E4942
:103240002E4E8CB0044608F0DDFB2D4B2D4993ED3E
:10325000008A03A808F0D6FB2B49684608F011FC49
:10326000694603A808F094FC314608F09DFC274B02
:1032700005461868FDF758F9254B41EC190B1868FD
:10328000FDF752F9B0EE491AF0EE691A41EC100B55
:1032900006A80A21FFF716FF06A9284608F078FCC1
:1032A000314608F081FC1B4908F07EFCBCEEC88A60
:1032B0000A2218EE101A054609A808F005FC09A90B
:1032C000284608F065FC144908F06EFC01462046CB
:1032D00008F0C8FB09A808F053FB06A808F050FB4B
:1032E000684608F04DFB03A808F04AFB20460CB0E6
:1032F000BDEC048B70BD00BFE0E0000891D8000871
:103300005C08002090D80008AC0800209408002039
:103310009808002093D8000898D800080000000002
:1033200010B5002186B0084602F0F4FD544B554C10
:103330001868FDF7F9F850A3D3E90023FDF74CF91D
:10334000FDF722FC01460620FDF7C8FE4E4B18682B
:10335000FDF7EAF848A3D3E90023FDF73DF9FDF7AF
:1033600013FC01460220FDF7B9FE484B1868FDF733
:10337000DBF841A3D3E90023FDF72EF9FDF704FCA8
:1033800001460A20FDF7AAFE414B1868FDF7CCF86C
:1033900039A3D3E90023FDF71FF9FDF7F5FB01463B
:1033A0001B20FDF79BFE3B4B0E20197802F0B2FD6F
:1033B000394BD3ED007AB2EE047A67EE877A0F20AC
:1033C000FCEEE77ACDED017A9DF8041002F0A2FD43
:1033D000324B10201968FDF7AAFE314B12201978E4
:1033E00002F098FD2F4B13201968FDF7A0FE2E4B1D
:1033F00015201968FDF79BFE2C4B1720197802F059
:1034000089FD2B4B1820197802F084FD294B1920D7
:10341000197802F07FFD284B1F20197802F07AFD01
:103420000721302002F076FD3C212020FDF77FFEB1
:103430004FF416512C20FDF751FE214603A808F049
:10344000E1FA03A93220FDF717FE03A808F098FA65
:10345000214603A808F0D6FA03A93C20FDF70CFE8C
:1034600003A808F08DFA0021502006B0BDE81040F6
:1034700002F050BDAFF300800000000080842E41B8
:10348000500200209BD800084002002020020020AB
:103490000C02002018020020140200201C02002050
:1034A000100200204C020020480200203C020020B4
:1034B0002D0200202C0200200802002010B52DED66
:1034C000028B062084B0FDF7F4FD013001D1FFF737
:1034D00027FF0620FDF7EDFD07EE900A9FED678AB6
:1034E000674B684CF8EE677A0A2087EE887A83ED9E
:1034F000007AFDF7DEFD07EE900AF8EE677A624B80
:1035000087EE887A022083ED007AFDF7D2FD07EE80
:10351000900AF8EE677A5D4B87EE887A1B2083ED80
:10352000007AFDF7C6FD07EE900AF8EE677A584B71
:1035300087EE887A132083ED007AFDF7EDFD554B79
:1035400018601520FDF7E8FD534B18600E2002F0BF
:103550009DFC524B18600F2002F098FCFCF7D2FF44
:1035600000224F4BFDF762F9FDF72EFB4D4B186023
:103570001020FDF7D1FD4C4B1860122002F086FCA4
:103580004A4B1860172002F081FC494B1870182034
:1035900002F07CFC474B1870192002F077FC464B78
:1035A00018701A2002F072FC20601F2002F06EFCDE
:1035B000424B18602020FDF7AFFD4FF47A7358435B
:1035C000A0F5DA503E4B18381860302002F05EFC4F
:1035D0003C4B1860002002F059FC3B4B18703B4BF1
:1035E00000F001021A703A4BC0F340021A70394BD6
:1035F000C0F380021A70384BC0F3C00210F0100FF5
:103600001A700CBF012302232360344BC0F3401215
:103610001A70334BC0F380121A70324BC009187005
:1036200008B10323236001A83221FDF701FD01A9A0
:103630002D4808F030FA01A808F0A2F901A83C21B1
:10364000FDF7F6FC01A9294808F025FA01A808F0C1
:1036500097F901A85021FDF7EBFC01A9244808F0D7
:103660001AFA01A808F08CF92C20FDF722FD214B55
:10367000186004B0BDEC028B10BD00BF002474497B
:1036800050020020280200202002002040020020DA
:103690000C0200204C0200204802002018020020EA
:1036A00000002440140200201C0200201002002010
:1036B0003C0200202D0200202C02002008020020E5
:1036C00058020020680200206C04002054020020F0
:1036D0002402002045020020A9080020A80800209C
:1036E000D008002044020020C4080020AC080020BC
:1036F000B80800208801002037B532241D481E4D2F
:1037000002F00EFC00941D231E221F211B4802F014
:1037100089F90094234616221721194807F0F4FD71
:1037200023461A2200941B21164C174807F0ECFD83
:103730002946164808F066F92146154808F062F94E
:103740002946144808F05EF9134B14481A78144BB4
:1037500021461A7008F056F92146124808F052F92D
:10376000114B1A68114B1A60114B1A68114B1A60F1
:1037700003B030BD0C0C00209BD80008880B002043
:10378000300A0020E0E00008D8080020C40800202B
:10379000B8080020AC080020040200207C080020AB
:1037A00088080020700800206402002038080020EB
:1037B000D40800200806002008B5084808F0E0F802
:1037C000074808F0DDF8074808F0DAF8064808F07E
:1037D000D7F8BDE80840054808F0D2B870080020C6
:1037E0007C080020AC080020B8080020C408002095
:1037F0002DE9F041C04E86B00024FD2C24D0304687
:1038000007F078FC0028FADDBB48BC4D07F00CFF40
:10381000C1B20A29295500F08880B74807F03FFF58
:103820002B5D082B08BF023C2B5D0D2B7DD10023A7
:1038300064202B5508F09CFCAF4807F05BFC002887
:1038400002DDAD4807F0F0FEAC49AD4800220C4661
:10385000064611F8013B202B06D03D2B04D01BB1AE
:103860000D2B01D0182A62D10021B154002B6DD14B
:10387000A449A34808F0F4FE002840F08980A2493A
:10388000A24C03A808F0BEF803A8FDF76BFC51ECAE
:10389000100BFDF799F9206003A808F071F894ED7A
:1038A000007ADFED9B7AB4EEE77ADFED9A7AF1EEFB
:1038B00010FAC4BFC7EE276AC4ED006A94ED007A1F
:1038C000B4EEE77AF1EE10FAC8BFC7EE276A9FEDB3
:1038D000927AC8BFC4ED006AD4ED007AF4EEC77ADC
:1038E000F1EE10FA4BDD9FED8D7AF4EEC77AF1EE32
:1038F00010FA44D58A49804807F0F0FE89497E488D
:1039000007F0C9FE2068FCF70FFE79A3D3E9002376
:10391000FCF762FEFDF738F901460620FDF7DEFBF5
:1039200006B0BDE8F041FFF7C9BD013465E7A3F17A
:103930006105192D9CBF03F05F0301F8013C11F8EC
:10394000013C00F8013B013283E70132A15C2029F0
:1039500004EB0203F9D03D29F7D06B481A46044620
:10396000002312F8011B19B10D2901D0132B02D12C
:103970000022E2547CE700F8011B0133F1E76A49B9
:103980005D4807F0ABFE67495B4807F084FEC7E778
:1039900066495B4808F064FE00284FD15A49644CE0
:1039A00003A808F02FF803A8FDF7DCFB51EC100B7F
:1039B000FDF70AF9206003A807F0E2FF94ED007A12
:1039C000DFED537AB4EEE77ADFED527AF1EE10FADA
:1039D000C4BFC7EE276AC4ED006A94ED007AB4EE66
:1039E000E77AF1EE10FAC8BFC7EE276A9FED4A7A70
:1039F000C8BFC4ED006AD4ED007AF4EEC77AF1EEE8
:103A000010FABCDD9FED457AF4EEC77AF1EE10FABC
:103A1000B5D54349384807F061FE4249364807F0BA
:103A20003AFE2068FCF780FD31A3D3E90023FCF7C0
:103A3000D3FDFDF7A9F8014602206FE73D49304864
:103A400008F00EFE002879D12F493B4C03A807F05F
:103A5000D9FF03A8FDF786FB51EC100BFDF7B4F876
:103A6000206003A807F08CFF94ED007ADFED287A40
:103A7000B4EEE77ADFED277AF1EE10FAC4BFC7EEB5
:103A8000276AC4ED006A94ED007AB4EEE77AF1EEAD
:103A900010FAC8BFC7EE276A9FED1F7AC8BFC4EDF2
:103AA000006AD4ED007AF4EEC77AF1EE10FA7FF7EF
:103AB00066AF9FED1A7AF4EEC77AF1EE10FA7FF551
:103AC0005EAF17490C4807F009FE16490A4807F08F
:103AD000E2FD2068FCF728FD05A3D3E90023FCF7ED
:103AE0007BFDFDF751F801460A2017E7AFF3008090
:103AF0000000000080842E41D80800200605002028
:103B00006D040020BCD8000886040020500200206C
:103B10000024744900007A440000D7430000DC43CD
:103B2000C5D80008C9D80008CBD80008E3D80008D9
:103B300040020020EBD80008200200209C499D484C
:103B400008F08EFD002851D19B499C4C03A807F03A
:103B500059FF03A8FDF706FB51EC100BFDF734F8F5
:103B6000206003A807F00CFF94ED007ADFED947A53
:103B7000B4EEE77ADFED937AF1EE10FAC4BFC7EE48
:103B8000276AC4ED006A94ED007AB4EEE77AF1EEAC
:103B900010FAC8BFC7EE276A9FED8B7AC8BFC4ED85
:103BA000006AD4ED007AF4EEC77AF1EE10FA7FF7EE
:103BB000E6AE9FED867AF4EEC77AF1EE10FA7FF565
:103BC000DEAE8349834807F089FD8349814807F0C9
:103BD00062FD2068FCF7A8FC73A3D3E90023FCF77F
:103BE000FBFCFCF7D1FF01461B2097E67B4971489F
:103BF00008F036FD60BB704808F040FBB0F5966FEA
:103C000017D0B0F5166F14D0B0F5965F11D0B0F59F
:103C1000165F0ED0B0F5964F0BD0B0F5164F08D00A
:103C2000B0F5614F05D0B0F5963F02D0B0F5E13F59
:103C30000CD16B4C6B492060664807F04FFD66491C
:103C4000644807F028FD21682C2067E6664997E65E
:103C50006649584808F004FD88B95748644C08F094
:103C600009FB5B4920605B4807F038FD5A49594819
:103C700007F011FD21781F2002F04CF950E65D4954
:103C80004C4808F0EDFC98B94B485B4C08F0F2FA50
:103C9000072820600AD84E494E4807F01FFD4E49BC
:103CA0004C4807F0F8FC21783020E5E7534967E6F7
:103CB0005349404808F0D4FCC0B93F48514C08F083
:103CC000D9FA4FF6E6532060013898420CD84049A3
:103CD000404807F003FD40493E4807F0DCFC2188DE
:103CE0001320FDF724FA1BE6474949E647493148C6
:103CF00008F0B6FCB0B93048454C08F0BBFA40F2C9
:103D00002E232060293898420AD83149314807F0DB
:103D1000E5FC31492F4807F0BEFC21881520E0E77B
:103D20003C492DE63C49234808F09AFCF8B9224862
:103D30003A4C08F09FFA3A4B93FBF0F31E4823608D
:103D400008F098FA282810DD1B4808F093FAB0F51F
:103D5000167F0ADA1E491F4807F0C0FC1E491D489D
:103D600007F099FC21881020BBE72E4908E62E4970
:103D7000104808F075FC00285CD10F482B4C08F067
:103D800079FA2060013803280AD81149114807F050
:103D9000A5FC11490F4807F07EFC217812206BE743
:103DA0002349EDE5AFF300800000000080842E4140
:103DB000F3D800086D040020860400200C020020C7
:103DC0000024744900007A440000D7430000DC431B
:103DD000C5D80008D8080020C9D80008FCD80008B9
:103DE0008801002004D9000822D9000841D9000820
:103DF000080200204CD900086802002055D90008AC
:103E000063D900084C0200206BD900088AD9000849
:103E10004802002093D90008B0D900081C020020F5
:103E200040420F00B8D90008D4D900081002002081
:103E3000DED90008A449A54808F012FCA0B9A4489E
:103E4000A44C08F017FA2060073801280AD8A249C4
:103E5000A24807F043FCA249A04807F01CFC2178C7
:103E60000E2009E79F498BE59F49984808F0F8FB29
:103E700000283ED196499D4C03A807F0C3FD03A836
:103E8000FDF770F951EC100BFCF79EFE206003A8C3
:103E900007F076FDD4ED007AB7EE007AF4EE477ABB
:103EA000F1EE10FA0DD0B0EE007AF4EE477AF1EEB2
:103EB00010FA06D0B7EE087AF4EE477AF1EE10FA6F
:103EC00015D18549854807F009FC8549834807F0E5
:103ED000E2FBD4ED007AB2EE047A67EE877A0F2027
:103EE000FCEEE77ACDED017A9DF80410C4E6804936
:103EF00046E58049754808F0B3FBA0B974487E4C8C
:103F000008F0B8F9C0B20F2820700AD87249734877
:103F100007F0E4FB7249714807F0BDFB21781720D8
:103F2000AAE676492CE57649684808F099FB70B90D
:103F3000674B744C1B7868496848237007F0CEFBC8
:103F40006749664807F0A7FB2178182094E66E4978
:103F50005E4808F085FB70B95D4B6C4C1B785E4980
:103F60005E48237007F0BAFB5D495C4807F093FB9D
:103F70002178192080E66649544808F071FBB8B9E9
:103F8000534808F07BF984B20F2C5349534838BF8B
:103F90000F2407F0A3FB5249504807F07CFB4FF475
:103FA0007A72E31F53435B4A21461360202098E650
:103FB0005949464808F054FB044670BB444D2B78E1
:103FC0004BB3DFF8588115F8016B04F132075EB985
:103FD000314603A80397FDF726F85048214607F01D
:103FE000F7FD06703C49CBE4A6F16103192B9CBF99
:103FF00006F05F0605F8016C2146404615F8016C95
:1040000007F0E6FD067015F8011C039703A8FDF7FD
:104010000AF80134D7E74249B2E442492B4808F094
:104020001FFB044660BB2A4B1B78002BF3D0284EA5
:104030003D4F16F8015B04F13C0355B9294603A82E
:104040000393FCF7F0FF3848214607F0C1FD0570E7
:10405000C8E7A5F16102192A9CBF05F05F0506F8C3
:10406000015C16F8011C039303A8FCF7DCFF214652
:10407000384616F8015C07F0ABFD01340570D8E74F
:104080002A49124808F0ECFA002855D1104C237840
:10409000BBB12146264807F006FD0F490F4807F03F
:1040A0001DFB0F490D4807F0F6FA214603A807F05B
:1040B000A9FC03A95020FCF7DFFF03A807F060FC70
:1040C0002EE41C495CE400BFFDD900086D0400200B
:1040D0008604002018020020C5D80008D808002057
:1040E000C9D8000806DA000818DA0008140200200F
:1040F00021DA00083CDA00083C02002045DA00081A
:1041000057DA00082D02002062DA00082C02002095
:104110006CDA00085802002074DA0008C408002095
:104120007DDA000892DA0008AC0800209BDA00086B
:10413000B8080020A3DA00088049814808F090FA06
:104140000546E0B97F4808F095F80128044614D8E0
:104150007D497E4807F0C2FA7D497C4807F09BFA0A
:104160007C4B04F001021A707B4A137803F07E0343
:10417000E118C9B2117028467EE5784900E4784913
:104180006F4808F06DFA0546D0B96E4808F072F82D
:1041900001280446F1D86C496C4807F09FFA6C4935
:1041A0006A4807F078FA6F4B04F001021A706A4B04
:1041B000197801F07D0101EB4401C9B21970DAE709
:1041C00069495F4808F04CFA0546C0B95D4808F0F7
:1041D00051F801280446D0D85B495C4807F07EFAC4
:1041E0005B495A4807F057FA604B04F001021A7015
:1041F000594B197801F07B0101EB8401DDE75C4943
:104200004F4808F02DFA0546C0B94E4808F032F87C
:1042100001280446B1D84C494C4807F05FFA4C4994
:104220004A4807F038FA534B04F001021A704A4B1F
:10423000197801F0770101EBC401BEE74E4940480F
:1042400008F00EFA0546B8B93E4808F013F8012800
:10425000044692D83C493D4807F040FA3C493B4867
:1042600007F019FA454B621C1A603B4B197801F0B4
:104270006F0101EB0411A0E74149314808F0F0F962
:104280000546C8B92F4807F0F5FF012804463FF658
:1042900074AF2D492D4807F021FA2D492B4807F01E
:1042A000FAF9384B04F001021A702B4B197801F01F
:1042B0005F0101EB441180E73349214808F0D0F950
:1042C0000546C8B91F4807F0D5FF012804463FF648
:1042D00054AF1D491D4807F001FA1D491B4807F05E
:1042E000DAF92A4B04F001021A701B4B197801F01D
:1042F0003F0101EB841160E72549114808F0B0F94E
:104300000546002848D10F4807F0B4FF01280446AD
:104310003FF633AF0C490D4807F0E0F90C490B4864
:1043200007F0B9F91B4B04F001021A700A4B197817
:1043300001F07F0101EBC4113FE700BFB7DA0008CD
:104340006D04002086040020C5D80008D80800208D
:10435000C9D80008540200206C040020C3DA000809
:10436000CADA000824020020D5DA0008450200203D
:10437000E0DA0008A9080020ECDA00082802002092
:10438000F5DA0008A8080020FFDA0008D0080020AD
:1043900007DB0008440200204449454808F060F962
:1043A00028B133783F2B02D0482B40F0C3804149DD
:1043B000414807F093F941493F4807F08FF94049D8
:1043C0003D4807F08BF93F493B4807F087F93E49E4
:1043D000394807F083F93D49374807F07FF93C49F0
:1043E000354807F07BF93B49334807F077F93A49FC
:1043F000314807F073F939492F4807F06FF9384908
:104400002D4807F06BF937492B4807F067F9364913
:10441000294807F063F93549274807F05FF934491F
:10442000254807F05BF93349234807F057F932492B
:10443000214807F053F931491F4807F04FF9304937
:104440001D4807F04BF92F491B4807F047F92E4943
:10445000194807F043F92D49174807F03FF92C494F
:10446000154807F03BF92B49134807F037F92A495B
:10447000114807F033F929490F4807F02FF9284967
:104480000D4807F02BF927490B4807F027F9264973
:10449000094807F023F92549074807F01FF924497F
:1044A000054807F01BF9FFF73BBA00BF10DB000817
:1044B0006D04002015DB0008D808002028DB000868
:1044C00069DB00087FDB0008A5DB0008B6DB00081D
:1044D000C7DB0008D9DB0008FDDB000820DC000892
:1044E00042DC000864DC000887DC0008B3DC00085C
:1044F000CEDC0008EADC000801DD00081DDD000854
:1045000037DD00084BDD000864DD000884DD0008AD
:1045100099DD0008BFDD0008E5DD000801DE0008C8
:1045200019DE000832DE000845DE000865DE0008FE
:1045300076DE0008A749A84808F092F8002840F065
:10454000D981A649A648A74DA74C07F0C7F8A749A7
:10455000A34807F0A0F8A64BA148197800290CBF82
:104560002946214607F0BAF8A2499D4807F093F87A
:10457000A1499B4807F0A8F8A049994807F08BF893
:104580009F4B974893ED000A032107F0A1F99D493D
:10459000934807F0A3F89C49914807F07CF89B49A1
:1045A0008F4807F091F89A498D4807F074F8994BB5
:1045B0008B4819780A2207F0DDF89749884807F0F8
:1045C0006AF8964B8648197807F08AF89449844827
:1045D00007F061F8934B8248197807F081F8924907
:1045E0007F4807F058F8914B914A1968914B7C48E5
:1045F000022914BF1146194607F070F88E49784811
:1046000007F049F88D4B7648197800290CBF2946E8
:10461000214607F063F88A49714807F03CF8894B56
:104620006F48197800290CBF2946214607F056F833
:1046300085496B4807F02FF8844B694819780029A1
:104640000CBF2946214607F049F88149644807F024
:1046500022F88049624807F037F87F49604807F040
:104660001AF87E4B5E4893ED000A032107F030F9FB
:1046700064495B4807F032F87949594807F00BF86C
:10468000784B574819680A2207F074F8764954485D
:1046900007F001F8754B524893ED000A012107F02D
:1046A0001CF973494E4806F0F6FF724B72491B68BD
:1046B0004B4891FBF3F10A2207F05CF86F49484838
:1046C00006F0E9FF6E4B464819680A2207F052F8D7
:1046D0006C49434806F0DFFF6B4B414819780029CD
:1046E0000CBF2946214606F0F9FF68493C4806F010
:1046F000D2FF674B3A4819680A2207F052F8654919
:10470000374806F0C8FF644B354893ED000A032193
:1047100007F0DEF83B49324806F0E0FF5F493048D9
:1047200006F0B9FF5E4B2E4819680A2207F022F8FE
:104730005C492B4806F0AFFF5B4B294819780029EC
:104740000CBF2946214606F0C9FF5849244806F007
:10475000A2FF574B224893ED000A032107F0B8F857
:1047600028491F4806F0BAFF52491D4806F093FF3A
:10477000514B1B4819680A2206F0FCFF4F491848A4
:1047800006F089FF4E4B4F4A19784F4B14480029C9
:104790000CBF1146194606F0A1FF4C49104806F01F
:1047A0007AFF4B4B0E4819680A2206F0E3FF49498D
:1047B0000B4806F070FF484B09481B6803F5DA53B5
:1047C00018330A224FF47A7193FBF1F106F0D2FF0D
:1047D00084E000BFB5DE00086D040020BADE0008EA
:1047E000D808002070DA0008A2D80008C9DE000846
:1047F00045020020D0DE0008C4080020DCDE0008EE
:1048000040020020EDDE0008F2DE0008B8080020BB
:1048100001DF00083C0200200DDF00082D0200200F
:104820001BDF00082C0200202FDF000828020020D8
:10483000A8D80008A5D800083BDF0008D008002051
:1048400046DF00084402002053DF00082402002055
:104850005ADF0008AC08002066DF000820020020B4
:1048600077DF00081802002083DF00081402002010
:1048700094DF00081C02002040420F00A4DF000863
:1048800010020020B1DF000854020020B9DF000848
:104890004C020020C4DF000850020020D6DF0008D0
:1048A00048020020E7DF0008A9080020EFDF000829
:1048B0000C02002001E00008080200200FE00008C0
:1048C000A8080020B4D80008AFD800081CE00008F1
:1048D000680200202AE00008580200200749084822
:1048E00006F0D9FE074B064819680A2206F063FF56
:1048F000FFF716B80449FFF747B800BF35E00008D6
:10490000D80800208801002045E0000810B50F48B5
:1049100006F0F0FB002801DDFEF76AFFC62007F075
:1049200007FB0446C52007F003FB323484420CD950
:10493000C52007F0FDFA502807D9054B1B68002B4E
:1049400003DDBDE81040FDF7FABD10BDD80800201A
:10495000A401002038B5684806F0CCFB002801DD32
:10496000FEF746FFC62007F0E3FA0446C52007F02D
:10497000DFFA3234844250D9C52007F0D9FA5028E2
:104980004BD95E4B1B68002B47D0012B03D1BDE8F0
:104990003840FDF7D4BD022B3FD1594C2368032B7F
:1049A00007DD2368013B032B35D8DFE803F01E3712
:1049B0005DA2C62007F0BCFA0546C52007F0B8FA8C
:1049C00032358542EDD9FDF70BFE4FF4C87007F084
:1049D000CFFBFDF7A9FD4FF4C87007F0C9FBFDF749
:1049E00015FE236801332360D8E7464B1B7893B14B
:1049F000454B1B68032B0EDC444B1B685BB1444BDF
:104A00001A7842B901221A70FDF78EFDC82007F00E
:104A1000AFFBFDF7FBFD0023236038BD3D4A157851
:104A2000002385B113701D4623689D42F3DAFDF71C
:104A30007BFD322007F09CFBFDF7E8FD322007F0FC
:104A400097FB0135F0E70123137023689D42E2DAFA
:104A5000FDF7C6FD322007F08BFBFDF7D7FD3220B6
:104A600007F086FB0135F0E72B4B1B68013330D193
:104A70002A4B18682A4B1A6882422A4A14D01860B6
:104A80001060C0B2FCF78CFD002523689D42C2DA9D
:104A9000FDF7A6FD322007F06BFBFDF7B7FD3220D6
:104AA00007F066FB0135F0E7002528461D6015601C
:104AB000FCF776FD23689D42ADDAFDF735FD322027
:104AC00007F056FBFDF7A2FD322007F051FB013540
:104AD000F0E70021272007F00DFB4FF4C87007F026
:104AE00047FB0121272007F005FB642007F040FB6E
:104AF00091E7FDF724FD8EE7D8080020A4010020EF
:104B00008C080020E901002050080020E40100206A
:104B1000120800205D0200206002002068020020D0
:104B200064020020380800202DE9F0411C4E1D4F82
:104B30000C46451E15F8013F0BB9BDE8F0812E2B40
:104B4000DFF864801AD1FCF781FC716814483B6877
:104B5000B3FBF8F363434268521A9342FBDCFCF761
:104B60007DFC71683B68104AB3FBF2F363437268E3
:104B7000521A9342FBDCFFF7EDFEDBE72D2BF0D161
:104B8000FCF764FC04EB4402716805483B68B3FB26
:104B9000F8F353434268521A9342FBDCDFE700BF4D
:104BA000001000E0D402002040420F00F8B5214D73
:104BB000214E224F97FBF1F7441E14F8013F03B931
:104BC000F8BDA3F14102D1B2192912D81C4B53F8F8
:104BD00022003946FFF7A8FF2B681A4A7168B3FB19
:104BE000F2F37B4303EB43037268521A9342FBDCFC
:104BF000E3E7A3F13002092A05D8114A163B3946EA
:104C000052F82300E6E7212B04D10D4B3946D3F8A7
:104C10009400DFE7202BDFD107492B68094A486859
:104C2000B3FBF2F37B43C3EBC3034A68121A93420C
:104C3000FBDCD1E7D4020020001000E080841E00DD
:104C40009C00002040420F001FB51F4B1B78002B1B
:104C500034D01E4B1B78002B30D01D4B1B7801A885
:104C60004BB3FDF70FFE01A91A4806F014FF01A887
:104C700006F086FE174B1C68FCF7F4FB164B186811
:104C8000FBF752FC0EA3D3E90023FBF7EFFAFBF787
:104C90009BFF00EE100AFCF707FC07F065FA0F4BCC
:104CA00018600F4B20461968FFF780FF04B0BDE87D
:104CB0001040FCF7D3BBFEF7BFFAD4E704B010BD39
:104CC0002D431CEBE2364A3FA90800205D0200207C
:104CD000A8080020700800200C02002028080020EE
:104CE00008020020264B10B518600446254806F03F
:104CF00001FA002801DDFEF77BFD8CB90021C720F9
:104D000007F02CF90021182007F028F90021C7200E
:104D100007F0F0F90021BDE81040182007F0EAB9CB
:104D2000631EFE2B0DD80021C72007F017F90021C4
:104D3000C72007F0DFF921461820BDE8104007F032
:104D40000DB9A4F58073F32B0AD8A4F1FF01C72095
:104D500007F004F9FF21182007F000F90121DAE734
:104D6000B4F5FA7FCAD1FF21C72007F0F7F8FF2179
:104D7000182007F0F3F80121C72007F0BBF9EDE791
:104D8000D8070020D80800202DE97043704B1B780D
:104D90002DED028B0C46154643B138B1FCF748FDAA
:104DA000FDEEC07A17EE903A142B44DD0020FCF79C
:104DB000C9FD684B1B78002B00F0BA80002D00F075
:104DC000B580002C00F0B480634B1B78002B40F0C2
:104DD000AF80624BD3ED007AF5EEC07AF1EE10FAB7
:104DE00040F1A6805E4B1B68552B40F3A1805D4BC4
:104DF0005D4D93ED008A5D4B2C68B8EEC88A38EEA5
:104E0000278AD3ED007A38EE678AF1EE087AB4EE9D
:104E1000E78AF1EE10FA1EDD0734554B1B689C4201
:104E2000A8BF1C4626462E603046BDEC028BBDE86E
:104E30007043FFF757BFA3F11302012A01D80120E5
:104E4000B5E7A3F11002022A01D80220AFE70A2B2E
:104E5000ACDC0320ABE7F1EE007AB4EEE78AF1EECA
:104E600010FA01DD0534D8E718EE100AFBF75CFBF9
:104E700031A3D3E9002380468946FBF73DFE08B104
:104E80000334CAE72EA3D3E9002340464946FBF783
:104E900033FE08B10234C0E7F7EE087AB4EEE78AD1
:104EA000F1EE10FA01DD0134B7E7FAEE007A314B8A
:104EB000B4EEE78AF1EE10FA1E6804D5083CA6426B
:104EC000B8BF2646AFE7F9EE007AB4EEE78AF1EE16
:104ED00010FA01D5043CF2E71BA3D3E900234046B6
:104EE0004946FBF7EBFD08B1023CE8E7FFEE087A24
:104EF000B4EEE78AF1EE10FA01D5013CDFE7A642F5
:104F000091DC1B4B1E68A642A8BF26468BE7134BBD
:104F1000D3ED007AF5EEC07AF1EE10FA08D5104B19
:104F20001B68552B04DD104B18687EE7002CEED172
:104F300000207AE7AFF30080666666666666064024
:104F40009A999999999901409A999999999901C031
:104F50009208002091080020DD07002004080020AE
:104F6000E8070020B8010020B0010020F807002069
:104F7000B4010020AC0100202DE9F843A14E2DED35
:104F8000028BFDF738FBFFF7C1FCFCF7F1FD33782E
:104F9000CBB10524FDF7C8FAFA2007F0E9F8FDF7D0
:104FA00035FB4FF4967007F0E3F8FFF7AFFC013CD8
:104FB000F0D1BDEC028B944B01221A702046BDE863
:104FC000F843FFF78FBEFFF7A1FC904B1B781BB394
:104FD000FDF71CFB8E4C322007F0CAF8FDF70BFBE7
:104FE00000232360FCF7C4FD8A4BD3ED007A8A4B83
:104FF00093ED007A77EEC77AFDEEE77AF8EEE77A7E
:10500000C4ED007AFDF702FB322007F0B1F8FDF79E
:10501000F2FA322007F0ACF8FDF7F8FA07F0A4F83E
:10502000002408EE104A7D4FDFF8EC81DFF808928B
:105030000546FFF76BFCFCF79BFD3378BBB1002006
:10504000FFF750FE0524FDF76FFAFA2007F090F8FD
:10505000FDF7DCFA4FF4967007F08AF8013CF2D1C4
:10506000694B01221A70BDEC028BBDE8F883D7EDC5
:10507000007A98ED007AD9F80030F8EEE76AF4EE9D
:10508000C76AF1EE10FA43D503F1140207EE902A35
:10509000F8EEE77AB4EEE77AF1EE10FA38D5FDF7DC
:1050A000AAFA3C2007F064F8FDF7B0FA5C4BB8EEC2
:1050B000488AD3ED007A38EE278A40F27710BCEEAA
:1050C000C88A0134FFF70EFE07F04EF8554B1B68F7
:1050D000401B98426CD94C4B534D012200201A7052
:1050E000FFF700FE0524FDF71FFAFA2007F040F84D
:1050F000FDF78CFA4FF4967007F03AF8284605F061
:10510000F9FF002801DDFEF773FB013CEBD1AAE7B4
:1051100003F11E0207EE902AF8EEE77AB4EEE77A82
:10512000F1EE10FA18DDFF20FFF7DCFDFDF763FA62
:10513000C82007F01DF8FDF769FAC82007F018F835
:10514000FDF759FAC82007F013F8FDF75FFA4FF49E
:10515000C87007F00DF8B7E703F10F0207EE902AC9
:10516000F8EEE77AB4EEE77AF1EE10FA02DD4FF4EA
:105170009B70D9E7053307EE903AF8EEE77AB4EE84
:10518000E77AF1EE10FA02DD4FF4B470CCE7F4EEFA
:10519000C76AF1EE10FA97DD4FF4FA70FFF7A2FD3F
:1051A000FDF729FAC82006F0E3FFFDF72FFA8BE799
:1051B000082C7FF43EAF0020FFF794FD0324FDF799
:1051C0000FFAC82006F0D4FFFDF720FAC82006F039
:1051D000CFFF013CF3D10C4B1C7018EE103ADB08EA
:1051E00008EE103A114BB8EEC88A83ED008A104BD6
:1051F000D3ED007A0F4BF8EE677A38EE678A83EDCD
:10520000008A30E7DE070020DC070020D001002004
:10521000D401002004080020F8070020C00100206D
:10522000F4070020C4010020D8080020F007002067
:10523000CC010020EC070020BC0100200246014800
:1052400005F0D6BF300A002008B5174B1B7873B1A4
:10525000164B1B78C3B116491120FFF7EFFF4FF42F
:105260007A7006F085FF12491120FFF7E7FF002151
:10527000262006F03FFF322006F07AFFBDE8084006
:105280000121262006F036BF0A4B1B78002BEED0FA
:1052900009492C20FFF7D2FF4FF47A7006F068FF1F
:1052A00005492C20E1E700BFF40100207102002035
:1052B00074010020080C00204801002010B50121D5
:1052C000272006F0B9FE0121262006F0B5FE0121B7
:1052D000092006F0B1FE01212C2006F0ADFE7D4B29
:1052E0001B781BB10121252006F0A6FE01211C2000
:1052F00006F0A2FE0121C22006F09EFE012113202D
:1053000006F09AFE0121C32006F096FE01212D2011
:1053100006F092FE01212E2006F08EFE01212920AA
:1053200006F08AFE01212A2006F086FE01212B20AC
:1053300006F082FE0021C12006F07EFE0121C7207A
:1053400006F07AFE0121182006F076FE01211920D0
:1053500006F072FE00211C2006F0CCFE0021C220C7
:1053600006F0C8FE0021132006F0C4FE0021C32071
:1053700006F0C0FE00212D2006F0BCFE00212E20EC
:1053800006F0B8FE0021262006F0B4FE00212720FA
:1053900006F0B0FE322006F0EBFE0121262006F0DA
:1053A000A9FE0121272006F0A5FE4B4B4B4C1968A6
:1053B0004B48062206F0FAF8FEF780F82378002B17
:1053C00078D0484B48481968062206F0EFF847495C
:1053D000434806F083F9237813B10C2006F074FDDE
:1053E000082006F08FFD4FF47A7006F09BFD404CCC
:1053F000404800F0ABFB01212C2006F07BFE237817
:10540000002B5CD03C4B1B68002B58D0FCF791FA6A
:1054100000212C2006F06EFEFBF71AFF374B1878A0
:10542000FCF7BEF805217220FBF7F6FE344B1A6834
:10543000344BB3FBF2F3344A00201360FCF782FADA
:105440000020FFF74FFC00210846FBF77FFD0021FD
:10545000262006F04FFE322006F08AFE012126208B
:1054600006F048FEC82006F083FE0021262006F044
:1054700041FE322006F07CFE0121262006F03AFE95
:10548000224B1B783BB1224B1B7823B1214B1B785D
:105490000BB1FFF771FD2378D3B1174B1B68BBB17C
:1054A000FCF74BFA4FF47A7006F062FEBDE810404C
:1054B000FFF7CABE184B1B78002B88D081E7FCF79A
:1054C0003CFA4FF47A7006F053FEFFF7BDFE9FE7FB
:1054D00010BD00BF70020020880100207102002072
:1054E000D80800206C020020300A002049E00008A3
:1054F000E9010020880B0020E4010020380800208A
:105500004802002040420F0068030020DC01002018
:10551000C9010020C8010020080C0020144B1B7892
:1055200070B5044653B1012809D1124D2B68012BE7
:1055300004D011490A20FFF781FE2C6070BD0228BB
:10554000FCD10C4E3368022BF8D00C4D06F00CFE4B
:105550002B68C01A0A4B1B689842EFD909490A20E8
:10556000FFF76CFE346006F0FFFD2860E6E700BF41
:10557000080C0020900100203E0100201C080020A3
:10558000E0010020340100202DE9F0417C4D2C6821
:105590002CB9FCF7CEF92B6853B9BDE8F081012C8A
:1055A00003D1FCF7CAF90120D4E0022C00F0CA8034
:1055B00006F0DAFD734E744FDFF8D08104463046B2
:1055C00005F098FD0546002840F0C78006F0CCFDA8
:1055D0003A68031B9342F2D36C4C6422236DB3FBF5
:1055E000F2F36B4A84F84D5004F14C00136000F064
:1055F000C7FD684B186004F14C0000F0CBFD664B12
:10560000186004F14C0000F0D3FD644B1860204694
:1056100000F04AFD51EC100BFBF7D6FA604B186016
:10562000204600F065FD51EC100BFBF7CDFA5D4B09
:1056300084F87D501860D4F88400FAF763FF0022E4
:10564000594BFBF7F3F8FBF7BFFA584B84F85D5062
:105650001860606EFAF756FF45A3D3E900230646AB
:105660000F46FAF7B9FF504B0022FBF7DFF8FBF7C4
:10567000ABFA4F4B394618603FA3D3E900233046BD
:10568000FAF7AAFF0022484B4A4E4B4FFBF7CEF8E1
:10569000FBF79AFA494B84F88D501860D4F894308F
:1056A000D4F8A400336084F89D50FAF72BFF3E4BEA
:1056B000434D0022FBF7BAF8FBF786FA2860FCF7A7
:1056C00095FB3B6813B33F4C237843B93368022BF7
:1056D0001CDC06F049FD3C4B18600123237006F0EA
:1056E00043FD394A1368C01A3B6898420ED93368A3
:1056F000022B4FF000032370136007DCFDF75AF80C
:105700004FF47A7006F034FDFFF79EFD2F4B1A78A8
:105710002F4B52B395ED007AF2EE0E7AB4EEE77AA3
:10572000F1EE10FA0BDC2B4A9FED2B7AD2ED007ACA
:10573000F0EEE77AF4EEC77AF1EE10FA15DD012209
:105740001A702AE7FCF7F9F81A4B1B68062B7FF74B
:105750002AAF2046FFF7E2FE1DE7304605F064FF62
:10576000C1B2404600F09AFE29E70022E8E700BFF8
:10577000CF16AD2F5476E03F6F1283C0CAA1FD3F14
:10578000E4010020300A0020F00100200C0C002071
:105790006C080020680800206408002060080020D1
:1057A0009808002094080020000059405C08002060
:1057B0005808002050080020EC0100205408002068
:1057C0004C08002024080020200800201008002099
:1057D0001108002030080020000096433D4B1B6854
:1057E00070B53D4C034423603C4B1B782BB13C4BC4
:1057F0001B7813B13B4B01221A703B4B1B78A3B3B0
:105800003A4B1B68032B30DC394B1B686BB3354BB1
:105810001B7853BBFBF71EFE0120FFF77FFE354EC2
:105820001424FCF7FFFEFCF799FEFFF7ADFE3046AF
:1058300005F060FC002801DDFDF7DAFF0525FFF724
:1058400089F80121262006F055FCC82006F090FCBE
:105850000021262006F04EFC40F2EE2006F088FCE7
:10586000013DECD1013CDCD170BD013841F2863301
:10587000984229D9204B1B780BB1FBF7EBFD06F0C2
:1058800073FC23689842EFD2FFF764F8FCF7CAFE76
:10589000FCF764FEFFF778FE002210460121FFF7B7
:1058A00073FAFCF765F9012211461046FFF76CFA0E
:1058B000E5E7FFF74FF8FCF7B5FEFCF74FFE0022D7
:1058C00011461046FFF760FA06F04EFC2368984236
:1058D000EFD3C9E7280800202C080020E8010020A9
:1058E0001008002012080020E901002050080020C4
:1058F000E4010020D80800205C02002010B5FFF76A
:1059000029F8012108460022FFF73EFAFCF78AFE3B
:10591000FFF73AFEFCF722FE002210460121FFF7B6
:1059200033FAFCF725F9012211461046FFF72CFA4D
:10593000FCF770FFFFF70EF8FCF774FE0121002260
:105940000846FFF721FA324B1B7853B1FFF77CF979
:10595000FFF700F8FCF766FE012100220846FFF77A
:1059600013FA2C4B1B7853B1FDF7CAF8FEF7F2FF80
:10597000FCF758FE012100220846FFF705FA264CE5
:10598000237853B1FDF7A4F9FEF7E4FFFCF74AFED4
:10599000012100220846FFF7F7F9FEF7DBFFFCF7CD
:1059A00041FE012100220846FFF7EEF923781B4C47
:1059B0008BB123787BB1FFF7E7FDFCF7CFFD002229
:1059C00010460121FFF7E0F9FCF7D2F80122114659
:1059D0001046FFF7D9F9FEF7BDFFFCF723FE0121C2
:1059E00000220846FFF7D0F9237853B1FDF7E8FA13
:1059F000FEF7B0FFFCF716FE012100220846FFF774
:105A0000C3F9074BBDE810401868FFF7E7BE00BFB9
:105A1000A908002024020020540200204502002092
:105A2000580200202DE9F0411C46454B83670123B5
:105A30001646A0F87C300D4668220021DDF818805B
:105A4000074606F005FEF3B2312B28D83D4A52F83E
:105A5000233006F4E0661E43EBB2312BBE6632D82B
:105A6000384A52F8233005F4E0651D43E3B2312B88
:105A7000FD663CD8334A52F8233004F4E0641C43FA
:105A80005FFA88F2312A3C6745D82E4951F8222026
:105A900008F4E06313437B673846BDE8F08106F005
:105AA000C002C02A0CD1CE2B0AD8274B06F03F02E9
:105AB00006F4E06653F82220224B53F82230CAE75E
:105AC0004FF0FF36C8E705F0C002C02A0CD1CE2B3C
:105AD0000AD81D4B05F03F0205F4E06553F822207B
:105AE000184B53F82230C0E74FF0FF35BEE704F003
:105AF000C002C02A0CD1CE2B0AD8134B04F03F02AF
:105B000004F4E06453F822200E4B53F82230B6E739
:105B10004FF0FF34B4E708F0C003C02B0CD1CE2AFD
:105B20000AD8094B08F03F0253F82210054A08F43E
:105B3000E06352F82120ADE74FF0FF33ABE700BF41
:105B400000093D00F8E70008BCE70008002210B497
:105B500006495DF8044B80F85D200123816780F8D9
:105B60007C3080F87D2000F04FB800BF00093D0078
:105B700007B5002A8DF807100DF107014FF001035A
:105B80000CBF0A46002200F045F99DF8070003B05B
:105B90005DF804FB07B532230093C622C123C72159
:105BA0000248FFF73FFF03B05DF804FBE80C00205C
:105BB00030B591FAA1F391FAA1F1B3FA83F3C46875
:105BC0005B000325B1FA81F105FA03F3490024EAE9
:105BD00003038A401A43C26030BD0000074A0346EF
:105BE00010684BB1064A934201D102F0A5B9054AAB
:105BF000934201D102F08EB9704700BFD402002059
:105C000000300140003800402DE9F74F0E461546A0
:105C10001F460446002800F0C2807549C06E04F09B
:105C2000EBFD74498146A06E04F0E6FD724983469F
:105C3000206F04F0E1FD71498046606F04F0DCFDE7
:105C40008246B9F1000F00F0AA80BBF1000F00F00E
:105C5000A680B8F1000F00F0A2805946484604F033
:105C6000F2FD51468146404604F0EDFD0146804676
:105C7000484604F0E8FD6066B9F1000F00F08F803F
:105C8000B8F1000F00F08B80002800F08880626F70
:105C90002060511C0CBF4FF400724FF480224FF46F
:105CA0008273A2616360FFF799FFB6EB500F79D260
:105CB000B6EB900F78D2B6EBD00F77D2B6EB101FC1
:105CC00076D2B6EB501F75D2B6EB901F74D2B6EBFE
:105CD000D01F2CBF30233823E361002D6ED0022D5E
:105CE0006ED0013D18BF01256D000123B7FA87F77B
:105CF000C4E904537F0907230026E362FF014FF440
:105D0000E063E3603A49E06EA660C4E90876A66203
:105D1000666304F059FD3749A06E04F055FD206F0D
:105D2000354904F051FD2369B342236FC3F30311D6
:105D300014BF01220222042998BF314803F00F0347
:105D400098BF50F821002F4988BF3046022A51F8E9
:105D5000231018BF0122FFF72BFF2849606F04F0C2
:105D600033FD2368284A93422CD1284B1A6E42F403
:105D700080521A661A6E02F480520092009A1A6CCF
:105D800042F480521A641A6C22F480521A6420463B
:105D900002F003F92268136843F04003136003B074
:105DA000BDE8F08F002397E7082395E7102393E7DA
:105DB000182391E720238FE728238DE72B4695E7CB
:105DC000002393E7124A9342E1D1104B9A6D42F4BB
:105DD00080429A659A6D02F480420192019A9A6B10
:105DE00042F480429A639A6B22F480429A63CEE72F
:105DF00000E30008B8E2000870E2000828E20008AA
:105E000098020020A0E1000800300140001002408C
:105E1000003800402DE9F0410D4616461C4633B3CC
:105E2000076800F0D3FB8046BB689907FCD5D5B165
:105E300015F8013B3B73BB68DA07FCD53B7B0EB121
:105E400006F8013B00F0C2FBA0EB0800B0F57A7F3A
:105E500004F1FF3409D2002CE6D12046BB681B06B2
:105E6000FCD4BDE8F081FF23E4E70120F6E702203F
:105E7000F7E7000008B5034903484FF4006206F055
:105E80007FFC08BD00F80108680D002010B504462D
:105E9000FFF7F0FF014B185D10BD00BF680D00203B
:105EA00070B5002386B0CDE901330122144B039273
:105EB000B3F8E035D340013BCDE9043201F078FA84
:105EC000D8B9104B9A6942F040429A614CF2FA32CA
:105ED0001A6101A902A801F057FB60B90A4D0B4CE9
:105EE0000B4EF5E802232146002001F0A7FA10B975
:105EF0000834B442F5D101F06DFA06B070BD00BFB0
:105F00000070FF1F00200240680D002000F801080B
:105F100000000208014B1954FFF7C2BF680D0020B2
:105F2000302180F834104E21002280F836100221F2
:105F300002808280826002730282426102768283E2
:105F4000026280F824200285C26280F830208287B5
:105F50000264A0F84C200265A0F85C204266A0F81C
:105F60006C204267A0F87C20C0F88420A0F88C2028
:105F7000C0F89420A0F89C20C0F8A42080F8BD10A0
:105F8000A0F8BE2080F8C020C0E93122C0E9332249
:105F9000C0E93522A0F8AC2080F8AE207047A1F10E
:105FA0004103052B02D8A1F137007047A1F161032D
:105FB000052B94BFA1F15700A1F13000704738B50F
:105FC000057804462D2D08BF0134204606F056F909
:105FD00064235843224614F8013BA3F130010929F8
:105FE000F8D92E2B0BD15378303B092B07D80A2137
:105FF00001FB03009378303B092B98BFC0182D2D6F
:1060000008BF404238BD000038B50D46044606F0D2
:1060100035F964231349B0FBF3F203FB12034B433E
:106020002A8020460278A2F13004092C014600F1B2
:106030000100F7D92E2A0BD10A480A2403E0B0FB4D
:10604000F4F000FB023311F8012F303A092AF6D997
:1060500003EB830301330322B3FBF2F36B600023F2
:106060002B7238BD80969800C36910B54360036AEF
:10607000836090F824300373836A0361C36A4361C9
:1060800090F83030037690F8353080F8343090F85E
:10609000373080F83630044606F066F840F20113D7
:1060A000A063238010BD00000023D0B504464370D8
:1060B0008068FAF717FA0CA3D3E90023FAF7B6FBC6
:1060C0000646A0880F46FAF71DFA0B4602463946E7
:1060D0003046FAF7CBF8237B13B101F100431946A0
:1060E00041EC100BD0BD00BF0000000065CDCD41DC
:1060F0000023D0B5044643704069FAF7F3F90CA3C6
:10610000D3E90023FAF792FB0646208A0F46FAF7F6
:10611000F9F90B46024639463046FAF7A7F8237ECE
:1061200013B101F10043194641EC100BD0BD00BF83
:106130000000000065CDCD4110B583684360044682
:1061400006F012F840F20113E060238010BD10B594
:1061500083684360044606F007F840F20113E060EC
:10616000238010BD10B504460846FFF728FFA06045
:1061700010BD10B50446084606F080F8A06010BDBA
:10618000002343704068024BB0FBF3F0C0B270478D
:1061900040420F0000234370406842F21073B0FB8E
:1061A000F3F06423B0FBF3F203FB1200C0B27047BC
:1061B0000023437064234068B0FBF3F0B0FBF3F2BC
:1061C00003FB1200C0B2704710B5C3688360044679
:1061D00005F0CAFF40F201136060238010BD10B5C6
:1061E00004460846FFF7EBFEE06010BD10B5C3683B
:1061F0008360044605F0B8FF40F20113606023801D
:1062000010BD10B50446084606F038F8E06010BD31
:1062100010B501460446103006F0AAFA05F0A4FFB6
:1062200040F201132062A38410BD0F2206F050BA81
:1062300070B590F8AD600446002E65D090F8AE10B1
:10624000FFF7ADFE94F8AF1002462046FFF7A7FE19
:1062500094F8AC3000EB0210C0B283424DD1D4F8B8
:10626000D8300133C4F8D83094F8C03023B1D4F812
:10627000D0300133C4F8D03094F8BD301BB3012BBB
:1062800015D104F13C00FFF757FF04F14C00FFF774
:106290005EFF94F8C03053B12046FFF7E5FE04F1ED
:1062A0005C00FFF791FF04F16C00FFF78DFFD4F85D
:1062B000C85035B1D4F8C830A86A996AF9F768FFB0
:1062C000B0B1304670BD04F14C00FFF740FF94F8C8
:1062D000C03033B12046FFF7C7FE04F17C00FFF762
:1062E00073FF04F18C00FFF781FF04F19C00DCE7F1
:1062F0002846FFF78DFF2D6BDBE7D4F8D430013350
:10630000C4F8D4300026DCE790F8BE209ABB90F8A1
:10631000AE30472B29D190F8AF105D4806F0CBF98D
:1063200018B304F1B0055B492846F9F731FFF0B125
:1063300059492846F9F72CFF003818BF01204000C2
:10634000D4F8C45084F8BD0004F1AE06C4F8C850B7
:10635000002DD7D0A86A3146F9F71AFF002808DBCC
:10636000D0D00023C4F8C830CCE70220E8E70120F1
:10637000E6E72D6BEAE790F8BD10022924D090F8EB
:10638000AE300BB342EA4112013A2B2A1CD8DFE8A7
:1063900002F0163C434A4D646D73771B1B1B1B1B9D
:1063A0001B1B1B1B1B1B1B1B1B1B1B1B1B1B1B1B3D
:1063B0001B1B16353C434A4D545A5E1B1B7B00F198
:1063C000AE014C30FFF7CEFED4F8C85004F1AE0653
:1063D000002D97D0D4F8C830A86A996AF9F7D8FE8A
:1063E00000288FD1EA6A94F8BE309A428ADC03D141
:1063F00031462846FFF719FF2D6BE9E7A3F141006D
:106400004342434184F8C030DEE700F11C0104F14F
:10641000AE00FFF7F9FDD7E7A3F153014B424B4123
:1064200080F82430D0E700F12801F0E7A3F157020B
:106430005342534180F83030C6E700F1AE015C3082
:10644000FFF7CDFEC0E700F1AE016C30F8E700F1D8
:10645000AE013C30FFF78DFEB6E7302B94BF002233
:10646000012280F8C02080F83530ADE700F1AE01A0
:106470008C30FFF7C6FEA7E700F1AE019C30DFE7E6
:1064800000F1AE017C30DBE780F837309CE700BFDD
:10649000D0E00008D6E00008DAE0000838B5D0F80F
:1064A000CC30242903F1010304460D46C0F8CC305A
:1064B0002AD090F8BF301CD80A2901D00D292FD13D
:1064C0000E2B4FF0000005D8234483F8AE00204681
:1064D000FFF7AEFE94F8BE30013384F8BE300023DF
:1064E00084F8BF30A5F12A035D425D4184F8AD50C8
:1064F00038BD2A29E4D02C2912D190F8AC2082F0A2
:106500002C0280F8AC20DBE700230222A0F8AC309C
:1065100080F8BD20A0F8BE3080F8C0300020E7E74A
:106520000D2B9FBF5A1C1B1984F8BF2083F8AE5057
:1065300094F8AD30002BF1D194F8AC305D4084F884
:10654000AC50EBE77047000038B50F4B1A780546A2
:106550000AB9012038BD4FF47A73B3FBF2F30B4A4A
:106560001068B0FBF3F000F03FFE04460028F0D1C5
:106570000F2DEED8024629464FF0FF3000F0E2FD25
:10658000034B20461D60E5E772020020D402002084
:106590007402002010B5032000F0C2FD0020FFF7B8
:1065A000D3FF044618B9FFF7CDFF204610BD0124E4
:1065B000FBE70000034A044B11681B780B4413608F
:1065C000704700BF6815002072020020014B186858
:1065D000704700BF6815002030B5CC0D04F00404EE
:1065E0001430C1F30451035907258D4023EA0503F4
:1065F0008A401343035130BD806800F001007047AA
:106600008068C0F38000704737B5002301930446CB
:10661000002800F0BF80456D25B903F07FFCA5651B
:1066200084F8505023689A68950041BF9A6822F018
:10663000204222F03F029A609A68D00040F189809F
:106640009A68D10000F19C80626D42F01002626590
:10665000A26D42F00102A26501211846FFF7D0FFAA
:10666000626D02F01002024340F09080626D22F4ED
:10667000817242F0020262651846FFF7BDFF78B9E9
:106680004548FFF7B9FF02464448FFF7B5FF02430C
:1066900006D143486568826822F47C122A438260EE
:1066A000E568626B94F820002A43A5682A43657E5A
:1066B000012842EA453242EA004202BF606A00F124
:1066C000FF3042EA4042A06A20B1E56A00F47070EF
:1066D00028430243DD68334828401043D8609A6855
:1066E00012071ED4D86894F83020257E520020F47A
:1066F000804042EA853220F002000243DA6094F8DA
:106700003820012A3ED1D4E90F2518692A436FF3B6
:106710008A000243606C0243A06C024342F0010213
:106720001A612269012A05BF186BE2691A6B02F12E
:10673000FF3206BF20F00F00024322F00F021A635F
:10674000636D23F0030343F001036365084603B060
:1067500030BD9A68144922F0104222F03F0242F004
:1067600080529A60114A1268B2FBF1F20132520073
:106770000192019A002A3FF463AF019A013AF7E7C8
:1067800000216AE71A6922F00102C9E7636D43F04C
:10679000100363650121D9E7000004500001045093
:1067A0000003045007C0F0FF400D0300D402002096
:1067B000354A2DE9F04145699768082D04460E4693
:1067C00007F01F0715D040F22123FB40D9070BD556
:1067D0000368DB6813F0010F0AD0636D43F02003F8
:1067E00063650120BDE8F081936813F4604FF3E71F
:1067F0000425FFF7EBFE804623681A682A4225D05D
:10680000626D42F400726265DA6812F4406F0FD173
:10681000627E6AB91A6816070AD5626D22F4807220
:106820006265626DD0045EBF626D42F00102626516
:10683000164A934204D140F22122FA40D1071BD5D7
:10684000DA68082D1BD11D600020CBE7721CD4D064
:10685000FFF7BCFEA0EB0800B04201D8002ECBD160
:1068600023681B682B40C7D1626D84F8503042F01A
:10687000040262650320B5E7054AD268E1E75204E5
:10688000E2D40C221A60DFE7000304500001045038
:10689000000004500368186C70470000F7B500232F
:1068A000019390F85030012B05460E4600F0AE8162
:1068B0000468012380F850302046FFF7A1FE00282D
:1068C00040F09E814B68052B06D8023B032B9ABFF4
:1068D000B74A32F8133006239909326801F00C01E7
:1068E00004F1300703F01F0378584FF01F0CC2F378
:1068F00084629A400CFA03F320EA03031A437A50A5
:106900002046FFF77DFEA26802F00802024325D16F
:10691000B3683168B3F1004F64D12046FFF75CFEE5
:10692000636943F00043636137697169E068336804
:10693000042F04F160025DD0C0F3C100400052F8A2
:1069400027C081409B4803F0F8430CEA000018433D
:1069500041EA000343F0004342F827302046FFF7A6
:106960004BFEA0BBF7683368934AD4F8B01007F029
:10697000180CC3F3120022FA0CF21A4021EA0001AB
:106980000A43C4F8B0208D4A974220D1002840F035
:1069900090809A0E013202F01F07092F4FF001017B
:1069A0004FEA826200F2A58002F0F842B94011433A
:1069B000002840F099809B0E013303F01F0303EB86
:1069C00043031B05B26819432046FFF705FE3168F3
:1069D0007B4B194240F0B5800020002385F85030F1
:1069E00003B0F0BD1A462046FFF7F6FD636923F0B9
:1069F000004398E7216E216EC3F31200C1F3846156
:106A0000002839D1C3F38463994202BF236E23F077
:106A100000432366636E3368616EC3F31200C1F3F3
:106A2000846100282FD1C3F38463994202BF636E4F
:106A300023F000436366936833689168C3F31200E0
:106A4000C1F3846130BBC3F38463994202BF93688E
:106A500023F000439360D3683368D168C3F3120016
:106A6000C1F38461E8B9C3F38463994202BFD36878
:106A700023F00043D36071E793FAA3F3002BC9D04E
:106A8000B3FA83F3C0E793FAA3F3002BD3D0B3FA9E
:106A900083F3CAE793FAA3F3002BDCD0B3FA83F3B2
:106AA000D3E793FAA3F3002B3FF458AFB3FA83F381
:106AB000DBE793FAA3F131B1B1FA81F2571C07F089
:106AC0001F07092F25D893FAA3F293FAA3F7B2FA76
:106AD00082F20132B7FA87F79206013702F0F842E4
:106AE00007F01F07012161E793FAA3F3B3FA83F3D9
:106AF00062E702F0F842B9401143A8B99B0E013396
:106B000003F01F0303EB43031E3B1B0543F000731D
:106B100058E7B1FA81F701329206013702F0F842E4
:106B200007F01F070121E6E793FAA3F2B2FA82F217
:106B3000013202F01F0203236FF01D0013FB02035A
:106B4000E3E7204B204E9A68B14202F0E0701DD17D
:106B500016023FF541AF1D4A94427FF43DAF9A685B
:106B600022F0E072024342F400029A60184B1A6865
:106B7000184BB2FBF3F20C2302FB03330193019B8E
:106B8000002B3FF429AF019B013BF7E7124EB142C6
:106B900024D1D1013FF520AF0C4A94427FF41CAFC1
:106BA0009A6822F0E072024342F080729A6013E722
:106BB00030E1000800F0FF03FFFF070000007F4006
:106BC0000000088000030450000052C70000045079
:106BD000D4020020400D0300000084CB0C4EB142D3
:106BE0007FF4FAAE52023FF5F7AE0A4A94427FF4C0
:106BF000F3AE9A6822F0E072024342F48002D5E7D5
:106C00006A6D42F020026A651846E6E60220E7E671
:106C10000100008000000450406D7047036870B5AB
:106C200004461846FFF7ECFC9A6802F0080202439B
:106C300001D1002070BDDA6892013AD5208B40F274
:106C40000112904235D1274A19684E0625D54022B7
:106C50001A6001211846FFF7D3FC50B19A689507D6
:106C600007D49A6822F0004222F03F0242F010025C
:106C70009A6001291FD10425FFF7A8FC0646236866
:106C80009B682B42D5D0FFF7A1FC801B0528F6D9C5
:106C900023689B682B42F2D001E0013AD4D1636DA6
:106CA00043F010036365A36D43F00103A365012066
:106CB000C0E70229CED19A6810070AD59A689207D0
:106CC00007D49A6822F0004222F03F0242F02002EC
:106CD0009A60022903D00329CDD10C25CCE70825E1
:106CE000CAE700BF010040A373B502680446002351
:106CF00010460193FFF780FC10B1002002B070BD78
:106D00009168214B194209D0636D43F0100363650C
:106D1000A36D43F00103A3650120EFE7936823F01F
:106D2000004323F03F0343F001039360174B9B683C
:106D300019021AD4FFF74AFC154E0546226813685B
:106D4000DB07DAD41046FFF757FC20B993683340CD
:106D500043F001039360FFF739FC401B0228EDD993
:106D600023681B68DA07E9D4CEE70A4B1A680A4B96
:106D7000B2FBF3F20C2302FB03330193019B002BC4
:106D8000D8D0019B013BF8E73F000080000304508E
:106D9000C0FFFF7FD4020020400D0300354B70B5CB
:106DA000044600689E68FFF72BFC054600285ED16C
:106DB00094F85030012B5AD0012384F850302046EB
:106DC000FFF792FF00284FD1636D2B4A23F47063C5
:106DD00023F0010343F4807363652368934206F054
:106DE0001F012FD100292FD1A2F58072656D25F4E6
:106DF00080156565656D15F480551CBFA56D25F082
:106E00000605A5651C251D6093424FF0000584F81A
:106E1000505005D040F2212525FA01F1C90715D5BA
:106E2000DA68920141BF626D22F4405242F480520E
:106E300062659A6822F0004222F03F0242F00402AA
:106E40009A6070BD1A46D1E70C4AD3E7636D43F4EC
:106E500080136365D3689B01F3D5636D23F44053BE
:106E600043F480536365ECE784F85050E9E702206F
:106E7000E7E700BF00030450000104500000045085
:106E8000026838B5044610469368FFF7B5FB08B9A9
:106E9000002038BD9907FBD4936803F00D03012B44
:106EA00019D1936823F0004323F03F0343F002031A
:106EB000936003231360FFF789FB054623689B68F3
:106EC000DB07E5D5FFF782FB401B0228F6D92368D4
:106ED0009B68DA07F2D5636D43F010036365A36D19
:106EE00043F00103A3650120D3E7000038B5044651
:106EF000002800F09880436D43F0020343650321AE
:106F0000FFF78CFE2268D36843F40013D360054674
:106F100030B92046FFF7B4FF054608B90123636581
:106F2000236842495A680A405A6040F2FF721A6068
:106F30009A6822F0A0429A609A6842F000529A60E1
:106F4000D8683B4A0240DA60DA683A4842F00042C8
:106F5000DA601A690A401A615A6902F080425A617D
:106F60009A6902F078429A611A6A02F0F0221A6273
:106F70005A6A02F0FF225A629A6A02F0FF229A626B
:106F8000196B2D4A0A401A635A6B2C490A405A63FE
:106F90009A6B0A409A63DA6B22F4FB6222F00702D2
:106FA000DA63196E264A11401966596E1140596606
:106FB000996E11409966D96E0A40DA66D3F8A0201E
:106FC00020490A40C3F8A020D3F8A4200A40C3F8FF
:106FD000A420D3F8B0200A40C3F8B020D3F8B420DE
:106FE00022F07F12C3F8B420FFF706FB03461648D1
:106FF000FFF702FB03430DD1144A936823F0FF739C
:1070000023F4F73323F48F7323F0010393602046B6
:1070100002F0A0FF0023C4E91733A36584F85030C1
:107020006365284638BD0125FBE700BF00F8FFFF78
:107030000480008000000450300882E0200882E0D4
:1070400000F0FF030000F8FF0001045000030450AB
:1070500010B590F85030012B044616D0012380F86B
:1070600050300321FFF7DAFD58B92046FFF708FF3B
:1070700038B9636D23F4885323F0010343F001030F
:107080006365002384F8503010BD0220FCE737B55B
:107090000023019390F85030012B04460D463CD05C
:1070A000012380F85030FFF7EBFE636D90BB23F4B3
:1070B000885323F00203226843F002036365936858
:1070C00023F0404323F03F0305F080452B4343F07A
:1070D000004393609368002B12DA019B0133019304
:1070E000019BB3F5912FF5D3636D23F0120343F0A9
:1070F00010036365002384F85030012003B030BDD5
:10710000636D23F0030343F001036365002384F8F8
:107110005030F3E743F01003F7E70220EEE70000FA
:107120000749CA6822F4E0620302120403F4E06330
:10713000120C134343F0BF6343F40033CB6070473A
:1071400000ED00E0164B30B5DC68C4F30224C4F156
:107150000703251D042B28BF0423062D4FF0FF3500
:107160008CBF033C002405FA03F321EA0303A54086
:1071700022EA0502A340002843EA0203ACBF00F163
:107180006040084A4FEA0313B8BF00F00F00DBB2BB
:10719000AABF00F56140135480F8003330BD00BF32
:1071A00000ED00E014ED00E0002807DB044A41098F
:1071B000012300F01F00834042F82130704700BFD8
:1071C00000E100E000280CDB4309064900F01F0045
:1071D00020330122824041F82320BFF34F8FBFF3B9
:1071E0006F8F704700E100E00138B0F1807F0BD273
:1071F0004FF0E023054A5861F02182F82310002067
:10720000072298611A6170470120704700ED00E085
:10721000002808DB4309044900F01F000122603305
:10722000824041F82320704700E100E0704708B534
:10723000FFF7FCFF08BD704710B5044608B90120F0
:1072400010BD437F03F0FF0213B90277FFF7F3FF8E
:10725000022363772379E3B92368134A5A619A6852
:1072600022F018029A6062792368D2B94FF0FF3297
:107270001A619A68616922F060020A439A609A680A
:10728000A16922F080020A439A60012363770020FB
:10729000D6E7D4E90212204600F008F80028E2D030
:1072A000CDE72269E4E700BFB71DC104CB0710B5E5
:1072B0000DD51F23013B1DD321FA03F4E407F9D5B3
:1072C000102A13D0102A04D83AB1082A10D001206D
:1072D0000BE0182AFBD1062BF9D8006841618368BE
:1072E00023F0180313438360002010BD072BF3E73E
:1072F0000F2BF1E7102AE5D1E9E790F82520022AC3
:10730000034606D00422C2630120002283F8242011
:1073100070470268116821F00E011160116821F0B8
:1073200001011160D0E91002012102F01C0201FAF2
:1073300002F2426083F825100020E6E710B590F8CD
:107340002520022A03D00422C263012010BD026856
:10735000836B116821F00E011160116821F00101A9
:107360001160D0E91042012102F01C0201FA02F280
:107370006260002280F8251080F8242003B198472D
:107380000020E3E7094A536943F4802310B55361B1
:10739000EFF3108272B60023CC58C4500433B3F517
:1073A000807FF9D182F3108810BD00BF0020024019
:1073B000064B5A69002ABFBF054A9A6002F188321B
:1073C0009A60BABF5869C00F002070470020024081
:1073D00023016745034A536943F00043536100208A
:1073E000704700BF0020024070B50546FFF7EEF879
:1073F0000F4C06462369DA030AD423690D4A134069
:107400000FD00D494A681A434A600120236170BDBC
:10741000691CEFD0FFF7DAF8801BA842EAD30320FB
:10742000F5E72369DB0744BF012323610020EEE772
:1074300000200240FAC30200780200202DE9F84340
:10744000254D99462B78012B04460F46904641D096
:1074500001234CF250302B70FFF7C6FF064630BBBD
:1074600068601E48026812F4806217BF03682A77BA
:1074700023F4806303601CBF02232B77E4B94369C4
:1074800043F001034361C7F80080BFF36F8F01240D
:10749000C7F804904CF25030FFF7A6FF064624B11F
:1074A0000E4A536923EA0403536100F03DF80023B8
:1074B0002B703046BDE8F883631E012B08D8414687
:1074C0003846FFF75FFFA31E5C425C41A404E1E77E
:1074D0000024DFE70226ECE77802002000200240CB
:1074E000064B10F0010F1EBF5A6942F004025A61A8
:1074F0005A6942F480325A61704700BF002002404E
:10750000084B5A69C00022F4FC7200F4FF6010437B
:1075100058615A6942F002025A615A6942F4803253
:107520005A617047002002401548037FDAB203F029
:10753000FD03012B10D1134B196821F40071196060
:10754000196841F400611960196821F4006119603B
:10755000196841F400711960931E012B0CD8094B76
:107560001A6842F480521A601A6822F480521A6033
:107570001A6842F480621A6000230377704700BFE4
:1075800078020020002002402DE9F843314D2B788D
:10759000012B064688465AD001274CF250302F70F6
:1075A000FFF722FF044610BB2B4B68601A6812F4E9
:1075B000007F1A6820D0510506D51A6822F480622F
:1075C0001A6003232B7700E02F773368012B1DD13E
:1075D0007068FFF785FF4CF25030FFF705FF1E4A39
:1075E000536923F0040304465361FFF79DFF002312
:1075F0002B702046BDE8F883520505D51A6822F4A1
:1076000080621A600223DDE72877DEE74FF0FF3360
:10761000C8F80030B768DFF84090D6E9023213446A
:10762000BB42E2D971683846FFF76AFF4CF250302E
:10763000FFF7DAFED9F8143023F4FD73C9F81430DB
:1076400018B1C8F800700446CFE70137E5E7022417
:10765000CFE700BF7802002000200240044A5169B1
:10766000014208B502D0506102F046FF08BD00BFDC
:1076700000040140024A136843F4807313607047AA
:1076800000700040024B186800F4C060704700BFF3
:1076900000700040174A1368B0F5007F03F4C06320
:1076A0001BD1B3F5007F1BD0136823F4C06343F4F0
:1076B00000731360104B1B6832214B430F49B3FB1F
:1076C000F1F301335169490500D523B953695B05CD
:1076D00006D503207047013BF4E7B3F5806F01D175
:1076E00000207047136823F4C06343F48063136081
:1076F000F6E700BF00700040D402002040420F00B7
:1077000037B51E4DAB6DDA00044618D5FFF7BAFF4A
:10771000B0F5007F23D1802C29D9A02C8CBF022466
:10772000012417490A6822F0070222430A60086808
:1077300000F00700001B18BF012003B030BDAB6D87
:1077400043F08053AB65AB6D03F080530193019B15
:10775000FFF798FFAB6D23F08053AB65D8E7802C23
:1077600007D808D0A4F170035C425C41D9E700243B
:10777000D7E70324D5E70224D3E700BF0010024077
:1077800000200240204B9A68D96812F00C0205D004
:107790000C2A2CD101F0030101292FD119681B48B3
:1077A000090755BFD3F894101968C1F30321C1F339
:1077B000031150F8210032B3DA6802F00302022A02
:1077C0001ED01349032A08BF0846D968DA68C2F3F5
:1077D00006224243D868C0F34160C1F30211013070
:1077E00001314000B2FBF1F2B2FBF0F07047042A25
:1077F00008D0082A064818BF002070470020DBE7A1
:107800000448E2E70348704700100240E0E1000846
:1078100000127A000024F4002DE9F743054618B958
:10782000012003B0BDE8F083944C0368A668E768C4
:10783000DB0606F00C0607F003073DD51EB10C2E43
:107840006AD1012F68D12368980702D5EB69002B14
:10785000E6D02368686A190756BFD4F894302368C5
:107860001B0903F0F00398423FD9FFF749FF0028B6
:10787000D6D1236843F00803236023686A6A23F0A3
:10788000F0031343236063682A6A23F47F4343EAC7
:1078900002236360FFF776FFA368794AC3F30313FB
:1078A000D35C03F01F03D840764B1860764B186802
:1078B000FEF74AFE0028B4D12B68D80763D42B68A2
:1078C000990700F1A2802B68180700F1DF802B6870
:1078D000590700F12F812B68990600F1AB81EB6A03
:1078E000002B40F0D18100209BE7236843F0080380
:1078F0002360236823F0F0030343236063682A6A4C
:1079000023F47F4343EA02236360002EC2D1FFF7D2
:10791000F7FE0028BED083E7EB691BB3236843F072
:1079200001032360FEF752FE804623689A0711D5B3
:10793000236843F00803236023686A6A23F0F00396
:107940001343236063682A6A23F47F4343EA0223D4
:107950006360B1E7FEF73AFEA0EB08000228E4D925
:1079600003205EE7236823F001032360FEF72EFE69
:10797000804623689B079FD5FEF728FEA0EB0800F2
:107980000228F6D9ECE7082E03D00C2E08D1032FDD
:1079900006D123689A0392D56B68002B8FD13FE7FD
:1079A0006B68B3F5803F10D1236843F480332360C4
:1079B000FEF70CFE804623689B0380D4FEF706FE8C
:1079C000A0EB08006428F6D9CAE7B3F5A02F04D1CC
:1079D000236843F480232360E6E7226822F48032A0
:1079E0002260226822F480222260002BE0D1FEF780
:1079F000EDFD8046236898037FF561AFFEF7E6FD55
:107A0000A0EB08006428F5D9AAE7042E03D00C2EB9
:107A100010D1022F0ED12368590503D5EB68002B36
:107A20003FF4FEAE63682A6923F0FE4343EA026333
:107A3000636048E7EB687BB1236843F4807323609D
:107A4000FEF7C4FD074623685A05EBD4FEF7BEFDDA
:107A5000C01B0228F7D983E7236823F480732360CF
:107A6000FEF7B4FD074623685B057FF52CAFFEF7F4
:107A7000ADFDC01B0228F6D972E700BF001002401E
:107A800018E20008D4020020740200206B69002B69
:107A90003CD0D4F89430A96903F0100291420ED082
:107AA00003F00302022A3FF4BBAEDA071BD4D4F87A
:107AB0009430AA6923F010031343C4F89430D4F827
:107AC000943043F00103C4F89430FEF77FFD07467D
:107AD000D4F8943098073FF5FAAEFEF777FDC01B57
:107AE0001128F5D93CE7D4F8943023F00103C4F809
:107AF0009430FEF76BFD0746D4F894309B07D6D53B
:107B0000FEF764FDC01B1128F6D929E7D4F894309C
:107B100023F00103C4F89430FEF758FD0746D4F86B
:107B2000943099077FF5D3AEFEF750FDC01B1128A6
:107B3000F5D915E7A36DDA0030D4A36D43F0805377
:107B4000A365A36D03F080530193019B0127DFF828
:107B50006C82D8F80030DB0522D5AA68D00733D470
:107B6000D4F8903023F00103C4F89030D4F890306A
:107B700023F00403C4F89030002A3CD1FEF726FD20
:107B800041F288398046D4F8903098074BD4D4F825
:107B9000903023F08003C4F8903035E00027D6E71A
:107BA000D8F8003043F48073C8F80030FEF70EFDBB
:107BB0008146D8F80030D905CFD4FEF707FDA0EBF9
:107BC00009000228F5D9CBE6D4F8903002F0800104
:107BD00023F080030B43C4F89030D4F89030520760
:107BE00042BF43F00403C4F89030D4F8903043F01F
:107BF0000103C4F89030FEF7E9FC41F28839804671
:107C0000D4F890309B0707D5002F3FF464AEA36DE6
:107C100023F08053A3655EE6FEF7D8FCA0EB0800D6
:107C20004845EDD99CE6FEF7D1FCA0EB080048459D
:107C3000A9D995E6AB6A9BB1D4F8983043F001031B
:107C4000C4F89830FEF7C2FC0746D4F898309A077B
:107C50003FF545AEFEF7BAFCC01B0228F5D97FE61A
:107C6000D4F8983023F00103C4F89830FEF7AEFC46
:107C70000746D4F898309B077FF531AEFEF7A6FC97
:107C8000C01B0228F5D96BE6022B7AD1E3682A6B78
:107C900003F0030191421CD1696B03F070020139BA
:107CA000B2EB011F15D1A96B03F4FE42B2EB012F19
:107CB0000FD1EA6B520803F4C001013AB1EB425F05
:107CC00007D12A6C520803F0C063013AB3EB426F4C
:107CD0003ED00C2E3FF4A4AD236823F080732360C4
:107CE000FEF774FC064623689F012BD4E268324BF2
:107CF00013402A6B1343AA6B43EA02236A6B013ACF
:107D000043EA0213EA6B5208013A43EA42532A6CEF
:107D10005208013A43EA4263E360236843F0807308
:107D20002360E36843F08073E360FEF74FFC054691
:107D3000236898013FF5D7ADFEF748FC401B0228A9
:107D4000F6D90DE6FEF742FC801B0228CBD907E6E8
:107D5000236899013FF5C7AD236843F08073236022
:107D6000E36843F08073E360FEF730FC0546236868
:107D70009A013FF5B8ADFEF729FC401B0228F6D961
:107D8000EEE50C2E3FF44CAD236823F080732360A6
:107D9000FEF71CFC054623689B0106D4E36823F02C
:107DA000887323F00303E3609DE5FEF70FFC401B9F
:107DB0000228F0D9D4E500BF8C809FF90070004004
:107DC0002DE9F0410D46044610B90120BDE8F081CF
:107DD0004B4A136803F007038B422CD321688807B2
:107DE00034D4C9073FD421688A0768D4444A136849
:107DF00003F00703AB426FD811F0040F414D77D168
:107E00000B0706D5AB68226923F4605343EAC2032B
:107E1000AB60FFF7B7FCAB683B4AC3F30313BDE8A5
:107E2000F041D35C03F01F03D840384B1860384B47
:107E30001868FEF789BB136823F007030B43136030
:107E4000136803F007038B42BFD1C7E72D4AA06830
:107E5000936803F0F003984281BF936823F0F00326
:107E600003439360BDE76268264E032A33681AD144
:107E700013F0007FA9D0B36823F003031343B3606A
:107E8000FEF7A4FB41F288380746B368626803F046
:107E90000C03B3EB820FA6D0FEF798FBC01B404546
:107EA000F3D9032092E7022A02D113F4003FE1E75D
:107EB00012B913F0020FDDE713F4806FDAE7114A0D
:107EC000A068936803F0F00398423FBF936823F0E3
:107ED000F0030343936089E7136823F007032B4300
:107EE0001360136803F00703AB427FF46EAF83E7C0
:107EF000AB68E26823F4E0631343AB6080E700BF44
:107F0000002002400010024018E20008D4020020C5
:107F100074020020054B064A9B68C3F30223D35C1E
:107F2000044A106803F01F03D84070470010024055
:107F300010E20008D4020020054B064A9B68C3F3F8
:107F4000C223D35C044A106803F01F03D840704773
:107F50000010024010E20008D40200200F2303604A
:107F60000B4B9A6802F0030242609A6802F0F0023A
:107F700082609A6802F4E062C2609B68DB0803F4E6
:107F8000E0630361034B1B6803F007030B6070475A
:107F90000010024000200240704770B504460028DF
:107FA00063D0436A002B59D14268B2F5827F00D07A
:107FB000C3610023A36294F85D3003F0FF0223B98C
:107FC00084F85C202046FFF7E7FF2068E168022381
:107FD00084F85D300368B1F5E06F23F0400303607F
:107FE0004FF000033ED91D46B1F5706F18BFA36274
:107FF000A6686368A26906F4044603F482733343F7
:10800000266906F002063343666906F0010633432B
:1080100002F400763343E66906F038063343266AF5
:1080200006F080063343A66A06F400563343036025
:10803000666B636A06F0080603F01003334301F42D
:108040007061120C0B4302F0040213432B43436094
:1080500000200123206684F85D3070BD0023C0E954
:108060000433A6E74FF48055C0E70120F5E7000090
:10807000036A026A22F00102026270B542688469F2
:108080000D6824F4803424F073042C438D6823F0AD
:1080900002032B430E4DA84207D005F5A055A84278
:1080A00003D005F58065A8420BD1CD6823F0080305
:1080B0002B43D1E9055622F44072354323F00403E3
:1080C0002A4342604A6884614263036270BD00BF14
:1080D000002C0140036A026A22F48072026270B5C9
:1080E0004268C4690D6824F4803424F073042C437E
:1080F0008D6823F4007343EA05230F4DA8420ED187
:10810000CD6823F4006343EA052323F48063D1E9B7
:10811000055622F44052354342EA051206E0074D67
:10812000A842F4D005F58065A842F0D042604A68C4
:10813000C461C263036270BD002C01400040014075
:10814000026A036A23F48053036230B54468C3694A
:108150000D6823F0807323F4E64343EA05238D681A
:1081600022F4005242EA05320A4DA84207D005F532
:10817000A055A84203D005F58065A84204D14D69F9
:1081800024F4804444EA85144460C3614B6803646A
:10819000026230BD002C0140026A036A23F480337E
:1081A000036230B54468436D0D6823F4803323F0D7
:1081B00070032B438D6822F4003242EA05420B4DD6
:1081C000A84207D005F5A055A84203D005F5806563
:1081D000A84204D14D6924F4803444EA0524446063
:1081E00043654B688365026230BD00BF002C0140CF
:1081F000026A036A23F48013036230B54468436D56
:108200000D6823F0807323F4E04343EA05238D686F
:1082100022F4001242EA05520A4DA84207D005F5A1
:10822000A055A84203D005F58065A84204D14D6948
:1082300024F4802444EA8524446043654B68C36584
:10824000026230BD002C014090F83D30012B1BD163
:1082500002230E4A80F83D300368934206D0B3F102
:10826000804F03D002F5A052934207D19968084A83
:108270000A40062A06D0B2F5803F03D01A6842F0C1
:1082800001021A600020704701207047002C014055
:108290000700010090F83C20012A03464FF002003D
:1082A00009D01A6883F83D0051610020012283F84B
:1082B0003D2083F83C00704770477047036870B5F5
:1082C000DD681E69B20704460DD5A9070BD56FF00E
:1082D00002021A61012202779B699A0775D001F0A8
:1082E000A6FD00232377730710D568070ED52368F2
:1082F0006FF004021A61022222779B6913F4407F17
:10830000204668D001F093FD0023237731070FD575
:108310002A070DD523686FF008021A61042222771C
:10832000DB699B0720465CD001F081FD00232377A9
:10833000F10610D5EA060ED523686FF010021A6117
:1083400008222277DB6913F4407F20464FD001F0EA
:108350006EFD00232377F30708D5E80706D52368C9
:108360006FF001021A61204601F03EFD16F4025F33
:1083700008D0290606D523686FF402521A612046F8
:1083800000F093FBF20508D52B0606D523686FF4A1
:1083900080721A61204600F089FB700608D56906D4
:1083A00006D523686FF040021A612046FFF785FF6B
:1083B000B20622D5AB0620D523686FF020022046F6
:1083C0001A61BDE8704000F06FBB01F02EFD204641
:1083D000FFF772FF85E701F028FD2046FFF76CFFED
:1083E00092E701F022FD2046FFF766FF9EE701F0CD
:1083F0001CFD2046FFF760FFABE770BD1B4A03681A
:1084000090420BD0B0F1804F08D002F5A0529042BC
:1084100009D1CA6823F44073134307E04A6823F084
:1084200070031343F5E7124A9042F2D04A6923F0F1
:108430008003134303608B68C3620B6883620B4B3A
:10844000984207D003F5A053984203D003F5806308
:10845000984201D10B690363012343610369DB0780
:1084600042BF036923F0010303617047002C014000
:108470000044014010B5044650B390F83D3003F07D
:10848000FF021BB980F83C2002F0EAFA02232068C0
:1084900084F83D30211DFFF7B1FF012384F84830F7
:1084A000002084F83E3084F83F3084F8403084F86F
:1084B000413084F8423084F8433084F8443084F802
:1084C000453084F8463084F8473084F83D3010BD9C
:1084D0000120FCE7036A026A22F01002026270B512
:1084E000426884690D6824F0807424F4E64444EA08
:1084F00005248D6823F0200343EA05130F4DA8429D
:108500000ED1CD6823F0800343EA051323F0400326
:10851000D1E9055622F44062354342EA850206E07D
:10852000074DA842F4D005F58065A842F0D042601E
:108530004A6884618263036270BD00BF002C014001
:108540000040014010B590F83C30012B044629D082
:108550000C2A1FD009D8042A14D0082A16D062B1D8
:108560000120002384F83C3010BD102A16D0142AB4
:10857000F6D10068FFF73CFE02E00068FFF778FDE7
:108580000020EEE70068FFF7A5FFF9E70068FFF7B6
:10859000A1FDF5E70068FFF7D3FDF1E70068FFF7FD
:1085A000FBFDEDE70220DFE738B590F83C30012B0A
:1085B000044673D001200C2A84F83C004ED008D821
:1085C000042A2BD0082A39D0BAB1002384F83C30D1
:1085D00038BD102A52D0142AF7D12068FFF708FEC0
:1085E000436D0A6943F400634365436D23F480637C
:1085F0004365436D43EA02234EE02068FFF738FDF0
:1086000083690A6943F008038361836923F00403E3
:1086100083618369134383610020D6E72068FFF7F5
:1086200059FF83690A6943F400638361836923F412
:1086300080638361836943EA0223ECE72068FFF7E4
:1086400049FDC3690A6943F00803C361C36923F0A4
:108650000403C361C3691343C361DDE72068FFF707
:108660006FFDC3690A6943F40063C361C36923F4FE
:108670008063C361C36943EA0223EDE72068FFF723
:108680008BFD436D0A6943F008034365436D23F096
:1086900004034365436D13434365BDE7022097E739
:1086A00070B5056A046A0F4E24F001040462B042FA
:1086B000846912D0B0F1804F0FD006F5A056B042B9
:1086C0000BD044F0010263F3071201F00A0125F018
:1086D0000A0319438261016270BD24F0030422433E
:1086E000F1E700BF002C0140F8B590F83C30012BB9
:1086F00005460C4600F082800120082A85F83C00DF
:108700005CD006D842B3042A36D0002385F83C302A
:10871000F8BD0C2AF9D12B68CE68186AD1E9002778
:10872000196A21F480511962D969120321F4407148
:1087300041EA072120F4204002F4204266F30F3181
:108740000243D9611A62DA69A16822F44062DA61EF
:10875000DA6942EA01224FE02868CB68D1E90012C9
:10876000FFF79EFF8369A26823F00C03836183698E
:10877000134383610020C8E72B68CE68186AD1E9EB
:108780000027196A21F0100119629969120121F478
:10879000407141EA072120F0A00002F0A00266F338
:1087A0000F31024399611A629A69A16822F440620A
:1087B0009A619A6942EA01229A61DBE72B68E768CD
:1087C000186A1E6A26F48076D1E900211E62DE69ED
:1087D000120226F00306314320F4206002F42062E6
:1087E00067F307110243D9611A62DA69A16822F0BE
:1087F0000C02DA61DA690A43DA61BBE7022087E733
:10880000036A01F01F0110B501248C4023EA040320
:108810000362036A8A401A43026210BD082908B540
:1088200018D005D859B1042911D090F8433008E088
:108830000C2912D01029F8D190F8423001E090F8BC
:108840003E30013B18BF012353B101203EE090F8B8
:108850003F30F6E790F84030F3E790F84130F0E72A
:1088600008294FF0020335D006D861B104292ED073
:10887000022380F8433008E00C292ED01029F7D1CC
:1088800080F8423001E080F83E3000680122FFF7B6
:10889000B7FF174A904206D0164B984203D003F513
:1088A0008063984220D1436C904243F40043436478
:1088B00016D18268104B1340062B06D0B3F5803FCB
:1088C00003D0036843F001030360002008BD80F873
:1088D0003F30DAE780F84030D7E780F84130D4E71E
:1088E000044B9842EDD1E4E7B0F1804FFAE700BFC6
:1088F000002C01400040014007000100FFF78EBF3F
:10890000082908B5034629D005D859B104291FD034
:1089100093F843002AE00C2926D01029F8D190F8CA
:10892000420023E090F83E0093F84420C0B20128B2
:10893000D2B256D1012A43D108294FF0020245D0C4
:1089400018D8F1B104293CD0022283F8432044E036
:1089500090F83F0093F84520C0B2E8E790F8400057
:1089600093F84620C0B2E2E790F8410093F8472020
:10897000C0B2DCE70C292ED01029E5D183F84220C3
:108980002BE083F83E2083F8442018680122FFF78B
:1089900037FF154B984206D0B0F1804F03D003F556
:1089A000A053984207D18268104B1340062B06D083
:1089B000B3F5803F03D0036843F001030360002058
:1089C00008BD83F83F2083F84520DEE783F8402088
:1089D00083F84620D9E783F84120022283F8472014
:1089E000D3E70120ECE700BF002C014007000100A5
:1089F000036A01F00F0110B504248C4023EA04033C
:108A00000362036A8A401A43026210BD08B529B99D
:108A100090F84430012B1DD001203DE0042907D1FE
:108A200090F84530012BF7D1022380F8453014E04F
:108A3000082907D190F84630012BEDD1022380F8A8
:108A400046300AE090F84730012BE5D1022380F848
:108A5000473002E0022380F8443000680422FFF728
:108A6000C7FF436C43F4004343640C4B984206D069
:108A7000B0F1804F03D003F5A053984207D182682C
:108A8000074B1340062B06D0B3F5803F03D0036895
:108A900043F001030360002008BD00BF002C01402B
:108AA00007000100FFF7B2BF7047704770470268C8
:108AB00052E8003F23F4907342E800310268002935
:108AC000F5D102F1080353E8003F23F0010302F15E
:108AD000080C4CE800310029F3D1036E012B07D1BB
:108AE00052E8003F23F0100342E800310029F7D19B
:108AF0002023C0F880300023036683667047026835
:108B000052E8003F23F0800342E800310268002968
:108B1000F5D152E8003F43F0400342E8003100291C
:108B2000F7D17047C26F212A034611D1B0F8522005
:108B300092B20AB9FFF7E3BFC26C016812F8010BE9
:108B40000885DA64B3F85220013A92B2A3F85220B1
:108B50007047C26F212A034613D1B0F8522092B257
:108B60000AB9FFF7CCBFDA6C006832F8021BC1F318
:108B700008010185DA64B3F85220013A92B2A3F8F1
:108B800052207047704700000346C06F202822D152
:108B900019B312B3A3F85220A3F850200022C3F84F
:108BA00084202122DA679A68D964B2F5805F10D1F7
:108BB00018690B4A0B49002818BF0A46DA6619687B
:108BC00051E8002F42F0800241E800200028F6D151
:108BD0007047044AF2E7022070470120704700BF47
:108BE000538B0008258B000808B5806A0023A0F885
:108BF0005A30A0F8523002F0BFF908BD70470000AB
:108C00000368DA69196870B540F60F0632429D684C
:108C100004460BD1960640F188808E0640F185808F
:108C2000836E002B7BD0BDE8704018479C4E05F04A
:108C300001000E40064378D0D50709D5CE0507D5EB
:108C400001251D62D4F8845045F00105C4F8845014
:108C5000950708D538B102251D62D4F8845045F037
:108C60000405C4F88450560708D538B104251D62A0
:108C7000D4F8845045F00205C4F8845015070BD58C
:108C800001F02005054307D008201862D4F88400BD
:108C900040F00800C4F8840016050AD54D0108D537
:108CA0004FF400601862D4F8843043F02003C4F815
:108CB0008430D4F88430002B31D0900605D58A0654
:108CC00003D5A36E0BB1204698472668D4F88420BC
:108CD000B36802F0280203F0400353EA020520467D
:108CE0001ED0FFF7E4FEB3685B0615D5226802F1DB
:108CF000080353E8003F23F04003083242E8003104
:108D00000029F3D1606F38B1664B8363FEF716FB21
:108D100028B1606F836B86E7204602F02DF970BDA5
:108D200002F02AF9C4F88450F9E7206E012840F0D7
:108D30008B80D60640F18880C80640F185801022DD
:108D40001A629968B4F8582049064FD5616F0868CF
:108D5000416889B2002941D091423FD2A4F85A100B
:108D6000026892062ED453E8002F22F4807243E862
:108D700000210029F7D103F1080252E8002F22F068
:108D8000010203F1080040E800210029F3D103F1BA
:108D9000080252E8002F22F0400203F1080040E8E8
:108DA00000210029F3D12022C4F88020216653E855
:108DB000002F22F0100243E800210029F7D1606F54
:108DC000FEF79BFA02236366B4F85A30B4F85810E1
:108DD000C91A89B22046FFF711FFA0E791429ED140
:108DE00003689B069BD502236366F3E7B4F85A1029
:108DF000B4F85A0080B289B2002890D0511A89B2D2
:108E000000298CD053E8002F22F4907243E8002010
:108E10000028F7D103F1080252E8002F22F00102E6
:108E200003F1080545E800200028F3D12022C4F80A
:108E30008020A066206653E8002F22F0100243E84D
:108E400000200028F7D1CEE7D60209D5680207D561
:108E50004FF4801220461A62BDE8704002F0E4B878
:108E6000160607D50D0605D5E36E002B3FF457AF68
:108E70002046D8E650067FF552AF4A067FF54FAF41
:108E800053E8002F22F0400243E800210029F7D1E7
:108E90002023E367E166204602F06AF83FE700BF5F
:108EA00020010004E98B0008D0F880100268222914
:108EB00008B5B0F85C3055D1918C426D0B40137001
:108EC000436D01334365B0F85A30013B9BB2A0F8C3
:108ED0005A30B0F85A309BB2002B42D1026852E8A7
:108EE000003F23F4907342E8003103680029F5D174
:108EF00003F1080252E8002F22F0010203F1080CEE
:108F00004CE800210029F3D12022C0F88020184A23
:108F100081669342416605D1026E012A0ED002F0AD
:108F200023F81EE05A681102F6D553E8002F22F00C
:108F3000806243E800210029F7D1EDE700220266B4
:108F400053E8002F22F0100243E800210029F7D156
:108F5000DA69B0F85810D20644BF10221A62FFF73F
:108F60004DFE08BD138B9BB243F008031383F8E753
:108F700000800040D0F88020B0F85C10222A08B5AC
:108F8000036852D19A8C1140426D22F8021B42654F
:108F9000B0F85A20013A92B2A0F85A20B0F85A20FC
:108FA00092B2002A40D153E8002F22F4907243E895
:108FB00000210029F7D103F1080252E8002F22F026
:108FC000010203F1080C4CE800210029F3D1202212
:108FD000C0F88020184A81669342416605D1026E2E
:108FE000012A0ED001F0C0FF1EE05A681102F6D52A
:108FF00053E8002F22F0806243E800210029F7D1D6
:10900000EDE70022026653E8002F22F0100243E849
:1090100000210029F7D1DA69B0F85810D20644BF10
:1090200010221A62FFF7EAFD08BD1A8B92B242F0D5
:1090300008021A83F8E700BF0080004010B590F8DE
:109040007830012B1CD0012380F878302423C367AB
:10905000026852E8003F23F00C0342E80034016844
:10906000002CF5D151E8002F42F0080241E800231E
:10907000002BF7D12022C26780F87830184610BD47
:109080000220FCE710B590F87830012B1CD00123AA
:1090900080F878302423C367026852E8003F23F049
:1090A0000C0342E800340168002CF5D151E8002F90
:1090B00042F0040241E80023002BF7D12022C267CE
:1090C00080F87830184610BD0220FCE7C26FD0F857
:1090D000800010437047000038B50446C06921691C
:1090E000A26823680A4361691D680A43654902430F
:1090F00029400A431A605A68E16822F440520A4340
:109100005A60614AA16993421CBF226A11439A685E
:1091100022F430620A439A605C4A934213D15C4B5A
:10912000D3F8883003F00303022B00F0A580032B53
:1091300000F09C80012B00F09380B0F5004F61D0CF
:10914000FEF7FAFE79E0534A934214D1504BD3F81C
:10915000883003F00C03082B00F08E8007D8002B1A
:109160007ED1B0F5004F66D1FEF7D4FE4CE00C2B5B
:109170007CD0012026E0484A934209D1444BD3F8E1
:10918000883003F03003202B76D0E8D9302BEFE77E
:109190003D4A9342EDD13E4BD3F8883003F440630F
:1091A000B3F5006F12D003D843B9FEF7B3FE07E062
:1091B000B3F5406FDDD14FF4004008E0FEF7E2FA6E
:1091C00028B900200023C4E91A3338BD3348626847
:1091D00002EB42038342CCD8B0EB023FC9D851081E
:1091E00000238C464FF480751946E0FB05C16046AC
:1091F000F7F73AFD2A4BA0F540729A42B9D8236896
:10920000D860DEE7FEF798FE0028DAD062685308DF
:1092100003EB4003B3FBF2F34FF6EF72A3F110013F
:109220009142A6D823F00F02216892B2C3F3420301
:109230001343CB60C5E7FEF76DFE0028C1D062681E
:1092400000EB5203B3FBF2F34FF6EF72A3F1100100
:1092500091428ED82268D360B3E7FEF793FAECE729
:10926000B0F5004FF9D1FEF78DFACDE7B0F5004F1C
:10927000CCD04FF40040E2E7B0F5004F0748DED114
:10928000C4E700BFF369FFEF0080004000380140F1
:109290000010024000440040004800400024F40058
:1092A000FFFC0F00436A1A0710B506D50168446B2E
:1092B0004A6822F4004222434A60DC0706D501686E
:1092C000846A4A6822F4003222434A60990706D52C
:1092D0000168C46A4A6822F4803222434A605A070D
:1092E00006D50168046B4A6822F4802222434A6052
:1092F000DC0606D50168846B8A6822F4805222431A
:109300008A60990606D50168C46B8A6822F4005207
:1093100022438A605A060FD50168046C4A6822F419
:1093200080122243B4F5801F4A6005D14A68446C1C
:1093300022F4C00222434A601B0606D50268816CF3
:10934000536823F400230B43536010BD2DE9F84309
:10935000DDF8209004460D46174698462268D369EA
:1093600035EA03030CBF01230023BB4201D00020D8
:1093700022E0B9F1FF3FF2D0FDF728F9A0EB080099
:10938000484529D8B9F1000F26D021680B685A0743
:10939000E4D5802DE2D0402DE0D0CE6916F008064D
:1093A0000CD0082520460D62FFF781FB0023C4F88E
:1093B000845084F878300120BDE8F883CB691B0520
:1093C000CCD54FF400630B622046FFF770FB2023DF
:1093D000C4F8843084F878600320EDE773B5044660
:1093E0000026C0F88460FDF7F1F823681B681A07AF
:1093F00005461BD56FF07E430093324603464FF47B
:1094000000112046FFF7A2FF80B1226852E8003F1A
:1094100023F0800342E800310029F6D12023E367DE
:109420000320002384F8783002B070BD23681B68E5
:109430005B0724D56FF07E43009300222B464FF448
:1094400080012046FFF782FFC8B1226852E8003F42
:1094500023F4907342E8003122680029F5D102F12B
:10946000080353E8003F23F0010302F1080040E83D
:1094700000310029F3D12023C4F88030D0E7202325
:109480000020E367C4F8803020666066C9E710B545
:10949000044640B3C36F1BB980F87830FFF772FB06
:1094A00022682423E367136823F001031360636ACF
:1094B00013B12046FFF7F6FE2046FFF70DFE012808
:1094C00011D023685A6822F490425A609A6822F0B8
:1094D0002A029A601A6842F0010220461A60BDE82A
:1094E0001040FFF77BBF012010BD10B5044660B3EC
:1094F000C36F1BB980F87830FFF744FB2268242340
:10950000E367136823F001031360636A13B1204615
:10951000FFF7C8FE2046FFF7DFFD012815D02368BE
:109520005A6822F490425A609A6822F022029A60A5
:109530009A6842F008029A601A6842F001022046D6
:109540001A60BDE81040FFF749BF012010BD0000C0
:1095500010B5A0F85820A0F85A2082684165002371
:10956000B2F5805F836630D10369002B40F2FF13B0
:1095700018BFFF23A0F85C300023C0F884302223FA
:10958000C0F88030026802F1080353E8003F43F05E
:109590000103083242E8003102680029F2D18368F1
:1095A0000169B3F5805F20D1154B164C002918BF17
:1095B00023468366D9B152E8003F43F4907342E8F2
:1095C00000310029F7D1002010BD2AB90369002B12
:1095D0000CBFFF237F23CDE7B2F1805FCAD10369BF
:1095E000002B0CBF7F233F23C4E7064BE1E752E883
:1095F000003F43F0200342E800310029F7D1E2E7C1
:10960000758F0008A98E0008D0F88030202B30B468
:1096100015D1B9B1B2B10023046803660A4B9C426C
:109620000AD063681B0207D554E8003F43F080630B
:1096300044E80035002DF7D130BCFFF789BF022088
:1096400030BC70470120FBE70080004090F8783084
:10965000012B12D0012380F87830016801F1080352
:1096600053E8002F42F40002194641E80023002B82
:10967000F3D180F87830184670470220704790F890
:109680007830012B12D0012380F87830016801F185
:10969000080353E8002F22F40002194641E8002392
:1096A000002BF3D180F878301846704702207047BD
:1096B00090F87830012B0FD0012380F878300168C2
:1096C00051E8002F42F0020241E80023002BF6D1BE
:1096D00080F87830184670470220704790F878304C
:1096E000012B0FD0012380F87830016851E8002F5A
:1096F00022F0020241E80023002BF6D180F87830F6
:109700001846704702207047836810B504462BB195
:109710000322014698470023C4E9023310BD836841
:1097200010B5044613B1032201469847204610BDE8
:109730004B1E032B00D9FEE78900081F704700006D
:109740000139435C13F0100004D0022916D80C4AEA
:1097500032F81100DB0712D503290FD8DFE801F03A
:109760000205080B40F00100704740F01000704700
:1097700040F48070704740F480507047FEE77047B7
:1097800040E100080139032900D9FEE7014B585C8C
:10979000704700BF3CE100080139032900D9FEE70A
:1097A000014B585C704700BF38E100082DE9F041DB
:1097B00004460E46FFF7BCFF04EB061808F16408E8
:1097C000054631462046FFF7DDFFD8F808302BB1BB
:1097D0002369C2431A61DA680243DA60771E04EB38
:1097E00047039B880B2B49D8DFE803F05118181862
:1097F000060618184A4A4A2AE35DDE0604D52946B9
:1098000004F11000FFF74EF9E35DD80736D529467D
:1098100004F11000BDE8F041FFF770B8E35DD90630
:1098200004D5294604F11000FFF7F0F8E35DDA07EC
:1098300024D5294604F11000BDE8F041FEF7EEBF43
:10984000294604F11000FFF75BF831462046FFF788
:10985000A3FF2569014606462046FFF771FF2B6AE4
:109860001843D8F80830286243B131462046FFF744
:1098700089FFC3432B61EB681843E860BDE8F081C2
:10988000294604F11000BDE8F041FFF739B823691B
:109890001B68DB07F2D404F11000BDE8F041FEF7CD
:1098A000D3BC70B501250446861C294636F8023F14
:1098B00023B129462046FFF779FF00210135052D08
:1098C000F4D1E36E3BB123696FF001021A61DA68EB
:1098D00042F00102DA6049B123691B68DB0705D455
:1098E00004F11000BDE87040FEF7AEBC70BD000092
:1098F0002DE9F0438DB004461F460E46FFF718FFD2
:109900004FF6FF730828059390462369054627D034
:1099100004D848B1042821D0DB6D06E00C2821D002
:109920001028F9D19B6D00E05B6B069300210123A9
:10993000CDE902319DF850300791CDE90911089128
:109940000B9101910493B8F10B0F1AD8DFE808F0DE
:109950000C123B3E40494B4D514F585A9B6BE4E72C
:10996000DB6BE2E71B6CE0E705912A4605A904F1F1
:10997000100004E0102305932A4605A9E018FEF71D
:10998000E1FD013E04EB4603A3F80480B8F1000FAB
:1099900016D07B1C14D0384601F0A8F8A8425BD141
:1099A0002E49384600F010FF2C49384600F046FF9B
:1099B000A35D10F4801F0CBF012210221343A35596
:1099C0000DB0BDE8F08320230593CEE73023FBE7FD
:1099D00060232A4605A904F110000593FEF7E4FD73
:1099E000CFE77023F5E75023EEE74023ECE70223AF
:1099F00001932A4601A904F11000FEF775FEC0E7A5
:109A00000A23F5E71549384600F018FF10F48010D6
:109A100000D0FEE704F11009012301902A4601A9B4
:109A200048460293FEF760FE31462046FFF7B4FE3B
:109A3000431E0146E25C42F00102E25404EB4303A0
:109A40000B229A8020460223CDE90133FFF770FEF6
:109A500001A902464846D0E7FEE700BF04E500083A
:109A6000013903299ABF00EB41008088002070472C
:109A700001211030FEF70EBC0369186800F00100E8
:109A8000704710B502460C46FFF7F6FF80B9CB6869
:109A9000DB070ED5CB6823F00103CB601046FFF740
:109AA000E7FF6FF001032361E36843F00103E36024
:109AB00010BDBDE810401046FFF7DABF0E4B9842CC
:109AC0000FD0B0F1804F0ED0A3F58E3398420CD05A
:109AD00003F5983398420AD003F58063984208D082
:109AE000FEE70020704701207047022070470320E6
:109AF00070470420704700BF002C0140024670B53B
:109B0000044652F8100FFFF7D9FF0546104600F043
:109B100023FF094A002342F8253004F16406E3607C
:109B200004F1B405B54204D0103D2846FFF7F7FD17
:109B3000F8E7204670BD00BF6C150020F8B504465C
:109B40000846FFF7BBFF236903B1FEE71B4D84F80E
:109B50002C3004F10C0245F8202004F110060E22EE
:109B6000C4E90C33C4E90E33C4E91033C4E9172344
:109B70002161A36484F84C3084F84D30E4603046B1
:109B800000F096FE04F1640504F1B4072846103590
:109B9000FFF7BAFDBD42F9D10023C4E900334FF607
:109BA000FF72C4E90632C4E90833A360636180230D
:109BB000A3623046BDE8F840FEF75CBC6C1500209F
:109BC00010B586B014220446002101A802F040FD21
:109BD0000023694601A80093FEF7C0F9206900F050
:109BE00067FF012802D002280FD0FEE7049CFEF791
:109BF00091F9B4F5C06F05D00BD824F48074B4F596
:109C0000806F00D1400006B010BD059CFEF794F9AE
:109C1000EFE7B4F5E06FF4E7012A38B505460C46E6
:109C20000BD0022A16D004B1013C29692846CC6227
:109C3000EC61BDE83840FFF724BFFFF7C1FF084BD8
:109C4000B0FBF3F044432A69230C93620133B4FB65
:109C5000F3F4E8E7FFF7B4FFB0FBF4F4F3E700BF79
:109C600040420F00F8B5054614461A46FFF760FD5E
:109C70002B699F6A822A064607F101072AD020D85D
:109C8000102A12D85ABB2969CB6A4FF6FF72934249
:109C900003D1B4F5803F08BF1C46082E34D025D828
:109CA00056B3042E2ED0CC6527E0812AEBD128466E
:109CB000FFF786FF164BB0FBF3F06043B0FBF7F401
:109CC000E1E7832ADFD1DB6A03FB04436424B3FBAF
:109CD000F4F4D8E72846FFF773FF6743EEE7DB6A43
:109CE00003FB044301249440013CF0E70C2E0DD00B
:109CF000102ED8D18C6500E04C632846BDE8F840B2
:109D0000FFF7BFBE8C63F8E7CC63F6E70C64F4E7BB
:109D100040420F0010B5074C206810B10430FEF728
:109D2000CDFA206920B1BDE810400430FEF7C6BA74
:109D300010BD00BF6C150020034B186810B1043033
:109D4000FEF7BCBA704700BF6C150020034B586883
:109D500010B10430FEF7B2BA704700BF6C15002096
:109D6000034B986810B10430FEF7A8BA704700BFE3
:109D70006C150020034BD86810B10430FEF79EBA72
:109D8000704700BF6C1500200022C0E90022C0E926
:109D900002227047F8B504460E4600F1640500F152
:109DA000B40728461035FFF7EFFFBD42F9D1002375
:109DB000204623613146FFF7C1FE2046F8BD826888
:109DC00010B50AB903F0B6FCBDE81040C3681847E7
:109DD00008B500B9FEE700F069FD0068C36E13B175
:109DE0006430FFF7ECFF08BDFFF7F2BF10B500B914
:109DF000FEE7037F013B072B10D8DFE803F00414D4
:109E00000F100F0F0F12012400F050FD2401006805
:109E10006434204483680BB1FFF7D1FF10BD0324E5
:109E2000F2E70424F0E70224EEE7FFF7DFBFFFF7D5
:109E3000DDBF02F027BA02F02DBA000086B0042878
:109E400042D8DFE800F003111D2935001F4BDA6C02
:109E500042F00102DA64DB6C03F001030193019B21
:109E60004FF0904006B07047184B1948DA6C42F03A
:109E70000202DA64DB6C03F002030293029BF1E757
:109E8000124B1448DA6C42F00402DA64DB6C03F023
:109E900004030393039BE5E70C4B0F48DA6C42F095
:109EA0000802DA64DB6C03F008030493049BD9E72F
:109EB000064B0A48DA6C42F08002DA64DB6C03F08D
:109EC00080030593059BCDE70020CBE700100240FF
:109ED0000004004800080048000C0048001C00482E
:109EE00008B5064900F0AAFCC0F3C430122800D916
:109EF000FEE7034B53F8200008BD00BF60E60008F2
:109F000054E10008A0F580500138022800D9FEE78E
:109F1000014B53F82000704748E100080A4BDA6C07
:109F200042F40052DA64DB6C82B003F40053019314
:109F3000019B064B1868C30403D4054902B000F026
:109F400043BC02B0704700BF00100240AC020020CA
:109F500060E600080A4BDA6A42F40052DA62DA6A12
:109F600022F40052DA62DA6A42F40052DA62DA6A01
:109F700022F40052DA62DA6C22F40052DA6470479A
:109F800000100240F0B5A3B0054664220E4609A8B1
:109F9000002102F05DFB1822002103A802F058FB0B
:109FA0000023EA04ADF80630029340F1C18041F28B
:109FB00003039D4200F2BC80844B09932846FFF7BF
:109FC000A1FF07270446082E00F0C3800A2E00F0E8
:109FD000C280062E0CBF182300234FF44032CDE977
:109FE0000A2300230422CDE90C33CDE912330E926B
:109FF000ADF83C3001228DF8443014938DF8543084
:10A000008DF85C301E931C938DF87430704B109259
:10A0100009A84FF4805216921D60FCF7F5FA00284B
:10A0200040F09280099B694A0394934240F09580E6
:10A03000684B9C4242D0684B9C423FD0674B9C424D
:10A040003CD0674B9C4239D003F1866310339C426D
:10A0500034D0644B9C4231D003F1866340339C4240
:10A060002CD0614B9C4229D003F1866303F58073A9
:10A070009C4223D05D4B9C4220D003F1042303F586
:10A0800040139C421AD003F1866303F500639C429F
:10A0900014D0574B9C4211D0564B9C420ED0564B7D
:10A0A0009C420BD0554B9C4208D0554B9C4205D04E
:10A0B000544B9C4202D0544B9C4245D10623CDE9DF
:10A0C00004377F240423CDE9064303A9002309A80C
:10A0D0000893FCF7E3FB002836D1214609A8FCF7DA
:10A0E000D6FF002830D109A8FCF758FE60BB0A2132
:10A0F00009A8FCF75DFB38BB09A8FCF78DFD8305BB
:10A1000005D509A8FCF7C6FB80B2ADF8060009A882
:10A11000FCF79EFFC0B909A8FCF7E8FEA0B93B4ACE
:10A12000936823F0E0739360BDF8060080B20CE002
:10A130003749284600F060FB02A909902846FFF73E
:10A14000CFFE099B044613B9002023B0F0BD0227BF
:10A1500039E7102341E708233FE72E4A9342F3D122
:10A160001C4B9C42AAD01C4B9C42A7D01B4B9C4230
:10A17000A4D01B4B9C42A1D003F1496370339C4295
:10A180009CD0194B9C4299D003F1866303F58073F0
:10A190009C4293D0154B9C4290D003F1042303F5CD
:10A1A00040139C428AD003F1866303F500639C420E
:10A1B00084D00F4B9C4281D00E4B9C423FF47EAF2B
:10A1C0000D4B9C423FF47AAF0C4B75E700000450F6
:10A1D000AC02002002003004040060080800900C6B
:10A1E0001000C01040002019000180210004002A46
:10A1F000002090360040C03A0080F03E000021432D
:10A2000001000080000052C7000084CB000304500E
:10A2100060E60008000104502DE9F3478A4625490D
:10A22000254F99469046064600F0E6FAFFF746FCB1
:10A2300057F82030044673B9B420FFF7FAFD1D49E2
:10A240000546304600F0D8FA01462846FFF7A2FD41
:10A2500057F824301D6057F8243016491C683046E2
:10A2600000F0ECFAC0F3C43529462046FFF7F8FBAE
:10A270000428074607D000230093042233462946CA
:10A280002046FFF735FB022251462046FFF7C4FC6B
:10A290004B46424629462046FFF7E4FC042F05D0F2
:10A2A000204602B0BDE8F047FFF7FBBA02B0BDE8B8
:10A2B000F08700BF04E500086C150020F8B51449CC
:10A2C000144E074600F098FAFFF7F8FB56F82030D6
:10A2D000044673B9B420FFF7ACFD0D490546384676
:10A2E00000F08AFA01462846FFF754FD56F824305C
:10A2F0001D6056F824301C6844B12046FFF7FEFB71
:10A300002046B421BDE8F840FFF795BDF8BD00BF79
:10A3100004E500086C15002037B5FCF757F94FF03D
:10A32000E0250446AB690093FCF750F9AB69019353
:10A330006969844201F101014FF47A7308D0019AEE
:10A340008A1A5A43B2FBF1F203FB002003B030BD7E
:10A35000009A8A1A5A43B2FBF1F203FB0420F5E794
:10A36000FCF734B9704708B5FCF724F9FCF75FFF38
:10A37000FFF7F8FF08BD000010B592B0442200219D
:10A38000044601A802F064F9FDF774F92C4B9A6DAC
:10A3900042F480629A659A6D02F480620092009A9B
:10A3A000032C11D8DFE804F00219283DD3F89420DB
:10A3B00042F00102C3F89420D3F894309C0703D4F0
:10A3C0000823019301230693019B002B36D001A89B
:10A3D000FDF722FA002831D0FEE71A6842F48072B5
:10A3E0001A601B685905EFD4022301934FF4807261
:10A3F0004023CDE90423E7E7D3F8902042F001029F
:10A40000C3F89020D3F890209407DDD4D3F890209F
:10A4100022F01802C3F89020042301930123039330
:10A42000D2E71A6842F480321A601B6899035EBF53
:10A4300001224FF48033CDE90123C5E712B010BDEE
:10A4400000100240704700000F4B9A6D42F080529E
:10A450009A659A6D84B002F080520192019A1A6E48
:10A4600042F001021A661A6E02F001020292029A8A
:10A470009A6C42F480529A649B6C03F48053039369
:10A48000039B04B0704700BF001002400C4BD3F890
:10A49000FC20D2015EBFD3F8FC2042F08072C3F8EA
:10A4A000FC20084B00225A601A6842F001021A6030
:10A4B00000BF00BF00BF5868B0FA80F04009704785
:10A4C00000ED00E0001000E008B5FFF7BDFFFFF76A
:10A4D000DDFFFCF75FF8FFF7B5FF00F0D5FDBDE845
:10A4E00008400148FCF7A8BEB00200200023C0E9E4
:10A4F0000033C0E9023370470023012803F1010251
:10A500000AD11422DBB25343054A181D1044816856
:10A5100029B11A441369184740081346EDE77047FC
:10A52000801500200120FDF799B80220FDF796B8AC
:10A530000420FDF793B80820FDF790B81020FDF730
:10A540008DB838B505242025A8B2FDF787F8013C61
:10A550004FEA4505F8D138BD38B506244FF480657B
:10A56000A8B2FDF77BF8013C4FEA4505F8D138BDAC
:10A57000344A104608B5062300F8043BFFF7B6FF3F
:10A58000072302F118001375FFF7B0FF082302F14B
:10A590002C0082F82830FFF7A9FF092302F14000C0
:10A5A00082F83C30FFF7A2FF0A2302F1540082F840
:10A5B00050301721FFF79AFF02F1680082F864100B
:10A5C000FFF794FF02F17C0082F87810FFF78EFF0E
:10A5D00002F1900082F88C10FFF788FF02F1A400CE
:10A5E00082F8A010FFF782FF02F1B80082F8B410E1
:10A5F0002821FFF77BFF02F1CC0082F8C810FFF79B
:10A6000075FF02F1E00082F8DC10FFF76FFF02F146
:10A61000F40082F8F010FFF769FF02F5847082F809
:10A620000411FFF763FF02F58E7082F81811FFF72F
:10A630005DFFBDE8084002F5987082F82C11FFF725
:10A6400055BF00BF8015002038B5054CA4F5A07596
:10A65000143C201DFFF763F8AC42F9D138BD00BFB0
:10A66000C016002030B591FAA1F391FAA1F1B3FA26
:10A6700083F3C4685B000325B1FA81F105FA03F3A3
:10A68000490024EA03038A401A43C26030BD431CD8
:10A6900004D00C3151F80C3C5A1C01D100207047F9
:10A6A000834201F10C01F5D101207047F8B5471C38
:10A6B00006460D4600D1FEE700F00F02414BC0F305
:10A6C000031053F82240FFF7B9FB94FAA4F3B3FA4E
:10A6D00083F3876803225B0002FA03F394FAA4F27F
:10A6E000B2FA82F227EA03075200032393403B4366
:10A6F00005F007018360032903D8DFE801F05F61FB
:10A700002C03FEE7032394FAA4F2B2FA82F206685D
:10A710005200032707FA02F226EA020694FAA4F28C
:10A72000B2FA82F2520093400139334301290360A7
:10A7300005D843682A074CBF2343A3434360C5F3AE
:10A740000112012A02D0022A18BF00222146BDE8C8
:10A75000F840FFF787BFC5F306227F2A01D1022305
:10A76000D1E7360716D5230A93FAA3F6B6FA86F68A
:10A77000476A93FAA3F3B6004FF00F0CB3FA83F3D2
:10A780000CFA06F69B0027EA060602FA03F33343A7
:10A790004362E4E794FAA4F3B3FA83F3066A9B00F6
:10A7A0000F2707FA03F326EA030694FAA4F3B3FA91
:10A7B00083F39B009A4032430262D0E70023A2E772
:10A7C0000123A0E7A0E10008431C06D170478342A3
:10A7D00002D18968FFF76ABF0C310B685A1CF6D1A9
:10A7E000FEE70B685A1C01D100207047834201D15B
:10A7F000486870470C31F4E7431C01D0FFF7F1BF04
:10A80000002070474B6813B94FF0FF307047834208
:10A8100001D1086870470C31F4E708B1FFF7F2BFC7
:10A820004FF0FF30704703460868421C00D1704764
:10A83000984201D1886870470C31F5E7431C01D07C
:10A84000FFF7F1BF704703468B42084604D01BB1A7
:10A8500000290CBF1846002070470000114B4FF034
:10A8600000629A60D3F8882042F47002C3F888200E
:10A870000D4B1A68002142F001021A6099601A68B3
:10A8800022F0A85222F410221A604FF48052DA60AB
:10A890001A6822F480221A6040F23F7299611A62AB
:10A8A000704700BF00ED00E0001002400438704720
:10A8B0000368244A934286B00BD1234B1A6E42F4AC
:10A8C00000621A661B6E03F400630193019B06B0DD
:10A8D0007047B3F1804F0BD103F504339A6D42F00A
:10A8E00001029A659B6D03F001030293029BEEE760
:10A8F000164A93420AD1144B9A6D42F010029A659F
:10A900009B6D03F010030393039BE0E7104A93420F
:10A910000AD10D4B1A6E42F480321A661B6E03F494
:10A9200080330493049BD2E70A4A9342CFD1064B6B
:10A930001A6E42F400321A661B6E03F4003305935C
:10A94000059BC4E7002C01400010024000100040AD
:10A9500000400140004401400368174A934206D179
:10A9600002F56442136E23F4006313667047B3F17B
:10A97000804F05D1114A936D23F001039365704711
:10A980000F4A934205D102F50032936D23F0100374
:10A99000F4E70C4A934205D102F55042136E23F4BA
:10A9A0008033E2E7084A9342E0D102F54C42136E4D
:10A9B00023F40033D9E700BF002C0140001002400F
:10A9C000001000400040014000440140431C14D0EE
:10A9D0000E4B98420FD007D8B0F1804F10D0A3F59E
:10A9E0008E3398420ED0FEE7094B98420CD003F507
:10A9F00080639842F7D1192070476FF00D007047BF
:10AA00001C2070473620704718207047002C0140EA
:10AA100000400140431C14D00F4B984214D007D87B
:10AA2000B0F1804F12D0A3F58E33984210D0FEE7DC
:10AA30000A4B98420ED003F580639842F7D1192053
:10AA400070476FF00D0070471B2070471C20704747
:10AA50003620704718207047002C0140004001400C
:10AA600038B5FFF725FF04460068FFF7AFFFD4E9CC
:10AA70001312FCF767FB2068FFF7A8FFFCF794FBB5
:10AA800022681046FFF7C6FF05461046FFF79EFFF7
:10AA900085420BD02846D4E91312FCF753FB2068FB
:10AAA000FFF7B8FFBDE83840FCF77EBB38BD0000BB
:10AAB000431C12D00B4B984211D003D8B0F1804FF9
:10AAC0000DD0FEE7084B20F480629A4203D0A3F534
:10AAD000A0539842F5D10220704700207047012012
:10AAE000704700BF001000400040014008B5064913
:10AAF000FFF7A4FEC0F3C430431E032B00D9FEE7CA
:10AB00008000043808BD00BF04E500082DE9F04FBF
:10AB100087B004460F46D0F89400B2499846109B7F
:10AB200001939146FFF768FEAF498246D4F898003A
:10AB3000FFF762FEAD490646D4F89C00FFF75CFEC5
:10AB4000AB490546D4F8A000FFF756FE8346BAF19C
:10AB5000000F00F0A480D4F89820013202D0002E1B
:10AB600000F09D80D4F89C20013202D0002D00F02E
:10AB70009680D4F8A020013203D0BBF1000F00F082
:10AB80008E8031465046FFF75EFE29462060FFF773
:10AB90005AFE59462060FFF756FE206000287ED0FE
:10ABA000944B98427ED103F558431A6C42F480428C
:10ABB0001A641A6C22F480421A641A6E42F48042BB
:10ABC0001A661B6E03F480430293029B2523A4F8AC
:10ABD000A4308449D4F89400FFF7F6FD26B18249E9
:10ABE000D4F89800FFF7F0FD002D00F0A7807F4912
:10ABF000D4F89C00FFF7E8FD4FF4807ABBF1000F1A
:10AC000006D07B49D4F8A0004AF4007AFFF7DCFDB7
:10AC100094F8A510784A019B94F9A400C4F80C900C
:10AC2000251D42F821502268C4E901270C22C4E9FD
:10AC3000062A0022C4E90438C4E90922226201215B
:10AC4000FCF780FA22686D4B9A4240F0A380B7F57A
:10AC5000165F284674D8FEF7F9FC2846FEF728FD53
:10AC60002846002E72D1FEF740FCC0B1B7F5165F42
:10AC70006FD80220FFF780FB2268604B9A4201BF29
:10AC80005F4AD2F8883043F44063C2F888302846DF
:10AC9000002E40F08680FEF728FC002859D107B02E
:10ACA000BDE8F08F574B984215D103F5E6339A6B08
:10ACB00042F400329A639A6B22F400329A639A6DDE
:10ACC00042F400329A659B6D03F400330393039BB7
:10ACD0004FF493737BE74C4B984215D103F5E43363
:10ACE0009A6B42F480229A639A6B22F480229A63D0
:10ACF0009A6D42F480229A659B6D03F4802304933D
:10AD0000049B40F2272362E73C4B98427FF461AFFB
:10AD100003F5C833DA6B42F00102DA63DA6B22F032
:10AD20000102DA63DA6D42F00102DA65DB6D03F0ED
:10AD300001030593059B40F2463348E7AA465DE7C9
:10AD4000FEF79DFC2846FEF7C9FC89E7FEF79FFB4E
:10AD50008BE72B4F22683B685B0525D42268274B85
:10AD60009A4205D1D7F8883023F44063C7F8883079
:10AD7000284676BBFEF7B9FB002890D022681F4B0F
:10AD80009A4207D1D7F8883023F4406343F48063B4
:10AD9000C7F888302846FEB907B0BDE8F04FFEF787
:10ADA000A4BBFEF774FB78E7144B9A4201BFD7F8B7
:10ADB000883023F4406343F40063C7F888302846A2
:10ADC00026B9FEF792FB0028C8D168E7FEF75FFBC3
:10ADD000F9E7FEF75CFBCFE707B0BDE8F04FFEF701
:10ADE00056BB00BF8CE4000814E40008A8E3000888
:10ADF00048E3000800380140C016002000800040F1
:10AE000000100240004400400048004010B4019C83
:10AE100020B101945DF8044BFFF778BE5DF8044B58
:10AE20007047000008B5074B90F8A52053F82200A2
:10AE3000FEF74CF900F02200A0F1220358425841DD
:10AE400008BD00BFC016002008B5074B90F8A5202C
:10AE500053F82200FEF73AF900F02100A0F1210397
:10AE60005842584108BD00BFC016002070B50E46BC
:10AE7000054610B94FF0FF3070BDFFF7D3FF044611
:10AE80000028F7D12946012211F8A63F337095F822
:10AE9000A500034B53F82000FEF7B6FB2046EBE776
:10AEA000C016002038B50D460446C0B1FFF7BAFF02
:10AEB000A8B994F9A400C4F88C50FCF783F994F86D
:10AEC000A500074B04F1A60153F820000122FEF76C
:10AED0009BFB94F9A400BDE83840FCF765B938BD88
:10AEE000C016002038B515460446C8B1C0F8901009
:10AEF00090F9A400FCF766F9D4F8AC30B4F8B610B9
:10AF000094F8A50013FA81F1064BAAB253F8200079
:10AF1000FDF73AFE94F9A400BDE83840FCF744B9C7
:10AF200038BD00BFC016002050B1D0F898300133B2
:10AF300006D190F8A520034B53F82200FEF77EB807
:10AF4000704700BFC016002050B1D0F898300133D0
:10AF500006D190F8A520034B53F82200FEF792B8D3
:10AF6000704700BFC0160020D0F88830043818475A
:10AF7000D0F88C300438184710B5044650F804391E
:10AF8000DA69D1070CD501221A62FFF74BFFB0B97D
:10AF900004F1A20120460122BDE81040FEF734BBB7
:10AFA000DA69920701D50222EEE7DA69510701D585
:10AFB0000422E9E7DA691207E7D50822E4E710BDC1
:10AFC00008B52520FCF724F9024B1868BDE80840B5
:10AFD000FDF716BEC016002008B52620FCF718F9AC
:10AFE000034B586818B1BDE80840FDF709BE08BD1D
:10AFF000C016002008B52720FCF70AF9034B986813
:10B0000018B1BDE80840FDF7FBBD08BDC016002023
:10B0100008B54620FCF7FCF8024BD868BDE80840AC
:10B02000FDF7EEBDC0160020012200F1A201FEF7DF
:10B03000EBBA00000A490346086810B50344EFF371
:10B040000882934205D9074B0C221A604FF0FF305B
:10B0500010BD054A054C121B9342F4D20B60F7E772
:10B06000D80200208019002000A000200004000069
:10B07000FEE70000024B16221A604FF0FF307047C7
:10B08000801900200120704700B597B044220021AC
:10B0900005A801F0DDFA14220021684601F0D8FA73
:10B0A0004FF40070FCF7F6FA00B1FEE740224FF4CF
:10B0B00080710120CDE908120A220223CDE9120293
:10B0C00005A8CDE91033CDE914330593FCF7A4FBB3
:10B0D00000B1FEE7CDE902000F2203230490042112
:10B0E0006846CDE90023FCF76BFE00B1FEE717B020
:10B0F0005DF804FBB0F84831B0F84421981A00F02C
:10B100003F007047B0F84831B0F844219BB29342F9
:10B110001ABFD0F83C31985C4FF0FF30704790F880
:10B120004631B0F84A01C0B2834227BFC3F13F03A2
:10B13000C018C01A00F1FF30704707B503688DF8DA
:10B1400007105B6801220DF10701984703B05DF815
:10B1500004FB13B50DF107010446FFF787FE90B914
:10B16000B4F8B430B4F8B020013303F03F03934295
:10B1700009D0B4F8B420D4F8A8109DF8070092B212
:10B180008854A4F8B43002B010BD0000B0F8B62066
:10B19000D0F8B81011FA82F202F03F0210B5A0F810
:10B1A000B620B0F8B610B0F8B22089B28A421BD0EF
:10B1B000B0F8B640B0F8B610A4B24032121B5442F8
:10B1C00089B204F03F0402F03F02C1F1400158BFD0
:10B1D00062428A4228BF0A46C0F8B8200349FFF7F6
:10B1E00081FE4FF0FF3010BD0020FCE78DB100085C
:10B1F0002DE9F843036804469B688846164698473D
:10B2000001232374D4F82C31B4F8467101338146FC
:10B21000C7F1400709D194F8503133B1002384F8C5
:10B22000503104F19400FFF77FFE236820469B68AD
:10B2300098470028F9D03546AF4225D34D4523D84D
:10B24000B4F84631D4F840015A19402A184430D88D
:10B250002A46414601F094FA2F46B4F846311D447F
:10B2600005F03F05A4F8465104F194052846FFF780
:10B27000EBFD30B91649C4F84C713A462846FFF741
:10B2800031FE3046BDE8F8834F45236828BF4F465E
:10B290003A4641465B6820469847236820469B68AB
:10B2A0009847ED1BB844B4F846718146C7F1400792
:10B2B000C2E7C3F140073A46414601F061FAD4F8CB
:10B2C0004001EA1B08EB070101F05AFAC5E700BF8D
:10B2D0008DB10008C0F83031009BC0F83431914284
:10B2E00008BF4FF0FF3100F11103C0E94A21C0F857
:10B2F0003C3100F151020023A0F84831C0E950234D
:10B30000A0F84A317047000073B54FF47A750026F3
:10B31000C0E901653D4D0560CDB2312D069C25D8B3
:10B320003B4E56F8255001F4E0612943D5B2312D4A
:10B3300030D8374E56F8255002F4E0622A43DDB289
:10B34000312D3BD8324E56F8255003F4E0632B43A1
:10B35000E5B2312D46D82E4E56F8255004F4E0645F
:10B360002C430094FFF7B6FF02B070BD01F0C00699
:10B37000C02E0CD1CE2D0AD8264D01F03F0601F487
:10B38000E06155F82660224D55F82650CDE74FF084
:10B39000FF31CBE702F0C006C02E0CD1CE2D0AD86B
:10B3A0001C4D02F03F0602F4E06255F82660184D8D
:10B3B00055F82650C2E74FF0FF32C0E703F0C00651
:10B3C000C02E0CD1CE2D0AD8124D03F03F0603F447
:10B3D000E06355F826600E4D55F82650B7E74FF05C
:10B3E000FF33B5E704F0C006C02E0CD1CE2D0AD82D
:10B3F000084D04F03F0604F4E06455F82660044D5F
:10B4000055F82650ACE74FF0FF34AAE7DCE8000817
:10B41000F8E70008BCE70008037C70B504460D4659
:10B42000A3B1FBF7D3F80646B4F84621B4F84A3185
:10B430009BB29A420AD0002DF8D0FBF7C7F8801BC8
:10B440008542F1D8B4F84A31A4F8463170BD0021E4
:10B45000FFF7E2BFCBB2312B08D80E4A52F82330A7
:10B4600001F4E0611943C0F82C11704701F0C002EB
:10B47000C02A0CD1CE2B0AD8074B01F03F0201F4B1
:10B48000E06153F82220034B53F82230EAE74FF0F3
:10B49000FF31E8E7F8E70008BCE70008CBB2312B42
:10B4A00008D80E4A52F8233001F4E0611943C0F87D
:10B4B0002811704701F0C002C02A0CD1CE2B0AD847
:10B4C000074B01F03F0201F4E06153F82220034BE7
:10B4D00053F82230EAE74FF0FF31E8E7F8E70008D9
:10B4E000BCE7000873B54FF47A7316460022C0E932
:10B4F00001231D4B03604FF0FF33C0F82C311B4B71
:10B50000984204460D4615D1C321FFF7A3FFC2217F
:10B51000FFF7C4FF012E4FF0FF3308BFC4F82C31F2
:10B5200000932046D4E94A214FF0FF33FFF7D2FEC3
:10B5300002B070BD0E4B0F499A680F4B53F82200B2
:10B54000FFF75AF9854202D1C3212046DDE70B49B6
:10B550002846FFF762F90749C4F82C012846FFF78F
:10B560005CF9C4F82801D5E7DCE80008D016002013
:10B57000BCE700088CE40008F8E7000814E40008C1
:10B58000D0F82C31013310B504460ED10368DB68C6
:10B59000984794F8503143B9012384F8503104F1AD
:10B5A0009400BDE81040FFF7CFBC10BD02F00703C8
:10B5B000023BDBB2042B73B50546C0F8541180F88A
:10B5C00051219CBF1548C45C02F0300388BF0024A1
:10B5D000302B1BD101344FF4C063073C022C1CD824
:10B5E000C2F3C002520300920D4A05F1940652F8CC
:10B5F00024203046FFF70AFC2846FFF7C1FF09491F
:10B60000304602B0BDE87040FFF74CBC12F020039A
:10B610001CBF01344FF48063DFE7FEE7CCE800088D
:10B62000C0E8000853B1000810B50446FFF7A8FFB2
:10B63000B4F84821B4F8443192B29A421FBFD4F80A
:10B640003C21D05C013303F03F0314BFA4F8443124
:10B650004FF0FF3010BD0000024903480022FFF701
:10B6600041BF00BF00800040D016002070B50546E5
:10B670000C46084649B1F4F795FD2B680246214671
:10B6800028465B68BDE87040184770BD03688A684B
:10B690005B680968184708B5FFF7E8FF08BD03684D
:10B6A0001B68184708B50249FFF7E0FF08BD00BF57
:10B6B000DEE0000838B50546FFF7D8FF0446284607
:10B6C000FFF7F0FF204438BD38B50546FFF7DEFF31
:10B6D00004462846FFF7E6FF204438BDFFF7EABFDF
:10B6E00038B50546FFF7DBFF04462846FFF7DAFFCB
:10B6F000204438BD30B58BB00023012A0C468DF8AC
:10B70000243098BF0A2209A92546B4FBF2F404FBB1
:10B71000125303F0FF03092B94BF30333733DBB2EE
:10B72000AA4201F8013DEFD9FFF7A0FF0BB030BDF1
:10B730002DE9F04107460E4614462AB90368BDE8D4
:10B74000F0411B68C9B218470A2A05D1002905DB58
:10B75000BDE8F041FFF7CEBFD2B2F9E72D21FFF7E8
:10B760009EFF2246054671423846FFF7C3FF284434
:10B77000BDE8F08138B50546FFF7DAFF04462846F4
:10B78000FFF790FF204438BD10B42AB902685DF875
:10B79000044B1268C9B210475DF8044BD2B2FFF7F0
:10B7A000A9BF38B50546FFF7EFFF04462846FFF767
:10B7B00079FF204438BD38B50546FFF7E5FF04465C
:10B7C0002846FFF76FFF204438BD000070B5B4EE87
:10B7D000400AF1EE10FA2DED048B0646B0EE408AD9
:10B7E0000D4607D73449FFF741FF0446BDEC048BF3
:10B7F000204670BD9FED317AF0EEC07AF4EE477AC4
:10B80000F1EE10FA01DD2E49EDE7DFED2E7AB4EE10
:10B81000E70AF1EE10FA02DD2B493046E3E7DFEDEF
:10B820002B7AB4EEE70AF1EE10FAF5D4B5EEC00AC1
:10B83000F1EE10FA39D52D21FFF731FFB1EE488A2C
:10B8400004460023F6EE007AB2EE047ADAB29542AC
:10B850002DD838EE278A0A22FCEEC88A304618EE28
:10B86000901AFFF747FF0444002DBFD02E21304629
:10B87000FFF715FFF8EE688A044438EE688AB2EEE6
:10B88000049A002DB2D028EE098A0A22FCEEC88A5A
:10B89000304618EE901AFFF72DFFF8EE688A013D4A
:10B8A00038EE688A0444EDB2EBE70024C9E7C7EE3E
:10B8B000877A0133CAE700BFE1E00008FFFF7F7F1E
:10B8C000E5E00008FFFF7F4FE9E00008FFFF7FCFC2
:10B8D00008B5C9B2FFF77AFF08BD38B5C9B2054649
:10B8E000FFF774FF04462846FFF7DCFE204438BD0E
:10B8F00010B5044600F038FCE060236820465B6920
:10B900009847002808DA00F02FFCE368C01AA36803
:10B910009842F2D34FF0FF3010BDF8B507460D4600
:10B920008E180C46B44201D1601BF8BD3846FFF7B3
:10B93000DFFF031EF8DB04F8013BF3E72DE9F041DC
:10B940000746884616461D4673B100243846FFF761
:10B95000CFFF031E05DB434503D033550134A54219
:10B96000F4D12046BDE8F0811C46FAE710B5441A30
:10B970000298C01A4443521A94FBF2F4E01810BD26
:10B9800010B50446006800F085FC204610BD10B5D7
:10B990000446006808B100F07DFC0023C4E90133CF
:10B9A000236010BD38B504460D460068013100F033
:10B9B00027FD10B1C4E90005012038BD036810B5AA
:10B9C000044613B143688B4207D22046FFF7EAFFD3
:10B9D00020B1A3680BB922681370012010BD70B5A7
:10B9E0000E46114604461546FFF7E8FF20B92046EB
:10B9F000FFF7CDFF204670BD2068A560314600F0FE
:10BA0000B7FEF7E738B50023C0E90033044683608A
:10BA10000D4639B10846F4F7C5FB294602462046D3
:10BA2000FFF7DDFF204638BD38B5054600680C46F7
:10BA3000096830B119B16A68A3689A420BD200F064
:10BA400029FC23682B6063686B60A368AB600023EC
:10BA5000C4E9003303E000F08BFEA368AB60002371
:10BA6000A36038BD884210B50B46044604D009686F
:10BA700021B19A68FFF7B3FF204610BDFFF787FF9B
:10BA8000FAE710B500230446C0E900338360FFF7EE
:10BA9000E9FF204610BD884210B5044601D0FFF7EB
:10BAA000C3FF204610BD38B505460C4649B10846CF
:10BAB000F4F778FB214602462846FFF790FF284618
:10BAC00038BDFFF764FFFAE710B504468AB00023DB
:10BAD000C4E90033A360084601A900F075F901A983
:10BAE0002046FFF7E0FF20460AB010BD10B504461F
:10BAF0008AB00023C4E90033A360084601A900F01E
:10BB000093F901A92046FFF7CEFF20460AB010BDE9
:10BB100070B5044600238AB0C4E90033A36010EE78
:10BB2000100A0D468E1CF4F7FFFC76B241EC100BA8
:10BB300001AA2946304600F059F801462046FFF791
:10BB4000B2FF20460AB070BD70B5856804460E4647
:10BB500009B9002070BD62B115442946FFF72EFFD8
:10BB60000028F6D02068A3683146184400F000FE93
:10BB7000A5600120EEE707B500238DF8041001222F
:10BB800001A98DF80530FFF7DFFF03B05DF804FB76
:10BB900010B58A6809680446FFF7D6FF10B9204639
:10BBA000FFF7F5FE204610BD38B504460D4621B915
:10BBB0002046FFF7ECFE204638BD0846F4F7F2FABF
:10BBC000294602462046FFF7BFFF0028F0D0F2E7E3
:10BBD00083688B4201D9006818B9034800230370B9
:10BBE00070470844704700BF281800202DE9F04F27
:10BBF00059EC108BA7B005460F46144600230022CF
:10BC000040464946F4F75AFF064618B109F1004389
:10BC10009946012647494FF0000A0020574571DC3C
:10BC200002460B4640464946F4F720FB02460B46C7
:10BC3000CDE90223F4F7A8FF8246002F6BD0DFF88E
:10BC40000C914FF0000B4FF00008404649463A4B2C
:10BC50000022F4F7C1FC0BF1010B5F4580468946D9
:10BC6000F3DC5046F4F73EFC02460B46DDE90201E8
:10BC7000F4F7FAFA42464B46F4F7AEFCF4F75CFFF1
:10BC80003B4600905246002E43D02C49204600F0FF
:10BC9000A5FC8122002105A800F0DAFC002D204639
:10BCA000AEBF00266D420126F4F77CFAA84225D2E9
:10BCB0008022202105A800F0CBFC2046F4F772FA80
:10BCC0002D1A05F198030DEB0305002305F8843CBC
:10BCD00056BB2046F4F766FA013000F0D3FA21464D
:10BCE000054600F045FD05A9204600F041FD294626
:10BCF000204600F0D1FC284600F0CCFA204627B0C0
:10BD0000BDE8F08F0C4B0022F4F790FD0AF1010A18
:10BD100084E70B49BAE7024626B10A49204600F0FB
:10BD20005DFCB6E70849F9E705A9204600F0B4FC38
:10BD3000E4E700BF0000E03F00002440EDE0000821
:10BD4000EEE00008F8E00008F9E000080000F03F2D
:10BD5000F0B503468BB0084669B3911E222931D84D
:10BD60000A2A06D1002B04DA5B42012601AD2946DE
:10BD70000EE00026FAE7B3FBF2F402FB1437092FBA
:10BD80002346FCB294BF30345734E4B201F8014B7F
:10BD9000002BF0D1A942EED0034616B12D2203F8B4
:10BDA000012B5C1E0A46AA4207D84A1B8D4288BF57
:10BDB0000022002199540BB0F0BD12F8016D04F877
:10BDC000016FF0E70020F6E7FFF7C2BF70B5044649
:10BDD0008AB0084689B1931E222B23D801AD29468B
:10BDE0006CB9A9420BD0421E0B46AB4215D84B1B77
:10BDF0008D4288BF00230022C2540AB070BDB4FB3C
:10BE0000F2F302FB1346092E1C46F3B294BF303303
:10BE10005733DBB201F8013BE2E713F8014D02F8BA
:10BE2000014FE2E70020E8E7FFF7D0BF08B50320A5
:10BE3000FBF776F9BDE8084000F0B6B908B5AFF3F6
:10BE40000080F9F73BFAF9F759FD00F09FF9FAE79E
:10BE5000DFF834D0FEF702FD0C480D490D4A0023EF
:10BE600002E0D458C4500433C4188C42F9D30A4AAF
:10BE70000A4C002301E013600432A242FBD300F01D
:10BE800051FCFFF7DBFFFEE700A0002000000020D0
:10BE90004003002044EA00084003002088190020E5
:10BEA000FEE791420FD008D9891A01238B409842AE
:10BEB00008D30130C8400138704720B10130521A10
:10BEC0009040F8E700207047431E1F2B0ED80C2827
:10BED0000DDC06280DDD08280DDD0B28B4BF0A2374
:10BEE0000C23064A1060064A13607047FEE70C23D5
:10BEF000F7E70623F5E70823F3E700BFEC0200208D
:10BF0000E8020020431E1F2B07D8044B102818609E
:10BF1000034BA8BF102018607047FEE7E402002022
:10BF2000E0020020014B1860704700BFDC020020D7
:10BF300010B500F03DF9431C0AD0064C2168FEF70D
:10BF400021F8054B21681A68BDE81040FFF7A9BF2A
:10BF5000002010BDE8020020EC020020C3B2312B0B
:10BF60002DE9F04107460E4631D82C4A52F82330CD
:10BF700000F4E0641C43621C4ED02949DFF8B48011
:10BF80002046FEF784FB0546002831D0C4F3031198
:10BF9000244A52F8210004F00F0520FA05F3DB07CC
:10BFA0005FBF0123AB40034342F821301E4BD8F85A
:10BFB00000101D6830462A46FFF773FF1B490246F2
:10BFC000EBB220460968BDE8F041FEF725B900F064
:10BFD000C002C02A20D1CE2B1ED8154B00F03F0244
:10BFE00000F4E06453F822200C4B53F82230C1E7F0
:10BFF0003846012100F020F8D8F800103046082219
:10C00000FFF74FFF7F2898BF2946384688BF012198
:10C01000BDE8F04100F06EB8BDE8F081F8E7000837
:10C0200004E500082C180020E0020020DC020020BB
:10C03000BCE70008E4020020C3B2312B2DE9F04137
:10C040000D462AD8274A52F8233000F4E0641C43F6
:10C05000621C44D0244EC4F3031704F00F0856F8B2
:10C06000273023FA08F3DB0710D520492046FEF7D6
:10C070000EFB10B12046FEF721F956F827300122B9
:10C0800002FA08F223EA020346F82730052D15D8F4
:10C09000DFE805F015211B1D1F2300F0C002C02A98
:10C0A0001DD1CE2B1BD8124B00F03F0200F4E064F0
:10C0B00053F822200B4B53F82230C8E7FEE700214B
:10C0C0002046BDE8F041FEF7F1BA1021F8E7202143
:10C0D000F6E70321F4E70121F2E70921F0E7BDE8E3
:10C0E000F08100BFF8E700082C18002004E50008E4
:10C0F000BCE70008C3B2312B17D8174A52F82330D7
:10C1000000F4E0601843C0F30313042B98BF134AF4
:10C1100000F00F0098BF52F82330114A88BF002367
:10C1200052F82020A9B19A61704700F0C002C02ADD
:10C130000CD1CE2B0AD80B4B00F03F0200F4E0608C
:10C1400053F82220044B53F82230DBE74FF0FF3046
:10C15000D9E79A62704700BFF8E70008980200200C
:10C16000A0E10008BCE70008FEF7FAB8FEF7D4B873
:10C1700038B5044648B1FEF7F3F8054600F016F866
:10C18000FEF7EEF8431BA342F8D338BD08B5044BC5
:10C190002BB10448FEF7AEFF08B1AFF3008008BD35
:10C1A00000000000D0160020FEF78EB97047000096
:10C1B00010B5C4B20E2C034617D82C4951F82410E0
:10C1C00000F4E0620A43C9B2312926D8284A0E2C6D
:10C1D00052F8210017D8254A52F824201A4302F4B5
:10C1E000E0621043421C1ED010BD00F0C002C02A05
:10C1F00019D1CE2C17D81D4900F03F0003F4E0629E
:10C2000051F82010DEE703F0C002C02A2AD1174AF5
:10C2100003F03F0152F82120E0E702F0C000C028FF
:10C2200001D1CE2908D9A3F1CF02022A94BF03F687
:10C2300032704FF0FF30D7E702F03F020B4951F860
:10C2400022000B4A0E2C52F8200002D851F824206C
:10C25000C4E703F0C002C02A04D103F03F0251F842
:10C260002220BBE74FF4E062BBE700BFBCE7000859
:10C27000F8E700080A22002100F072B90A22002122
:10C2800000F06EB9024B0146186800F02DB800BFEF
:10C29000F0020020024B0146186800F085BA00BF8A
:10C2A000F002002070B50F4E0C463168054611B9FA
:10C2B00000F022FA30602146284600F01DFA431CA7
:10C2C00003D14FF0FF34204670BDC41C24F003049A
:10C2D000A042F8D0211A284600F00EFA0130F2D11F
:10C2E000EFE700BF401800202DE9F843CD1C25F0F2
:10C2F000030508350C2D38BF0C25002D064601DB43
:10C30000A94204D90C2333600020BDE8F883DFF88C
:10C31000D48000F069F8D8F800301C4644BB2946A8
:10C320003046FFF7BFFF431C044658D1D8F8004001
:10C330002746002F43D1002C4BD023683946304686
:10C3400004EB030900F0D8F9814542D121686D1A48
:10C3500029463046FFF7A6FF01303AD023682B4428
:10C360002360D8F800305A6862BBC8F800700FE04C
:10C370002268521B20D40B2A17D96119A3422560C9
:10C3800018BF5960636808BFC8F8001062514B605D
:10C39000304600F02FF804F10B00231D20F00700B9
:10C3A000C21A1CBF1B1AA350AFE76268A3420CBF9E
:10C3B000C8F800205A60EBE723466468AEE73C46C5
:10C3C0007F68B6E71A465B68A342FBD1002353603F
:10C3D000DEE70C233360304600F00CF894E705608C
:10C3E000D6E700BF44180020014800F0BFB900BFE5
:10C3F00084190020014800F0BAB900BF8419002058
:10C40000024B0A460146186800F002B8F00200200C
:10C410002DE9F041074614460D4621B9BDE8F0412B
:10C420001146FFF761BF2AB900F0BEF9254628463C
:10C43000BDE8F08100F002FA8442064602D8B4EB6F
:10C44000500FF4D821463846FFF74EFF804608B912
:10C450004546ECE7B4422246294628BF324600F062
:10C460008FF92946384600F09FF9F1E7242B2DE992
:10C47000F0478646904601D8012B06D100F04CF9D2
:10C48000162303600020BDE8F08734480D462A4695
:10C4900015F8014B065D16F00806F8D12D2C10D1C9
:10C4A0002C780126951C33F0100215D1302C0DD1BB
:10C4B0002A7802F0DF02582A08D16C78023510235E
:10C4C0000AE02B2C04BF2C78951CECE7002BF6D14E
:10C4D000302C14BF0A23082306F1004C0CF1FF3C5A
:10C4E0000022BCFBF3F9104603FB19CAA4F1300784
:10C4F000092F0FD83C46A3421BDD571C07D08145AE
:10C5000014D301D1A24511DB00FB0340012215F831
:10C51000014BEBE7A4F14107192F01D8373CEAE7BB
:10C52000A4F16107192F04D8573CE4E74FF0FF321C
:10C53000EDE7531C08D12223CEF800306046B8F155
:10C54000000FA0D0691E06E006B14042B8F1000F0E
:10C5500099D0002AF6D1C8F8001094E701E9000844
:10C5600013460A46014602480068FFF77FBF00BF36
:10C57000F00200200CB430B5174B0C1E1D689DB0A6
:10C5800008DA8B232B604FF0FF301DB0BDE8304040
:10C5900002B070474FF40273ADF8143014BF04F1C9
:10C5A000FF332346049307934FF6FF7302900690E0
:10C5B000ADF81630209A21AB02A92846019300F06D
:10C5C000A1F9431CBCBF8B232B60002CDDD0029B48
:10C5D00000221A70D9E700BFF00200200EB400B5A7
:10C5E0009CB01DAB029006906FF000410948079186
:10C5F0000491094953F8042B05910068019302A99D
:10C6000000F080F9029B00221A701CB05DF804EB68
:10C6100003B07047F00200200802FFFF884210B507
:10C6200001EB020402D98442234607D8431EA142EB
:10C6300008D011F8012B03F8012FF8E70244014656
:10C640008A4200D110BD13F8014D02F8014DF7E701
:10C6500002440346934200D1704703F8011BF9E7F7
:10C6600030B50C4D024612F8013BE85C00F00300C7
:10C67000012811F8010B2C5C04F0030408BF2033DF
:10C68000012C08BF20301B1A02D10028EBD130BD8D
:10C690001846FCE701E9000810B502461478134675
:10C6A0000132002CFAD1013B11F8012B03F8012FC4
:10C6B000002AF9D110BDC9B20346184613F8012B60
:10C6C00012B18A42F9D17047002918BF0020704783
:10C6D00010B50139034632B111F8014F03F8014B8F
:10C6E000013A002CF7D11A440021934200D110BD29
:10C6F00003F8011BF9E7000038B5064D0023044696
:10C7000008462B60FEF796FC431C02D12B6803B150
:10C71000236038BD80190020014B1868704700BFA6
:10C72000F002002070B50D4D0D4C641BA4100026C6
:10C73000A64209D10B4D0C4C01F000F8641BA4106B
:10C740000026A64205D170BD55F8043B9847013636
:10C75000EEE755F8043B98470136F2E720EA000877
:10C7600020EA000820EA000838EA0008704770470D
:10C77000034611F8012B03F8012B002AF9D1704769
:10C780000A44914200F1FF3300D1704710B511F80F
:10C79000014B03F8014F9142F9D110BD9FED010A01
:10C7A000704700BF0000C07F38B50546002941D062
:10C7B00051F8043C0C1F002BB8BFE418FFF714FE1F
:10C7C0001D4A136833B9636014602846BDE83840D9
:10C7D000FFF710BEA34208D9206821188B4201BF81
:10C7E00019685B6809182160EDE71A465B680BB1B0
:10C7F000A342FAD911685018A0420BD12068014415
:10C80000501883421160E0D118685B685360084497
:10C810001060DAE702D90C232B60D6E720682118D4
:10C820008B4204BF19685B68636004BF091821600C
:10C830005460CAE738BD00BF4418002051F8043CDA
:10C84000181F002BBCBF0B58C01870472DE9F047CC
:10C850008E681F46BE420B6882460C4690462DD815
:10C86000B1F90C2012F4906F26D06569096905EBC7
:10C870004505A3EB010905EBD5757B1C4B446D10F9
:10C880009D4238BF1D46530527D52946FFF72CFD8D
:10C89000064660B321694A46FFF772FFA38923F475
:10C8A000906343F08003A381266165614E44A5EB4C
:10C8B00009052660A5603E46BE4200D93E46206876
:10C8C00032464146FFF7AAFEA3689B1BA36023687C
:10C8D000334423600020BDE8F0872A46FFF798FD27
:10C8E00006460028E0D121695046FFF75DFF0C2382
:10C8F000CAF80030A38943F04003A3814FF0FF3012
:10C90000E9E700002DE9F04F98468B891B069DB0A2
:10C9100007460D46144610D50B6973B94021FFF741
:10C92000E3FC2860286130B90C233B604FF0FF30F6
:10C930001DB0BDE8F08F40236B61002309932023D5
:10C940008DF82930CDF80C803023DFF89C818DF8EC
:10C950002A304FF0010923469A4613F8012B0AB1F9
:10C96000252AF9D1BAEB040B0BD05B4622462946A7
:10C970003846FFF76BFF013000F0A780099A5A4450
:10C9800009929AF80030002B00F09F8000234FF0AE
:10C99000FF32CDE905230AF1010A049307938DF8CC
:10C9A00053301A935446052214F8011B4E48F3F7EE
:10C9B00007FC049AD8B9D00644BF20238DF8533021
:10C9C000110744BF2B238DF853309AF800302A2BDF
:10C9D00015D0079A544600204FF00A0C214611F852
:10C9E000013B303B092B4BD9B0B1079214E0A0EBCF
:10C9F000080309FA03F313430493A246D2E7039B07
:10CA0000191D1B680391002BBBBF5B4242F0020261
:10CA100007930793B8BF049223782E2B0AD163782B
:10CA20002A2B32D1039B1A1D1B68039243EAE3733E
:10CA300002340593DFF8C0A0217803225046F3F7B3
:10CA4000BFFB38B1049BA0EB0A0040228240134395
:10CA50000134049314F8011B24488DF82810062291
:10CA6000F3F7AEFB002836D0214B1BBB039B0733EB
:10CA700023F0070308330393099B334409936AE7C0
:10CA80000CFB02320C460120A8E700230134059379
:10CA900019464FF00A0C204610F8012B303A092AAB
:10CAA00003D9002BC6D00591C4E70CFB0121044635
:10CAB0000123F0E703AB00932A460E4B04A9384646
:10CAC000AFF30080421C0646D6D1AB895B063FF52A
:10CAD0002DAF09982CE703AB00932A46054B04A918
:10CAE000384600F079F8EDE7FDE0000807E10008BE
:10CAF000000000004DC8000803E100082DE9F047E0
:10CB0000164698468A680B69DDF820909342B8BFB4
:10CB10001346336091F8432007460C460AB10133AF
:10CB200033602368990642BF336802333360256857
:10CB300015F0060506D104F1190AE36832689B1A5C
:10CB4000AB4226DC94F843302268003B18BF012337
:10CB500092062BD404F1430241463846C8470130BF
:10CB60001ED02368226903F00603042B02BFE56888
:10CB70003368ED1AA3680CBF25EAE57500259342DA
:10CB8000C4BF9B1AED1800261A34B5421AD10020F2
:10CB900008E00123524641463846C847013003D1D8
:10CBA0004FF0FF30BDE8F0870135C6E7E1185A1CA9
:10CBB000302081F84300224494F8451082F8431055
:10CBC0000233C7E70123224641463846C8470130B1
:10CBD000E6D00136D9E700002DE9FF470F7E0C9E15
:10CBE000782F914680460C469A4601F1430207D8B9
:10CBF000622F0AD8002F00F0D180582F00F0B880A3
:10CC000004F1420684F842703AE0A7F16303152B61
:10CC1000F6D801A151F823F071CC000885CC0008AA
:10CC200001CC000801CC000801CC000801CC0008B0
:10CC300085CC000801CC000801CC000801CC00081C
:10CC400001CC000883CD0008AFCC00083DCD000822
:10CC500001CC000801CC0008A5CD000801CC0008DB
:10CC6000AFCC000801CC000801CC000845CD00087D
:10CC700033681A1D1B68326004F1420684F84230A2
:10CC800001239CE033682068191D3160060601D538
:10CC90001D6803E04506FBD5B3F90050002D03DA0B
:10CCA0002D236D4284F8433058480A2311E021684F
:10CCB0003368080653F8045B02D4490648BFADB296
:10CCC0006F2F5248336014BF0A230823002184F8D1
:10CCD00043106668A660002E05DB21682E4321F014
:10CCE000040121604BD01646B5FBF3F103FB11574D
:10CCF000C75D06F8017D2F46BB420D46F4D9082BCF
:10CD00000BD12368DF0708D5236961689942DEBF2C
:10CD1000302306F8013C06F1FF36921B2261CDF864
:10CD200000A04B4603AA21464046FFF7E7FE01302C
:10CD30004AD14FF0FF3004B0BDE8F087236843F0DC
:10CD4000200323603248782784F8457023683168CF
:10CD50001F0651F8045B02D45F0648BFADB23160D4
:10CD6000D90744BF43F0200323601DB11023ADE772
:10CD70002648E9E7236823F020032360F6E71646F8
:10CD8000BDE7336825686169181D30602E061B6891
:10CD900001D5196002E06806FBD5198000232361E4
:10CDA0001646BCE733681A1D32601E6862680021AF
:10CDB0003046F3F705FA08B1801B606063682361B1
:10CDC000002384F84330AAE72369324649464046A7
:10CDD000D0470130ADD023689B0713D4E068039B94
:10CDE0009842B8BF1846A6E7012332464946404656
:10CDF000D04701309DD00135E36803995B1AAB42FF
:10CE0000F2DCEBE7002504F11906F5E70EE1000876
:10CE10001FE1000808B5062000F02CF80120FEF7FD
:10CE200027F91F2938B505460C4604D91623036097
:10CE30004FF0FF3038BDC26B12B152F821304BB900
:10CE4000284600F031F8224601462846BDE8384021
:10CE500000F018B8012B0AD0591C03D11623036027
:10CE60000120E7E7002142F82410204698470020DF
:10CE7000E0E70000024B01461868FFF7D2BF00BF91
:10CE8000F002002038B5074D00230446084611463D
:10CE90002B60FEF7EFF8431C02D12B6803B123602F
:10CEA00038BD00BF80190020FEF7ECB8F8B52DEDB5
:10CEB000028B57EC106B55EC114B00F05DF83046CF
:10CEC000394622462B46B0EE408AF0EE608AF3F7F0
:10CED0001DFE30B90022002320462946F3F7E4FD69
:10CEE00030B9B0EE480AF0EE680ABDEC028BF8BD2E
:10CEF000FFF712FC00220023212101601046194691
:10CF0000F3F794FC41EC180BB0EE480AF0EE680A17
:10CF1000BDEC028BF8BD00BF08B52DED028BB0EE65
:10CF2000408A00F0AFF9B4EE488AF1EE10FA0FD65D
:10CF3000B5EEC08AF1EE10FA0ADCB5EE408AF1EEE9
:10CF400010FA08D1FFF7E8FB22239FED090A0360DE
:10CF5000BDEC028B08BDFFF7DFFBBDEC028B034687
:10CF600021221A600348BDE80840FFF717BC00BF44
:10CF7000000080FF04EA000853EC112B2DE9F04774
:10CF800023F0004852EA080155EC104B47D0B7494E
:10CF900025F0004A8A45A94641D85042B44E40EA9D
:10CFA000020148EAD171B142964638D8C2451F46BF
:10CFB000214605F0004C3EDCC0F28480A24200F223
:10CFC000818000F0B580354245D1BAF1000F34D1EF
:10CFD000002C234640F32A81A64A5B00002B02F175
:10CFE000FF32FADCA24B3B40002B40F09380B8F1BB
:10CFF000000F40F0DF80BEF1000F73466DDC9D4EE8
:10D000009D48801A1F2800F3F08002F21E4321FA87
:10D0100003F30AFA00FA43EA0A0381406AE0204671
:10D020002946F3F7D9FA02460B46F3F7FFFB41EC2A
:10D03000100BBDE8F08735420DD18F4A4FEACA2365
:10D040005B00002B02F1FF32CCDD5B00002B02F114
:10D05000FF32F5DCC6E7864B4FEA2A523B40A2F28C
:10D06000FF3293B34FEA2850C9F31303A0F2FF36FF
:10D0700043F48013A1EB0E00C7F3130545F48015AC
:10D08000921B0BD163E0013858D4A1EB0E04E30FDF
:10D09000013A03EB40034FEA440156D07145A3EB3C
:10D0A0000500F0D30028A1EB0E0447DB50EA04038F
:10D0B000EDD1724B4FEADC7C03EBCC0393ED000B1C
:10D0C000BDE8F08745EC104BB3E7B8F1000F71D124
:10D0D000BEF1000F734640F3B480664E5B00002B38
:10D0E00006F1FF36FADC644B9A4289DBC9F313037D
:10D0F00043F48013604CA41B1F2C4CDC06F21E452D
:10D100002EFA05F508FA04F00EFA04FE0543A1EB29
:10D110000E00B5E7584CA41A4FEA28581F2CA8F265
:10D12000FF3672DD564B9B1A01FA03F30021A3E789
:10D13000524B03EB1C7393ED000B7AE7C80F013AD7
:10D1400000EB43034FEA4101A8D1A1EB0E005A1BAB
:10D150008E4588BF02F1FF32002ABCBF08461A463E
:10D1600052EA000305D1A4E7C30F03EB42024000DB
:10D17000013EB2F5801FF7DB3F4B9E4223DBA2F559
:10D18000801242EA0C0106F2FF3641EA06530246DB
:10D1900043EC102B4DE73A4D921BA5EB06050EFA1A
:10D1A00005F518BF4FF0000E7FF478AF5A1B084604
:10D1B000D2E7304A304E4FEAC8235B00002B06F11D
:10D1C000FF36FADC8FE79B1B142B14DC06F21E41A2
:10D1D000D84002FA01F142FA03F3014343EA0C0C8E
:10D1E00063460A4643EC102B23E7254B9B1A01FAB2
:10D1F00003F300217EE71F2B13DC06F21E4120FA09
:10D2000003F302FA01F11943EAE702F21E4321FA9D
:10D2100003F30AFA04FA43EA0A03A140A1EB0E0061
:10D220002AE71749891B42FA01F1D9E7104B3B4025
:10D230007BB14FEA28500F4AA0F2FF36E30A61059E
:10D24000ECE7C9F313030B4E43F480130B251524AD
:10D2500056E7B8F1000FACD1BEF1000F054A734696
:10D260003FF73BAF15201646CFE600BFFFFFEF7F2D
:10D270000000F07FEDFBFFFF02FCFFFF08EA000863
:10D28000E2FBFFFF10EE102A32F000432FD0002AFD
:10D29000134633DBB2F1FF4F40DAB2F5000F34DB57
:10D2A0004FF0000C6448C3F31601084400F4000278
:10D2B00082F07E520A43DB1500EE102A7F3B5F4A64
:10D2C000634401F10F0CF7EE007A0CEA020230EE33
:10D2D000670A03EBD05322BBB5EE400AF1EE10FA19
:10D2E00062D1002B40F090809FED550A70479FED72
:10D2F000557ADFED537A87EE270A704770EE407A51
:10D300009FED4F7A87EE870A7047DFED4F7A60EE28
:10D31000277A6FF0180C17EE903AC3E730EE000A48
:10D320007047F0EE007A70EE277A07EE103A80EE42
:10D33000274A4648C1F55712084402F522720243B3
:10D34000002A9FED433ADFED434ADFED435ADFED1C
:10D35000433A9FED435ADFED437ADFED436A24EE13
:10D36000046AF8EEC72A26EE067AE7EE034AA7EE2D
:10D37000235AE4EE875AE5EE076AE5EE877A67EE10
:10D38000867AE6EE877A2ADDB6EE007A20EE077A14
:10D3900027EE007A77EE877A67EE847A3BBB37EE2A
:10D3A000677A30EE470A70479FED307AF6EE007AE2
:10D3B000E0EE477A20EE007A27EE277A002BF0D0B5
:10D3C00007EE903A9FED2A6ADFED2A6AF8EEE77AD7
:10D3D000A7EEC67A37EE400A97EEA60A704770EEBF
:10D3E000677A67EE847AE3B930EE670A70479FED9B
:10D3F000206ADFED206AE2EE867A37EE677A37EE52
:10D40000400A92EEA60A704707EE903A9FED180A7E
:10D410009FED187AF8EEE77A27EE800AA7EE870AE2
:10D420007047DFED136A9FED137AE2EEE67A37EE8E
:10D43000C00A92EE870A704720FB4A00F0FF7F0087
:10D4400000000000000000CC0000004C305CCFFF6A
:10D450009788173E25333A3E2549923E4FD01C3ED1
:10D46000298E633EABAA2A3FCDCCCC3EABAAAA3EC6
:10D47000D1F717378071313F2DE9F047089D0E46EF
:10D4800004460F46002B4AD194468C45B2FA82F2EC
:10D4900060D942B1C2F12003974020FA03F30CFA9D
:10D4A00002FC1F4394404FEA1C4E1FFA8CF6B7FB58
:10D4B000FEF1230C0EFB117743EA074301FB06F054
:10D4C00098420AD91CEB030301F1FF3780F0158164
:10D4D000984240F21281023963441B1AA4B2B3FB92
:10D4E000FEF00EFB103344EA034400FB06F6A642AE
:10D4F0000AD91CEB040400F1FF3380F00081A6423E
:10D5000040F2FD806444023840EA0140A41B00213F
:10D510001DB1D4400023C5E90043BDE8F0878B422C
:10D5200005D90DB1C5E9000100210846F5E7B3FAB8
:10D5300083F1002946D1B34202D3824200F2F58042
:10D54000841A66EB030201201746002DE5D0C5E9D9
:10D550000047E2E7002A40F09380A1EB0C034FEA7A
:10D560001C471FFA8CFE0121B3FBF7F607FB1630B0
:10D57000230C43EA00430EFB06F0984208D91CEB4B
:10D58000030306F1FF3802D2984200F2D0804646EB
:10D590001B1AA4B2B3FBF7F007FB103344EA0344B1
:10D5A0000EFB00FEA64508D91CEB040400F1FF3376
:10D5B00002D2A64500F2B6801846A4EB0E0440EA5B
:10D5C0000640A5E7C1F120078B4022FA07FC4CEA90
:10D5D000030C06FA01FE20FA07F426FA07F344EAE0
:10D5E0000E0400FA01F84FEA1C404FEA1449B3FB5D
:10D5F000F0FE1FFA8CF600FB1E3349EA03430EFBD4
:10D6000006F9994502FA01F20BD91CEB03030EF15E
:10D61000FF3A80F08580994540F28280AEF1020E9B
:10D620006344A3EB0909A4B2B9FBF0F300FB13991F
:10D6300044EA094403FB06F6A64208D91CEB04049D
:10D6400003F1FF3068D2A64266D9023B644443EA44
:10D650000E40A41BA0FB02E6B4427346B14652D36F
:10D660004FD05DB1B8EB030264EB090404FA07F78D
:10D6700022FA01F31F43CC40C5E9007400214CE7B6
:10D68000C2F1200120FA01F30CFA02FC26FA01F1A2
:10D69000964033434FEA1C471FFA8CFEB1FBF7F06C
:10D6A00007FB1016190C41EA064100FB0EF68E42EC
:10D6B00004FA02F408D91CEB010100F1FF382DD265
:10D6C0008E422BD902386144891B9BB2B1FBF7F61D
:10D6D00007FB161143EA014306FB0EF1994208D9F4
:10D6E0001CEB030306F1FF3814D2994212D9023E13
:10D6F00063445B1A46EA004136E73946EDE61846D0
:10D7000002E7F045ADD2BEEB020366EB0C06013832
:10D71000B146A6E74646ECE7034698E74046D3E71E
:10D72000D6467EE76444023847E708460DE7023EE6
:10D7300063442DE708B5FFF76DFB0000F8B500BFA7
:10D74000F8BC08BC9E467047F8B500BFF8BC08BCE2
:04D750009E4670473A
:10D75800000000000000344000000000000000400D
:10D768001975ADBD4F55B53F2C0FD253E410813F0D
:10D77800E5BEC26F30C1363F000000000000244003
:10D78800000000000000F03F1975ADBD4F55A53FE2
:10D798007D09151C5E10713F4FB7C67A7DC0263FC4
:10D7A80041505A4E4657006025632563256325631B
:10D7B8002563256325632563002573256325632574
:10D7C800637D0025303264253032642E2530326482
:10D7D80025630025303364253032642E25303264C9
:10D7E80025630021257325632573256300253032C1
:10D7F800643A253032643A25303264002564002CBE
:10D8080000253034580024242424002A002F413DC8
:10D81800253036642F5025645325645425303264EE
:10D8280056253034644330302025730020616C74F1
:10D838003A25646D202573002125732F25735F63B6
:10D848002530336473253033646725303364742599
:10D858003033646825303264622530356420545F83
:10D868004578743D25644320545F496E743D2564B2
:10D87800432052483D2564252520556261743D2585
:10D88800646D562C20257300212000414C54200043
:10D898004D20004E3043414C4C004F4E005758002D
:10D8A8004E4F524D414C0046554C4C005245445544
:10D8B80043454400484F525553465251000A4F4B76
:10D8C800003E000A4672657175656E6379206F7552
:10D8D80074206F662072616E67650041505253462E
:10D8E80052510052545459465251004D4F525345CB
:10D8F8004652510055415254424452000A4F4B205F
:10D90800284F6E6C792076616C6964206166746555
:10D9180072207265626F6F7429000A554152542053
:10D928006261756472617465206973206F75742013
:10D938006F662072616E6765004D4F5253455350B4
:10D9480045454400524144494F505752000A504FF0
:10D95800574552203020746F203700484F52555396
:10D968004944000A486F727573205061796C6F6181
:10D9780064204944206F7574206F662072616E6759
:10D988006500484F525553424452000A486F727519
:10D9980073204261756472617465206F7574206FBD
:10D9A800662072616E6765005254545942445200B1
:10D9B8000A52545459204261756472617465206F2B
:10D9C8007574206F662072616E67650052545459F1
:10D9D8005348494654000A525454592053686966BA
:10D9E8007420313D3237302C20323D353430202EF2
:10D9F8002E2E487A005254545942495453000A5220
:10DA080054545920626974732037206F722038008B
:10DA18005254545953544F50000A52545459207375
:10DA2800746F706269747320312C20312E35206F29
:10DA3800722032004150525353534944000A415016
:10DA4800525320535349442030202D203135004172
:10DA580050525353594D424F4C0041505253544128
:10DA6800424C4500484F4C444F46460041505253A3
:10DA780043414C4C000A4E6F2043414C4C5349479C
:10DA88004E20646566696E6564005254545943417A
:10DA98004C4C00415052534D5347000A4E6F204D95
:10DAA80045535341474520646566696E656400487F
:10DAB8004F525553454E41424C45000A4572726FCC
:10DAC800720052545459454E41424C4500415052FF
:10DAD80053454E41424C45004D4F525345454E41EA
:10DAE800424C4500415052534D4F4445004D4F5212
:10DAF80053454D4F4445004150525348414200411F
:10DB08005052534D4943450048454C5000417661B9
:10DB1800696C61626C6520636F6D6D616E64730022
:10DB2800636F6D6D616E643C53504143453E706157
:10DB380072616D657465723C454E5445523E2028AD
:10DB4800636F6D6D616E647320616C6C776179735E
:10DB580020776974686F75742053504143452129B3
:10DB68000064697370202873657420706172616D38
:10DB780065746572732900686F72757366727120B7
:10DB880066727175656E63792028696E20487A2CF3
:10DB9800206B487A206F72204D487A290061707294
:10DBA800736672712066727175656E63790072743E
:10DBB80074796672712066727175656E6379006D2D
:10DBC8006F7273656672712066727175656E6379BE
:10DBD80000686F6C646F66662074696D65202874D0
:10DBE800696D6520696E207365632E206D696E2EE0
:10DBF8002031352900686F727573656E61626C65D6
:10DC080020782028302D64697361626C6520312D7D
:10DC1800656E61626C65290061707273656E616220
:10DC28006C6520782028302D64697361626C6520EA
:10DC3800312D656E61626C65290072747479656E48
:10DC480061626C6520782028302D64697361626C8C
:10DC58006520312D656E61626C6529006D6F727388
:10DC680065656E61626C6520782028302D64697363
:10DC780061626C6520312D656E61626C6529006199
:10DC88007072736D736720636F6D6D656E74202895
:10DC98006170727320636F6D6D656E74206D61784D
:10DCA80020313230206368617229006170727363B9
:10DCB800616C6C2063616C6C20286D617820362063
:10DCC8006368617229007274747963616C6C206393
:10DCD800616C6C20286D6178203135206368617231
:10DCE8002900686F727573696420782028506179FB
:10DCF8006C6F61642049442900686F7275736264AF
:10DD08007220782028686F7275732062617564725A
:10DD180061746529007274747962647220782028AD
:10DD28007274747920626175647261746529007215
:10DD3800747479626974732078202837206F722090
:10DD48003829007274747973746F702078202831C0
:10DD58002C20312E35206F7220322900727474798C
:10DD68007368696674207820287368696674203D32
:10DD78002078202A20323730487A2900617072735F
:10DD880073736964207820283020746F2031352916
:10DD9800006170727373796D626F6C2078202873DC
:10DDA800796D626F6C2066726F6D2061707273207E
:10DDB8007461626C652900617072737461626C656C
:10DDC80020782028617072732073796D626F6C20DF
:10DDD8007461626C65202F206F7220290061707257
:10DDE800736D6F646520782028302D6E6F726D61B9
:10DDF8006C2C20312D77782900617072736861620C
:10DE080020782028302D6F66662C20312D6F6E29E2
:10DE180000617072736D69636520782028302D6FFA
:10DE280066662C20312D6F6E29006D6F72736573D5
:10DE3800706565642078202857504D29006D6F72F1
:10DE480073656D6F646520782028302D7265647560
:10DE58006365642C20312D66756C6C2900726164D1
:10DE6800696F70777220782028302D372900756106
:10DE7800727462647220782028313230302C323447
:10DE880030302C343830302C393630302C3139326F
:10DE980030302C33383430302C35373630302C375E
:10DEA800363830302C31313532303029004449533E
:10DEB800500053657420706172616D65746572738A
:10DEC80000415052533A2000415052532043414C94
:10DED8004C3A200041505253204672657175656E68
:10DEE80063793A2000204D487A004150525320432C
:10DEF8006F6D6D656E743A20004150525320535334
:10DF080049443A2000415052532053796D626F6C56
:10DF18003A2000415052532053796D626F6C20545F
:10DF280061626C653A200041505253204D4F444580
:10DF38003A200041505253204841423A2000415073
:10DF48005253204D49432D453A2000525454593AD2
:10DF58002000525454592043414C4C3A200052540A
:10DF68005459204672657175656E63793A2000527E
:10DF780054545920426974733A2000525454592019
:10DF880053746F7020426974733A20005254545984
:10DF98002042617564726174653A20005254545984
:10DFA8002053686966743A2000484F5255533A2006
:10DFB80000484F5255532049443A2000484F525583
:10DFC80053204672657175656E63793A2000484F33
:10DFD8005255532042617564726174653A20004D50
:10DFE8004F5253453A20004D4F52534520467265D3
:10DFF8007175656E63793A20004D4F525345205331
:10E00800706565643A20004D4F525345204D6F644A
:10E01800653A2000524144494F20504F5745523AE3
:10E028002000484F4C44204F46463A200055415264
:10E03800542062617564726174653A20000A3E3F3B
:10E048000052533431206261736564207061796CC9
:10E058006F616420666F722053544D3332463130FD
:10E0680030002D2E2D2E002E2E2D2E002E2D2E2E54
:10E07800002E2D2D2E002D2D2E2D002D2E2E2D0077
:10E088002D2E2D2D002D2D2D2D2D002E2D2D2D2D10
:10E09800002E2E2D2D2D002E2E2E2D2D002E2E2E27
:10E0A8002E2D002E2E2E2E2E002D2E2E2E2E002D15
:10E0B8002D2E2E2E002D2D2D2E2E002D2D2D2D2EDC
:10E0C800002E2D2E2D2E2D00504E41424C00524D2B
:10E0D8004300474741000D0A006E616E00696E6695
:10E0E800006F7666002D256C642E25302A6C64003E
:10E0F8002D256C6400232D302B2000686C4C0065A6
:10E10800666745464700303132333435363738395B
:10E11800414243444546003031323334353637388E
:10E1280039616263646566000C0012001800000122
:10E138000201040302040810040040000004000067
:10E14800000052C701000080000084CB01000000DD
:10E1580002003004040060080800900C1000C01091
:10E168002000F014400020198000501D000180217B
:10E178000002B0250004002A0008302E001060328A
:10E18800002090360040C03A0080F03E0000214355
:10E19800000052470000844B01000000020000000C
:10E1A800040000000800000010000000200000002B
:10E1B8004000000080000000000100000002000094
:10E1C800000400000008000000100000002000000B
:10E1D8000040000000800000A0860100400D030000
:10E1E800801A060000350C0040420F0080841E0093
:10E1F80000093D0000127A000024F40000366E0188
:10E208000048E801006CDC02000000000102030481
:10E2180000000000000000000102030406070809CE
:10E228000400000000300140120500000F0000004B
:10E2380000300140120500001000000000300140CD
:10E248001205000019000000003800401205000007
:10E258001C0000000038004012050000FFFFFFFF0F
:10E268000000000000000000010000000030014034
:10E2780012050000050000000030014012050000F2
:10E288001300000000300140120500001A000000D1
:10E2980000380040120500001D0000000038004052
:10E2A80012050000FFFFFFFF000000000000000053
:10E2B8000600000000300140120500000B000000BD
:10E2C8000030014012050000140000000030014039
:10E2D800120500001E000000003800401205000072
:10E2E800220000000038004012050000FFFFFFFF79
:10E2F800000000000000000007000000003001409E
:10E30800120500000C00000000300140120500005A
:10E318001500000000300140120500001F00000039
:10E3280000380040120500002300000000380040BB
:10E3380012050000FFFFFFFF0000000000000000C2
:10E348000000000000440040120700000600000022
:10E35800008000401208000006010000004800404C
:10E36800120700000B0000000038014012070000EF
:10E378001400000000380140120700001D000000D2
:10E3880000800040120800001D0100000048004005
:10E3980012070000FFFFFFFF000000000000000060
:10E3A8000100000000440040120700000C000000BB
:10E3B80000380140120700000F000000004800402C
:10E3C8001207000011000000008000401208000041
:10E3D800110100000048004012070000130000006F
:10E3E80000380140120700001C00000000800040B7
:10E3F800120800001E00000000480040120700003C
:10E40800FFFFFFFF00000000000000000300000005
:10E418000080004012080000030100000044004092
:10E42800120700000A00000000380140120700002F
:10E438000F00000000440040120300001700000015
:10E4480000380140120700001A0000000080004058
:10E45800120800001B0000000048004012070000DE
:10E468002000000000800040120800002B0000007F
:10E478000048004012070000FFFFFFFF00000000F7
:10E4880000000000020000000080004012080000A8
:10E4980002010000004400401207000009000000CB
:10E4A8000038014012070000160000000038014043
:10E4B800120700001A000000004800401207000080
:10E4C8001B0000000080004012080000210000002E
:10E4D80000800040120800002400000000480040AE
:10E4E800120700002A000000004800401207000040
:10E4F800FFFFFFFF00000000000000000000000018
:10E5080000000040128100000100000000000040EF
:10E51800120101000101000000400140128E1000AC
:10E52800020000000000004012810100020100000A
:10E5380000400140128E000003000000000000406F
:10E54800120102000301000000400140120E010008
:10E5580005000000000000401281000006000000D5
:10E5680000440140128E000007000000002C01400A
:10E578001281100008000000002C014012810000E8
:10E5880009000000002C0140120101000A000000EF
:10E59800002C0140128101000B000000002C0140FA
:10E5A800120102000F00000000000040128100006C
:10E5B80010000000002C01401201110011000000A1
:10E5C800002C0140128111001300000000000040DF
:10E5D800120101001600000000440140128E1000D4
:10E5E8001800000000440140128E00001A000000CC
:10E5F80000000040128101001B00000000000040E4
:10E60800120102001D000000002C014012811000C0
:10E618001D01000000400140128E10001E00000085
:10E62800002C0140120111001E01000000400140B1
:10E63800128E00001F000000002C01401281110002
:10E648001F01000000400140120E0100FFFFFFFF04
:10E65800000000000000000000000000000004505E
:10E6680003800200010000000000045003000300C2
:10E6780002000000000004500380030002010000B3
:10E688000001045003800300030000000000045050
:10E69800030004000301000000010450030004000B
:10E6A800040000000000045003800400040100007E
:10E6B800000104500380040005000000000004501D
:10E6C80003000500050100000001045003000500D7
:10E6D8000600000000000450038005000601000049
:10E6E80000010450038005000700000000000450EA
:10E6F80003000600070100000001045003000600A3
:10E708001000000000000450038007001001000002
:10E7180000010450038007001100000000000450AD
:10E728000300080011010000000104500300080064
:10E7380020000000000004500380000020010000B9
:10E748000001045003800000210000000000045074
:10E758000300010021010000000104500300010032
:10E768002200000000000450038001002201000084
:10E778000001045003800100230000000000045041
:10E7880003000200230100000001045003000200FE
:10E79800240000000000045003800600240100004B
:10E7A8000001045003800600FFFFFFFF0000000087
:10E7B800000000000000000001000000020000004E
:10E7C800030000000400000005000000060000002F
:10E7D80007000000100000001100000020000000E9
:10E7E8002100000022000000230000002400000097
:10E7F800000000000100000002000000030000000B
:10E8080004000000050000000600000007000000EA
:10E8180008000000090000000A0000000B000000CA
:10E828000C0000000D0000000E0000000F000000AA
:10E83800100000001100000012000000130000008A
:10E84800140000001500000016000000170000006A
:10E8580018000000190000001A0000001B0000004A
:10E868001C0000001D0000001E0000001F0000002A
:10E87800200000002100000022000000230000000A
:10E8880024000000260000002700000028000000E7
:10E89800290000002A0000002B0000002C000000C6
:10E8A8002D0000002E0000002F0000004000000096
:10E8B80041000000430000000000001000000000BC
:10E8C800001000000600070008000000000000001B
:10E8D800000000003BB10008F1B100081FB10008BA
:10E8E8004FB40008F5B0000829B6000805B10008C3
:10E8F8001BB900083DB90008002020202020202056
:10E9080020202828282828202020202020202020D7
:10E9180020202020202020202088101010101010E7
:10E928001010101010101010100404040404040433
:10E9380004040410101010101010414141414141CD
:10E9480001010101010101010101010101010101AF
:10E9580001010101101010101010424242424242BF
:10E96800020202020202020202020202020202027F
:10E978000202020210101010200000000000000027
:10E98800000000000000000000000000000000007F
:10E99800000000000000000000000000000000006F
:10E9A800000000000000000000000000000000005F
:10E9B800000000000000000000000000000000004F
:10E9C800000000000000000000000000000000003F
:10E9D800000000000000000000000000000000002F
:10E9E800000000000000000000000000000000001F
:10E9F800000000000000000000000000000000000F
:10EA0800000000000000000000000000000000807E
:08EA18007817FF7F01000000E8
:10EA20002DBE0008C10C0008F9360008955B0008EF
:08EA300071A5000859B60008A9
:0CEA38009D0C0008B937000849A6000832
:10EA440002000300050007000B000D001100130075
:10EA540017001D001F00250029002B002F00350082
:10EA64003B003D004300470049004F00530059005C
:10EA74006100650067006B006D0071007F0083001A
:10EA840089008B00950097009D00A300A700AD00AE
:10EA9400B300B500BF00C100C500C700D300DF004C
:10EAA400E300E500E900EF00F100FB0001010701CC
:10EAB4000D010F01150119011B0125013301370156
:10EAC40039013D014B0151015B015D017B017F0176
:10EAD4008501F502F90201030503000080E0000846
:10EAE400B8E000086AE00008BFE00008C7E00008DA
:10EAF4006FE00008C5E00008B2E00008C0E00008CC
:10EB04009AE000087FE0000874E0000890E0000844
:10EB1400C6E000088FE0000879E000087EE0000805
:10EB24006BE00008B9E0000891E0000884E0000808
:10EB3400A6E0000889E0000883E0000888E00008F7
:10EB4400BEE000088DE0000893E0000899E00008AA
:10EB54009FE00008A5E00008ABE00008B1E0000871
:10EB6400B7E00008BDE00008C3E0000891D8000841
:10EB7400C9E00008B5620611020008012292B562DC
:10EB84000611020008002191B56206242400FFFF4B
:10EB9400060300000000102700000500FA00FA0038
:10EBA40064002C0100000000102700000000000099
:10EBB40000004DDBB562068A090000010000210057
:10EBC400112006F24F00000080250000FFFF000026
:10EBD4000100000001000000010000000000803F6F
:10EBE4004000000001000000010000000A000000D5
:10EBF4000F000000FF000000050000007D00000081
:10EC040064000000E093040001010000B60300006A
:10EC14000100000000000C42000040400100000020
:10EC2400E0930400010000000101000040771B0094
:10EC3400E20400000100000004000000FFFFFFFFE9
:10EC4400E80300000100000028000000CD4CD94377
:10EC54000200000000000040070000001027000030
:10EC6400CD4CD94301000000010000002F4F015793
:10EC74004944453200415042433431000B00000006
:10EC84000040D843010100006400000000010000BE
:10EC9400CDCCDA43010000000500000001010000B2
:10ECA400FFFFFFFF010000000700000000960000C6
:10ECB400010101001000000000000000000000003D
:10ECC400000000000000000001000000000000003F
:10ECD400000000000000000000000048000400489C
:10ECE40000080048000C0048001C0048FFFFFFFF1C
:10ECF400003002400000000000000000000000009E
:10ED040000000000000000000000000000000000FF
:10ED14000100000000093D0088190020E8030000FC
:10ED240008000000080000000A0000000A000000BB
:10ED3400F40200200000000048180020B018002051
:10ED4400181900200000000000000000000000006E
:10ED540000000000000000000000000000000000AF
:10ED6400000000000000000000000000000000009F
:10ED7400000000000000000000000000000000008F
:040000050800BE51E0
:00000001FF
